:020000040800F2
:100000007830002001010008F91A0008551900088D
:100010005B1A000893100008472B0008000000003E
:10002000000000000000000000000000251F000884
:100030009514000800000000811B00083121000811
:100040001B0100081B0100081B0100081B01000820
:100050001B0100081B0100081B0100081B01000810
:100060001B0100081B0100081B0100081B01000800
:100070001B0100081B0100081B0100081B010008F0
:100080001B0100081B0100081B0100081B010008E0
:100090001B0100081B0100081B0100081B010008D0
:1000A0001B0100081B0100081B0100081B010008C0
:1000B000952100081B0100081B0100081B01000816
:1000C0001B0100081B0100081B0100081B010008A0
:1000D0001B0100081B010008A52800081B010008DF
:1000E0001B0100081B0100081B010008DFF80CD0F1
:1000F00000F080FE00480047B96200087830002018
:100100000648804706480047FEE7FEE7FEE7FEE7B1
:10011000FEE7FEE7FEE7FEE7FEE7FEE73521000823
:10012000ED000008A0F14101192900D820307047E6
:1001300040EA01039B0703D009E008C9121F08C069
:10014000042AFAD203E011F8013B00F8013B521EE9
:10015000F9D27047D2B201E000F8012B491EFBD260
:1001600070470022F6E710B513460A4604461946C2
:10017000FFF7F0FF204610BD421E12F8013F002B92
:10018000FBD111F8013B02F8013B002BF9D170477C
:1001900030B505462A460B4612F8010B13F8014B01
:1001A00008B1A042F8D01CB1002802D06D1CF1E7C4
:1001B000284630BD421C10F8011B0029FBD1801AD3
:1001C000704710B5002200E0521C835C8C5CA34297
:1001D00001D1002BF8D1D8B2E1B2401A10BD0346CC
:1001E00011F8012B00F8012B002AF9D118467047AD
:1001F00030B505460020034600E05B1C934205D263
:10020000EC5CC85C201A01D1002CF6D130BD000096
:1002100070B500B91068002512E00B4602E0A64256
:1002200003D05B1C1C78002CF9D1E3B22B4305D022
:100230002CB125B1002100F8011B04E00546401C4B
:100240000678002EE9D11060284670BD004ADFE72D
:10025000B00100202DE9FF4F087881B09946FF28B2
:1002600005D0491C2D2804D00024002308E00023D9
:100270000BE00124F9E703EB830300EB4303491C84
:100280000878FF28F7D104B15B4200200090147871
:1002900001462D2C01D02B2C04D1521C2D2C12D018
:1002A0000024009400251678FF2E0ED00A24A0FB0F
:1002B00004C801FB0481002700FB0711521C16EB48
:1002C0000C006941EFE70124EBE7994450EA010291
:1002D0000ED00024AA4D2646DFF8A88200F04AFD81
:1002E00082468B46B9F1000009DAC9F100071BE02C
:1002F00001980021C0E9001105B0BDE8F08F074664
:1003000012E0F80707D022462B463046414600F05F
:100310002AFA0646884622462B461046194600F021
:1003200022FA04460D467F10002FEAD1B9F1000FE2
:10033000324643465046594602DA00F0ACFC01E032
:1003400000F011FA009A0AB181F00041019AC2E965
:100350000001D1E72DE9FF4F1F468DB0D7E90146D7
:100360004FF0FF382E2045464FF000090B90B96939
:100370006D1C0E988847396A824688470028F6D156
:10038000BAF1FF3F0AD024F4D064002E11DDBAF197
:100390002B0F08D0BAF12D0F0BD102E0404611B05F
:1003A000ABE744F48064B9696D1C0E9888478246B7
:1003B000761E6946600501D52D2000E02B208DF8C2
:1003C000000001F1010B0DF1200809E0B9696D1C75
:1003D0000E98884782460F9844F40074761E056094
:1003E000002E02DDBAF1300FF0D00B998A453ED1D4
:1003F00044F0800406E00F99681CA9F1010944F457
:1004000000740860B9696D1C761E0E988847824694
:100410003028F0D02BE00B998A4505D1200603D473
:1004200044F08004761E18E0504602F09BFD08B3AD
:100430000DF11301761E44F400748B4508D2AAF125
:1004400030000BF8010B200607D5A9F1010003E0ED
:10045000200602D409F101008146A00502D50F99BA
:10046000681C0860B9696D1C0E9888478246002E8A
:10047000D1DC53E0002E51DDBAF1650F02D0BAF1A4
:10048000450F4BD1A00549D5B9696D1C24F44074C2
:10049000761E0E9888478246002E0CDD2B2804D04D
:1004A000BAF12D0F07D144F48074B9696D1C0E9810
:1004B00088478246761EE00501D52D2100E02B21DC
:1004C00008F8011BCDF82C8021E00DF12901761EE2
:1004D00044F4007488450CD2AAF1300010F0FF00FB
:1004E00088F8000002D10B99884509D908F1010864
:1004F00006E0E00501D5244801E042F20F70814694
:10050000B9696D1C0E98884782460F980560002EC9
:1005100004DD504602F026FD0028D6D1F9690E9878
:100520008847FF208BF8000088F800000020069024
:1005300007904B466A4608A906A8FFF78BFEA00560
:1005400002D46FF001002AE714F0240F0AD0E0076C
:1005500014D1DDE906123868031D3B600068C0E96C
:1005600000120BE0DDE9060100F028FC0146E0077F
:1005700004D13868021D3A600068016028460EE721
:10058000000024400000F03FF1D8FFFF2DE9F05FAC
:1005900093460F4680460446002602F0C7FBD0F87B
:1005A0000090824614F8015B2DB100F015FA006846
:1005B000405DC007F6D12B2D02D02D2D1AD0641E20
:1005C0000021CAF800105A463946204600F031FA98
:1005D000014627B13868A04201D1C7F80080DAF897
:1005E0000000022809D0CAF80090700505D54842DD
:1005F000BDE8F09F46F48066E2E70846F8E770B58C
:10060000064602F093FB046805460A2200213046A4
:1006100000F0ACFA2C6070BD2DE9FE4F804681EAF7
:100620000300C00F0C46009021F0004123F000456C
:10063000B8EB0200A94105D24046214690461C462F
:100640000B46024623F00040104347D0270DC7F366
:100650000A00C3F30A510290401A019040286BDA55
:10066000C3F3130040F4801B0098924620B100238E
:10067000D2EB030A63EB0B0B01985946C0F1400221
:10068000504600F078F906460D4650465946019A04
:1006900000F090F910EB08006141002487EA115244
:1006A00084EAE7731A4340D0009A62B3019A012AA0
:1006B0004FEA075215DC001B61EB02014FF00042CC
:1006C00002EA0752CDE90042001C41F58011324692
:1006D0002B4600F092FA03B0BDE8F08F4046214669
:1006E000F9E7001B61EB0201001C41F580130018C3
:1006F0005B412018A2F5001747EB030140EAD570D3
:10070000B6196D4111E06D084FEA360645EAC0752D
:100710004FEA0752001B61EB0201001C41F58011FA
:1007200049084FEA30000019514132462B4603B0C8
:10073000BDE8F04F00F052BA0098012240000023BB
:10074000D0EB020263EBE073009821464FEAE074BD
:10075000B8EB000061EB0401E9E783F000435BE7DD
:1007600081F0004158E72DE9FE4F81EA030404F0CF
:10077000004421F0004100944FF0000B23F00043AF
:1007800050EA01045ED052EA03045BD0C3F30A547A
:10079000C1F30A552C44A4F2F3340194A0FB025493
:1007A000C1F3130141F48011C3F3130343F4801325
:1007B00001FB024400FB034E840A970A44EA815479
:1007C00047EA8357A4FB076802958D0A05FB078556
:1007D0004FEA932C04FB0C542705029D4FEA065860
:1007E00047EA1637B5EB08056EEB070C870E920E3D
:1007F00047EA811742EA8312A7FB0201B6EB0B011D
:1008000064EB00042B0D43EA0C335E1844EB1C50E0
:10081000DA465146E7FB0201C5F313044FEA0B33F6
:1008200043EA14534FEA0432019C43EA0603A4F15D
:100830000C040294009CCDE900B400F0DEF903B092
:10084000BDE8F08F00200146F9E770B5C1F30A5208
:1008500001F000450024C1F3130140F2FF3341F4DD
:1008600080119A4201DA002070BD40F233439A426F
:10087000A2F2334203DC524200F08CF800E09040D8
:100880002C43F1D0404270BD30B5041E71F100041C
:1008900004DB4FF00044404264EB0101141E73F18D
:1008A000000405DB1C464FF00043524263EB040397
:1008B0008B4208BF824230BD30B5041E71F1000486
:1008C00004DB4FF00044404264EB0101141E73F15D
:1008D000000405DB1C464FF00043524263EB040367
:1008E000994208BF904230BD30B50B46014600200A
:1008F0002022012409E021FA02F59D4205D303FAE2
:1009000002F5491B04FA02F52844151EA2F1010262
:10091000F1DC30BD2DE9F05F0546002092469B4694
:1009200088460646814640241BE028464146474605
:10093000224600F02FF853465A46C01A914110D370
:1009400011461846224600F016F82D1A67EB0108EA
:100950004F4622460120002100F00DF817EB000958
:100960004E41201EA4F10104DFDC484631462A46F0
:100970004346BDE8F09F202A04DB203A00FA02F14A
:10098000002070479140C2F1200320FA03F319437D
:1009900090407047202A04DB203A21FA02F000211F
:1009A000704721FA02F3D040C2F12002914008437F
:1009B00019467047202A06DBCB17203A41FA02F08D
:1009C00043EAE07306E041FA02F3D040C2F12002AC
:1009D000914008431946704700487047E0D8000826
:1009E00010B50446FFF7F8FF0068005D00F0010055
:1009F00010BD426842B1016811F8013B23B1521E9B
:100A0000C0E90012184670470121C160881E704776
:100A100042685AB1C368016843B983688B4205D004
:100A2000491E521CC0E90012002070474FF0FF30F1
:100A300070472DE9F05F82460078002715468B4607
:100A40000AF10104B946302801D09DB113E014F831
:100A5000010B0127782803D0582801D045B10AE0BE
:100A60000DB1102D07D10027102514F8010B02E05D
:100A7000082500E00A250026B0460EE005FB080028
:100A800005FB06F1012701EB10461FFA80F8B6F5C9
:100A9000803F00D3B94614F8010B294600F0BCF999
:100AA0000028EBDABBF1000F05D00FB1641E00E0A7
:100AB0005446CBF80040B9F1000F06D002F036F9E9
:100AC00002210160C81EBDE8F09F48EA0640FAE72F
:100AD0000FB4002300B589B00CA900910B996FF0F9
:100AE0000042CB601E4B06931E4B07930423CDE9B7
:100AF00001321D4A089202466B460020FFF72AFC8D
:100B000009B05DF814FB70B586B006464FF0FF30B3
:100B10000091CDE90101002015460C4604903246B3
:100B2000694604A8FFF7D4FF03460498211825B1AD
:100B300008B10A4600E022462A6000280DD0002BAA
:100B400002DD0098884208D0081B0094CDE901041A
:100B50003246694604A8FFF7BBFF06B070BD00002F
:100B6000F3090008110A0008E10900082DE9F0471F
:100B700091460F4680460446002614F8015B2DB1CD
:100B8000FFF72AFF0068405DC007F6D12B2D02D089
:100B90002D2D18D0641E4A4639462046FFF749FFDE
:100BA00027B13968A14201D1C7F8008071054FF023
:100BB00002040BD54042002803DD02F0B7F80460C0
:100BC000A007BDE8F08746F48066E4E70028F8DA7D
:100BD00002F0ACF804606FF00040F2E710B5141EAC
:100BE00073F1000408DA401C41F1000192185B41E6
:100BF0001A4301D120F0010010BD2DE9F04D9246BD
:100C00009B4611B1B1FA81F202E0B0FA80F22032D3
:100C10009046FFF7B0FE04460F4640EA0A0041EA5C
:100C20000B0153465A46084313D0114653EA0100BC
:100C300019D0C8F140025046FFF7ACFE05460E46FB
:100C4000504659464246FFF796FE084305D001201C
:100C500004E020463946BDE8F08D0020054346EA11
:100C6000E0762C4337430A986305E40AA0EB0800BA
:100C70000022FD0A44EA47540A3002D5002001460A
:100C8000E9E7010510196941DDE9084500196941E5
:100C9000BDE8F04DA2E72DE9F04D81EA030404F030
:100CA000004B21F0004514464FF0000A23F00041AC
:100CB00050EA050220D054EA01021DD0C5F30A57BC
:100CC0000246C5F31303C1F31300C1F30A5640F4FF
:100CD000801543F48013A7EB0608101BD64608F2D4
:100CE000FD3873EB050002D308F1010801E092180A
:100CF0005B41B8F1000F03DA00200146BDE8F08D3A
:100D000000204FF48011064684460EE0171B73EB5B
:100D1000050705D3121B63EB050306434CEA010CE0
:100D200049084FEA300092185B4150EA0107EDD1C3
:100D300052EA030012D082EA040083EA0501084364
:100D400005D0101BAB4106D20122002306E0002291
:100D50004FF0004302E06FF0010253101AEB06005F
:100D60004CEB085110EB0A0041EB0B01BDE8F04DD4
:100D7000FFF734BF0EB540F2334202920022CDE9B4
:100D800000221346FFF739FF03B000BDC1F30A523A
:100D9000C1F3130140F2FF3341F480119A4202DAA9
:100DA00000200146704740F233439A42A2F2334298
:100DB00002DC5242FFF7EEBDFFF7DDBD01F000435C
:100DC00030B421F0004150EA010206D00A0DA2F52C
:100DD0006072C1F31301002A02DC30BC00207047AE
:100DE000440F44EAC104C100E01830BC00EBC2501B
:100DF00000F020B8064C074D06E0E06840F0010323
:100E000094E8070098471034AC42F6D3FFF772F924
:100E1000F0D9000810DA00083A2800D2303820F063
:100E20002002412A01D3A2F13700884201D34FF0BA
:100E3000FF3070470029A8BF7047401C490008BF19
:100E400020F00100704710B4B0FA80FC00FA0CF0FA
:100E500050EA010404BF10BC704749B1CCF1200432
:100E600021FA04F411FA0CF118BF012121430843BF
:100E7000A3EB0C01CB1D4FEA00614FEA102042BFEB
:100E8000002010BC704700EBC35010440029A4BFE1
:100E900010BC7047401C490008BF20F0010010BC86
:100EA000704770B58C1810F8015B15F0070301D17D
:100EB00010F8013B2A1106D110F8012B03E010F8BD
:100EC000016B01F8016B5B1EF9D12B0705D40023E0
:100ED000521E0DD401F8013BFAE710F8013BCB1A82
:100EE000921C03E013F8015B01F8015B521EF9D577
:100EF000A142D8D3002070BD10B50020064908706B
:100F00004FF400710448401CFFF72BF90020024900
:100F1000A1F8020210BD0000C001002010B54FF47E
:100F200000710448FFF71DF900200249491EA1F88D
:100F3000020210BDC101002010B50A48007878B93E
:100F40000848B0F8020200280ADD07A000F02AFDD8
:100F50000448B0F80212401C00F052FDFFF7CCFF2D
:100F600010BD0000C0010020CEB4B4A6C0EDCAFD83
:100F7000BEDD3A0D0A00000070B504460D460120A2
:100F8000034908702946204601F0D0FD70BD0000DD
:100F9000C001002070B504462046FFF70BF985B26A
:100FA00029462046FFF7E8FF70BD000001490870A0
:100FB00070470000C001002000487047C1010020B8
:100FC0000148B0F802027047C001002030B5034666
:100FD000002006E01C5C00EB02154D5D6C401C54CB
:100FE000401C1028F6DB30BD2DE9F04106460F46C7
:100FF00015462A4639463046FFF7E8FF304600F0EE
:1010000022FA304600F038FA6C1E0EE022463946CD
:101010003046FFF7DBFF304600F0B8F9304600F00D
:1010200012FA304600F028FA641E012CEEDA002293
:1010300039463046FFF7CAFFBDE8F0812DE9F0419F
:1010400006460F461546002239463046FFF7BEFFDA
:1010500001240EE0304601F05DF8304601F040F822
:10106000304600F0FCFC224639463046FFF7AEFF22
:10107000641C681EA042EDDA304601F04BF83046A1
:1010800001F02EF82A4639463046FFF79FFFBDE8AB
:10109000F08100BFFEE700000148008870470000B3
:1010A0002000002000487047C40500207CB504469D
:1010B0000E46154632462146684600F0FBFB9DF879
:1010C000000060B1002006E0BDF802100144615C40
:1010D0002954411CC8B2BDF804108142F4DC2846F2
:1010E0007CBD3CB504460D462A462146684600F0C4
:1010F000E1FBBDF804003CBD01460A7802F00F0098
:101100007047000010B504200849088000200849F5
:1011100008804FF400710748FFF723F8054800786E
:1011200040F040000349087010BD0000200000207E
:1011300022000020C40500200149487070470000CB
:10114000C405002018B50446200A8DF80000E0B25E
:101150008DF8010002226946104604F0B1FE18BD68
:101160002DE9F04380460D46914647480488012604
:1011700046480088A8EB0007002F01DABDE8F0839D
:101180000D2F06DA4248005D40EA07104049085535
:101190002DE0B7F5867F0FDA3D49095D41F0D001BA
:1011A0003B4A1155A7F10D01C8B23146721C96B2E7
:1011B0002144374A50541AE04FF6FF70874216DA3E
:1011C0003349095D41F0E001314A1155A7F20D1193
:1011D00088B2030A3146721C96B221442C4A5354F9
:1011E0003146721C96B22144294A505400BF012D49
:1011F00000DAC3E70D2D06DA2548005DE9B20843A1
:10120000234908552DE0B5F5867F0FDA2049095DA1
:1012100041F00D011E4A1155A5F10D01C8B231462C
:10122000721C96B221441A4A50541AE04FF6FF70CD
:10123000854216DA1649095D41F00E01144A11552E
:10124000A5F20D1188B2030A3146721C96B22144F0
:101250000F4A53543146721C96B221440C4A5054E2
:1012600000BFA11988B22A46494604F029FE701928
:1012700086B2054800883044034908800348A0F836
:10128000008000BF7AE7000020000020220000203C
:10129000C405002038B505460C46FF2C07DCE0B23B
:1012A00000906A4601212846FFF75AFF0BE0200A0A
:1012B0008DF80000E0B28DF801006A460221284650
:1012C000FFF74EFF00BF38BD2DE9F04107460C4641
:1012D0002046FEF76FFF85B2A846404601F058FD54
:1012E0000646002003E0215C3154411C88B2A8422C
:1012F000F9DB324629463846FFF732FF304601F027
:1013000019FDBDE8F081000070B505460C4609489E
:101310000688FF2008498855711C88B22246294654
:1013200004F0CEFD03480188601C08440149088090
:1013300070BD000020000020C40500202DE9F04110
:1013400006463046FEF736FF84B22746384601F09F
:101350001FFD0546002003E0315C2954411C88B282
:10136000A042F9DB21462846FFF7CEFF284601F0D0
:10137000E1FCBDE8F08100000349097841EA001171
:10138000014A117070470000C4050020F8B50446FA
:10139000002555E0207809F0AFFF0646607809F097
:1013A00091FF4640A07809F09AFF4640E07809F0A6
:1013B00082FF46408DF80060207809F07CFF0646E9
:1013C000607809F099FF4640A07809F07BFF46401D
:1013D000E07809F084FF46408DF80160207809F03C
:1013E0007EFF0646607809F066FF4640A07809F067
:1013F00083FF4640E07809F065FF46408DF80260C3
:10140000207809F05FFF0646607809F068FF4640E3
:10141000A07809F050FF4640E07809F06DFF4640A3
:101420008DF803609DF8000020709DF80100607049
:101430009DF80200A0709DF80300E0706D1C241D53
:10144000042DA7DBF8BD417B427A42734279427298
:101450004278427141708178827A8270817281799A
:10146000827B82718173C178C279C270C27AC27183
:10147000C27BC272C17370470146002004E00A5C5F
:10148000034B9A5C0A54401C1028F8DB704700009C
:101490002AB4000870472DE9F04106460C4617466D
:1014A0009846002500BF07E0102101FB0560424679
:1014B0003946FFF799FD6D1CE11704EB1171B5EB8F
:1014C000211FF1DB304602F058FEBDE8F0812DE926
:1014D000F04106460F4690460025304604F010FCC9
:1014E000044600BF07E0102101FB05604246394673
:1014F000FFF7A4FD6D1CE11704EB1171B5EB211F83
:10150000F1DB2046BDE8F08130B5044604254FF4F8
:10151000302000F06FF80546042D17D10C48006903
:1015200040F002000A49086108464461006940F041
:10153000400008614FF4302000F05CF80546044894
:10154000006941F6FD71084001490861284630BD37
:101550000020024004200B49C96801F0010109B1D3
:1015600001200EE00749C96801F0040109B1022019
:1015700007E00449C96801F0100109B1032000E047
:1015800004207047002002400348006940F08000BA
:1015900001490861704700000020024070B5044610
:1015A0000D460426F00200F025F80646042E11D15F
:1015B0000948006940F00100074908612580F002F0
:1015C00000F018F806460448006941F6FE7108402C
:1015D00001490861304670BD0020024002480349BD
:1015E0004860034848607047230167450020024077
:1015F000AB89EFCD00B502460423FFF7ABFF0346EE
:1016000003E0FFF7A7FF0346521E012B01D1002A7A
:10161000F7D102B90523184600BD000008B5012125
:10162000402000F06DFB10208DF803002020ADF865
:10163000000003208DF802006946044800F008F815
:101640002021024800F091F808BD00000018014078
:101650002DE9F04102460025002600200023002449
:10166000002791F803C00CF00F0591F803C00CF0AF
:10167000100CBCF1000F03D091F802C04CEA050534
:1016800091F800C0BCF1000F31D0146800202BE0AD
:101690004FF0010C0CFA00F3B1F800C00CEA03069D
:1016A0009E4220D183004FF00F0C0CFA03F7BC438D
:1016B00005FA03FC4CEA040491F803C0BCF1280FBE
:1016C00006D14FF0010C0CFA00FCC2F814C00AE07D
:1016D00091F803C0BCF1480F05D14FF0010C0CFA92
:1016E00000FCC2F810C0401C0828D1D31460B1F827
:1016F00000C0BCF1FF0F34DD546800202EE000F183
:10170000080C4FF0010808FA0CF3B1F800C00CEA1D
:1017100003069E4221D183004FF00F0C0CFA03F711
:10172000BC4305FA03FC4CEA040491F803C0BCF185
:10173000280F05D100F1080C08FA0CF8C2F8148043
:1017400091F803C0BCF1480F07D100F1080C4FF02D
:10175000010808FA0CF8C2F81080401C0828CED303
:101760005460BDE8F081416170470161704700003D
:10177000FEB51D464E4FD7E90064BF68CDE901476D
:101780000096ADF802508C5C04F00F04ADF80440F4
:10179000ADF806208C5C23090D2B09DA00248DF8A6
:1017A0000840BDF802401C44A4B2ADF8024033E04A
:1017B0000D2B0DD101268DF80860561C8C5DBDF8EF
:1017C000027004F10D063E44B6B2ADF8026023E0AB
:1017D0000E2B16D102268DF808600024561C8E5D53
:1017E00026434FF6FF7707EA0624961C8E5D3443A6
:1017F000BDF8027004F20D163E44B6B2ADF80260B8
:101800000AE000248DF80040009C0460019C4460C4
:10181000BDF808400481FEBDBDF804400D2C03DA7C
:1018200000248DF8094039E0BDF804400D2C0CD19E
:1018300001268DF809609DF808601644761C8C5DC1
:1018400004F10D06ADF8046028E0BDF804400E2C4C
:1018500019D102268DF8096000249DF8086016440D
:10186000761C8E5D26434FF6FF7707EA06249DF827
:1018700008601644B61C8E5D344304F20D16B6B2F1
:10188000ADF804600AE000248DF80040009C04607C
:10189000019C4460BDF808400481BCE7009C0460E2
:1018A000019C4460BDF80840048100BFB3E700001C
:1018B00018B300082DE9F04385B007460D461646DB
:1018C0002846FFF719FC814609F104044FF000088F
:1018D0001F4903C9CDE900012FE0285DFF280CD185
:1018E00001208DF80000601C80B2ADF80200301BB2
:1018F000401E80B2ADF8040021E04346224629464E
:1019000002A8FFF735FF9DF8080038B900208DF8D0
:101910000000ADF80400ADF8020010E0BDF80A8048
:10192000BDF80E009DF8101008449DF811100844F1
:10193000BDF80C100844401C84B2B442CDDB00BF9B
:1019400000983860BDF80400B88005B0BDE8F083A9
:1019500024B3000800BFFEE7F0B50446059D002053
:1019600005E01E18965D0F18E655461CB0B2A84259
:10197000F7DBF0BD0FB408B54FF400710848FEF76F
:10198000F0FB03A800900648009A029901F0BCF908
:1019900000200090024800F053F801B05DF814FBFD
:1019A000C40300200FB408B50C48007810B901B08A
:1019B0005DF814FB4FF400710948FEF7D2FB03A851
:1019C00000900748009A029901F09EF900200090CB
:1019D000034800F035F800BFE9E7000018000020D8
:1019E000C403002070B505460E46002404E0285DBF
:1019F00000F016F8601C84B2B442F8DB70BD000041
:101A000070B504460D460548007800B970BD2946FA
:101A10002046FFF7E7FF00BFF8E7000018000020AE
:101A200010B504462146054801F07CF800BF80212E
:101A3000024800F0C3FF0028F9D010BD0038014073
:101A400070B50446002504E0605DFFF7E9FF681CFF
:101A500085B2605D0028F7D170BD00BFFEE7F8B524
:101A60000446002545E0207809F0FDFB0646607835
:101A700009F005FC4640A0784640E07846408DF8E5
:101A80000060607809F0EFFB217880EA0106A07819
:101A900009F0F5FB4640E07846408DF80160A078FB
:101AA00009F0E1FB21786278514080EA0106E07894
:101AB00009F0E5FB46408DF80260207809F0DFFB75
:101AC00061784840A17880EA0106E07809F0CBFB14
:101AD00046408DF803609DF8000020709DF80100DD
:101AE00060709DF80200A0709DF80300E0706D1C0E
:101AF000241D042DB7DBF8BD7047000070B5002130
:101B000000230F22C47804B3154C246804F4E06465
:101B1000C4F5E064210AC1F10403CA40447804FA20
:101B200003F184781440214309010E4C0678A15535
:101B3000047804F01F050124AC4005786D11AD0058
:101B400005F1E025C5F8004109E0047804F01F051F
:101B50000124AC40044D0678761145F8264070BD4E
:101B60000CED00E000E400E080E100E00249014308
:101B7000024A1160704700000000FA050CED00E019
:101B80007047000000B589B02A48007830B90020BD
:101B9000294908600120274908700BE027480068A0
:101BA0004FF47A71484324490968884202D20120DF
:101BB0002349087022480078012839D100F05EFEE0
:101BC00088B900201B49087000F052F800F06CF84A
:101BD00024221C496846FEF7ABFA1A4810380FC891
:101BE00000F032FE24E000F049FE02280ED1164932
:101BF00016A0FFF7BFFE00F0A5FB002010490870FB
:101C000016480088401C1549088011E000F036FE97
:101C100003280DD10C4912A0FFF7ACFE00F092FB97
:101C20000020074908700D480088401C0B490880B7
:101C300009B000BDD0000020D4000020D800002052
:101C4000DD00002090150020C5070020B7A2CBCDF5
:101C5000B3C9B9A6A3BA25730D0A0000DE0000209F
:101C6000B7A2CBCDCAA7B0DCA3BA25730D0A00007A
:101C700000200C490880887048600877487788778A
:101C8000C87781F8200081F8210081F8220081F8CE
:101C9000230081F8240081F8250081F8260081F8CE
:101CA00027007047801500204FF47A7003490880A0
:101CB00001208870EA2048607047000080150020ED
:101CC00029B1064AD2690243044BDA6104E0034AAF
:101CD000D2698243014BDA61704700000010024074
:101CE00029B1064A12690243044B1A6104E0034A0F
:101CF00012698243014B1A617047000000100240D4
:101D000029B1064A92690243044B9A6104E0034AEE
:101D100092698243014B9A617047000000100240B3
:101D200029B1064AD2680243044BDA6004E0034A50
:101D3000D2688243014BDA60704700000010024015
:101D400030B500210022002400232D4D6D6805F0E0
:101D50000C0121B1042905D0082923D105E0294D22
:101D6000056022E0274D05601FE0254D6D6805F4F4
:101D70007012234D6D6805F48034022505EB924204
:101D80001CB9214D554305600BE01D4D6D6805F4F0
:101D900000351DB11C4D5543056002E0194D5543FA
:101DA000056002E0174D056000BF00BF144D6D686F
:101DB00005F0F0010909154D6B5C0568DD404560D3
:101DC0000F4D6D6805F4E061090A104D6B5C4568C4
:101DD000DD4085600A4D6D6805F46051C90A0B4D00
:101DE0006B5C4568DD40C560054D6D6805F440419C
:101DF000890B074D6B5CC568B5FBF3F5056130BD1C
:101E00000010024000127A0000093D00000000208E
:101E10001000002030B503460C461546002207E0AE
:101E2000184600F008F824F812009B1C501C82B2DF
:101E3000AA42F5DB30BD0146088870472DE9F05F06
:101E400080468A461746B8F1006F02D33348804572
:101E500001D3BDE8F09FFFF7C1FBA8F1006B4FEA8B
:101E6000DB25CBF34909C9F58064A74200DC3C4679
:101E70004DE04FF0006101EBC5204A142849FFF7FF
:101E8000C9FF00260BE009EB0600254931F81000D8
:101E90004FF6FF71884200D003E0701C86B2A64264
:101EA000F1DB00BFA6421BDA4FF0006101EBC52059
:101EB000FFF72AFB002608E03AF8160006EB0901B6
:101EC000174A22F81100701C86B2A642F4DB4FF0CC
:101ED000006101EBC5204A14114909F0B1F904E091
:101EE00022465146404609F0ABF9A74200D10FE027
:101EF0006D1C4FF000090AEB440AA044381B87B25E
:101F0000B7F5806F02DD4FF4806400E03C46B0E737
:101F100000BFFFF739FB00BF9BE700000000080887
:101F20002417002070470000F8B505460C46002134
:101F300002E06F5C6754491C97008F42F9DC114640
:101F400051E0002008E04F1E4FF0040C0CFB070787
:101F5000E75D0DF80070401C0428F4DB91FBF2F7FC
:101F600002FB17174FBB9DF800609DF801708DF8BC
:101F700000709DF802708DF801709DF803708DF867
:101F800002708DF80360002008E01DF80070DFF893
:101F900060C01CF807700DF80070401C0428F4DBCA
:101FA00091FBF2F77F1EDFF84CC01CF807709DF81C
:101FB00000C087EA0C078DF80070002010E08F1A2F
:101FC0004FF0040C0CFB0707E75D1DF800C087EA23
:101FD0000C074FF0040C0CFB010C04F80C70401CB7
:101FE0000428ECDB491C5F1CBF008F42A9DCF8BD54
:101FF0002AB300082AB5000810B500F001F810BD9A
:102000000CB50020019000903348006840F4803007
:102010003149086000BF3048006800F4003000908B
:102020000198401C0190009818B90198B0F5A06F74
:10203000F1D12948006800F4003010B1012000906F
:1020400001E0002000900098012843D12348006857
:1020500040F01000214908600846006820F00300A5
:1020600008600846006840F0020008601A484068AE
:10207000194948600846406848600846406840F48E
:10208000806048600846406820F47C10486008463C
:10209000406840F4E81048600846006840F08070EE
:1020A000086000BF0C48006800F000700028F9D0FC
:1020B0000948406820F00300074948600846406826
:1020C00040F00200486000BF0348406800F00C0088
:1020D0000828F9D10CBD0000001002400020024089
:1020E000417842794270427A4271427B4272417336
:1020F0008178827A827081728179827B8271817328
:10210000C17BC27AC273C279C272C278C271C17015
:10211000704700000146002004E00A5C034B9A5C13
:102120000A54401C1028F8DB704700002AB300084E
:102130007047000010B51348006840F001001149D5
:10214000086008464068104908400E494860084643
:1021500000680E4908400B4908600846006820F4F2
:10216000802008600846406820F4FE0048604FF474
:102170001F008860FFF740FF4FF0006004490860CF
:1021800010BD0000001002400000FFF8FFFFF6FE47
:1021900008ED00E010B50121880700F023F80128C0
:1021A0000AD107F093FE05480068401C0349086007
:1021B0000121880700F007F810BD0000140000207E
:1021C000CA4302827047CA430282704721B1028823
:1021D00042F00102028004E002884FF6FE731A40CA
:1021E0000280704730B50246002000230024158A83
:1021F00005EA0103958905EA010413B10CB1012038
:1022000000E0002030BD1AB183890B43838102E0D6
:1022100083898B438381704701894FF6F87211409F
:1022200001817047002202881D4B98420ED01D4B41
:1022300098420BD0B0F1804F08D01B4B984205D08C
:102240001A4B984202D01A4B984204D14FF68F7322
:102250001A404B881A43174B984207D0164B9842A6
:1022600004D04FF6FF431A40CB881A4302808B8874
:1022700083850B8803850A4B98420BD0094B984203
:1022800008D00E4B984205D00D4B984202D00D4B12
:10229000984201D10B7A03860123838270470000A4
:1022A000002C0140003401400004004000080040C0
:1022B000000C0040001000400014004000400140AD
:1022C00000440140004801401FB501210846FFF7C6
:1022D000F7FC4FF08040FFF79FFF0020ADF80A00A9
:1022E000ADF806000920ADF8080041F61F40ADF832
:1022F000040000208DF80C0001A94FF08040FFF78A
:1023000091FF01218807FFF75BFF0122114690072B
:10231000FFF779FF4FF4A060FFF728FC1C208DF831
:10232000000001208DF8030002208DF8010001203B
:102330008DF802006846FFF7E1FB01218807FFF7EF
:1023400045FF1FBD10B5002003F074FD00200149BA
:10235000087010BDC407002010B58CB0CE480078BE
:102360001A2876D2DFE800F00D0E17EFEE75A7758C
:10237000CDDDFD75ECEBEAE9E8751F75354B90E7AF
:10238000E6E585E10020C5490870C54908700220CE
:1023900003F050FD7CE1C349C86880470321122047
:1023A00003F054FD74E1BF48416A01208847BE49EB
:1023B000087008460078012803D1142003F03AFD84
:1023C00006E0B9480078022802D1B8A003F012FD57
:1023D0005EE1B448C16A02208847B34908700846E4
:1023E0000078012803D1152003F024FD06E0AE4853
:1023F0000078022802D1B2A003F0FCFC48E1A94811
:10240000B34BB44AB449446BB448A047A6490870DA
:102410000846007801282FD1AF480078012819D14B
:10242000AC480088AE494885A9480068C862AD48F4
:10243000AD492422CDE90910A94910316846FDF7BC
:1024400077FEA7480FC801F043FA162003F0F2FC0C
:1024500019E01CE1914800780A2803DDA3A003F0ED
:10246000C9FC10E04FF4C87003F020FD8B480078E1
:10247000401C8A49087006E08B480078022802D187
:102480009FA003F0B7FC03E18648C16CA048007828
:1024900088478549087008460078012803D106203E
:1024A00003F0C8FC06E080480078022802D199A019
:1024B00003F0A0FCECE09B480121CDE90010794835
:1024C000446C99480388994A99A191480078A0479B
:1024D000754908700846007801280AD1914800889B
:1024E00018B9082003F0A6FC0AE092A003F082FCD1
:1024F00006E06D480078022802D192A003F07AFC31
:10250000C6E003F0CDFE9349087008460078012824
:1025100003D10A2003F08EFC02E0092003F08AFCBC
:10252000B6E05F48007800280EDD8BA003F062FC67
:1025300016E0ABE085E080E094E04DE032E01BE0A7
:1025400083E00EE076E09AE08749884803F0EEFCED
:102550000D2003F06FFC52480078401C5049087071
:1025600096E060480178804B804A5F4803F090FD18
:102570000D2003F05FFC8BE04A48416D0020884746
:102580004949087008460078012803D10E2003F05D
:1025900051FC06E044480078022802D174A003F000
:1025A00029FC75E03F48C36D6F4802886F49584861
:1025B000007898473C49087008460078012803D104
:1025C0000F2003F037FC06E037480078022802D1DC
:1025D0006CA003F00FFC5BE0324842F21073624AD9
:1025E0006249846E4A480078A0472F49087008461F
:1025F0000078012816D15C4801885C4808F0CAF8C8
:1026000004461CB9082003F015FC0AE0012C03D194
:102610000A2003F00FFC04E0022C02D15DA003F0BD
:1026200025FC06E020480078022802D15CA003F0D7
:10263000E1FB2DE008F0E2FD2AE00C2003F0FAFBBC
:1026400026E00C2003F0F6FB22E01648C1690120C9
:102650008847154908700846007810B1102003F02B
:10266000E9FB15E00F48416A002088470E490870D1
:102670000846007810B1032003F0DCFB08E00949AC
:1026800008698047192003F0D5FB01E000E000BF96
:1026900000BF0CB010BD000024000020B4000020DA
:1026A000B5000020E4000020A8000020C9E8D6C33F
:1026B000C8ABB9A6C4DCC4A3CABDCAA7B0DC0000BD
:1026C000C9E8D6C37073D3F2CAA7B0DC000000001B
:1026D000B0000020AC000020AA000020A9000020CB
:1026E0005C0B00209C000020900B0020B2E9D1AFD1
:1026F0007073D3F2B4CECAFDB9FDB6E0000000009D
:10270000B2E9D1AF7073D3F2CAA7B0DC0000000009
:1027100026000020B9D8B1D5C1ACBDD3CAA7B0DC62
:1027200000000000B600002082000020C908002040
:1027300055445000BFCDBBA7B6CBB4F2BFAAB4ED91
:10274000CEF30000B4F2BFAABFCDBBA7B6CBCAA7D9
:10275000B0DC0000B8000020C8CFD6A4B4CECAFDBB
:10276000B9FDB6E000000000880000204B09002001
:10277000B9D8B1D5B7A2CBCDBBD8CFD4CAA7B0DC1E
:1027800000000000B7A2CBCD73656E64CAA7B0DCB1
:1027900000000000B7A2CBCDB3C9B9A6000000006D
:1027A000B5C8B4FDBDE1B9FBCAA7B0DC00000000AC
:1027B00010B515491548FDF712FD13491E3114488F
:1027C000FDF70DFD104932391248FDF708FD3C2197
:1027D0001148FDF7C6FC0D490F48FDF7CDFC0FA1D0
:1027E0000D48FDF7C9FC3C211548FDF7BAFC074927
:1027F0001348FDF7C1FC13A11148FDF7BDFC0449C6
:102800000F48FDF7B9FC10BDE61600202700002098
:102810003B0000204F000020C90800202E636F619C
:10282000702E636E2D7368616E676861692E6C69C6
:102830006E6B2E616C6979756E63732E636F6D00BC
:102840008D080020260000000FB410B5084800785D
:1028500058B9342202A90748FDF76AFCFFF7A8FF20
:1028600001200549087003F0E5FA10BC5DF814FB7F
:10287000240000205C0B0020C407002007480078DB
:1028800010B906480078704705480078192802D129
:1028900002480078F7E70120F5E70000C4070020B0
:1028A0002400002010B540F225510D4800F086F8B4
:1028B000012814D10A4800F01FF9C4B20948B0F841
:1028C0000212B0F80202401C064AA2F80202501C92
:1028D000445440F22551024800F006F800BF10BDF4
:1028E00000440040C001002010B50022002340F643
:1028F0006A14A14200D100BF0A1201249440A3B27D
:10290000DC43048010BD21B1828942F400528281EF
:1029100004E082894DF6FF731A40828170470000FF
:1029200010B504462048844209D101218803FFF7ED
:10293000F7F900214FF48040FFF7F2F932E01B482D
:10294000844209D101214804FFF7CAF900214FF45C
:102950000030FFF7C5F925E01548844209D101216F
:102960008804FFF7BDF900214FF48020FFF7B8F984
:1029700018E01048844209D10121C804FFF7B0F9DA
:1029800000214FF40020FFF7ABF90BE00A48844226
:1029900008D101210805FFF7A3F900214FF48010A9
:1029A000FFF79EF910BD00000038014000440040D0
:1029B00000480040004C004000500040024600200B
:1029C000B1F5007F00D100BF13880B400BB101208F
:1029D00000E000207047F0B50346002400260025E3
:1029E000002040F66A17B94200D100BF1846C1F373
:1029F000421401F01F06012707FA06F5012C01D148
:102A00000C3004E0022C01D1103000E014301AB177
:102A100007682F43076002E00768AF430760F0BD17
:102A20002DE9F04786B005460E460024A24600BFB9
:102A3000A1460027B08900B100BF2F462C8A4CF672
:102A4000FF700440F08804432C82AC894EF6F310EA
:102A50000440B08831890843718908430443AC813C
:102A6000AC8A4FF6FF400440B0890443AC8201A811
:102A7000FFF766F91F48874202D1DDF810A001E098
:102A8000DDF80CA0A88900F4004040B10AEBCA00B0
:102A900000EB0A1031684900B0FBF1F807E00AEBDF
:102AA000CA0000EB0A1031688900B0FBF1F864201D
:102AB000B8FBF0F004012009642101FB1089A8890A
:102AC00000F4004040B1322000EBC900B0FBF1F04F
:102AD00000F00700044308E0322000EB09106421F5
:102AE000B0FBF1F000F00F0004432C8106B0BDE80C
:102AF000F08700000038014001468888C0F30800D4
:102B00007047000010B504462146054800F00AF859
:102B100000BF80210248FFF751FF0028F9D010BD07
:102B200000440040C1F308028280704770B505463A
:102B30000E46002404E0285DFFF7E4FF601C84B229
:102B4000B442F8DB70BD00BFFEE7000000B587B0FF
:102B500001218803FFF7D4F801210420FFF7D0F802
:102B600018208DF81B004FF40070ADF818000320FA
:102B70008DF81A0006A92148FEF76AFD48208DF855
:102B80001B004FF48060ADF8180003208DF81A0088
:102B900006A91A48FEF75CFD4FF4E13002900020D0
:102BA000ADF814000C20ADF812000020ADF81000B4
:102BB000ADF80E00ADF80C0002A91148FFF730FF88
:102BC000012240F225510E48FFF705FF4FF4A060A7
:102BD000FEF7CCFF25208DF8040001208DF80700BA
:102BE00003208DF805008DF8060001A8FEF786FF8A
:102BF00001210348FFF787FE07B000BD0008014030
:102C00000038014000B587B001214804FFF758F8AB
:102C100001210420FFF774F82548FFF781FE1820F2
:102C20008DF81B000420ADF8180003208DF81A0061
:102C300006A92048FEF70CFD04208DF81B00082093
:102C4000ADF8180006A91B48FEF702FD4FF4E1306D
:102C500002900020ADF814000C20ADF81200002006
:102C6000ADF81000ADF80E00ADF80C0002A9104848
:102C7000FFF7D6FE012240F225510D48FFF7ABFECB
:102C80004FF4A060FEF772FF26208DF804000120AB
:102C90008DF807008DF805008DF8060001A8FEF7F5
:102CA0002DFF01210248FFF72EFE07B000BD0000F6
:102CB00000440040000801400FB41CB50A46521EF3
:102CC000CDE9000207A9054B6A46069800F052F9C3
:102CD000009A002111701CBC5DF814FBA33600089B
:102CE0000FB4084B10B504A902AA039800F042F9EA
:102CF000044602A9002000F0DFFC204610BC5DF86D
:102D000014FB0000B936000837B514460846064BD8
:102D10006A46214600F02EF904466946002000F07C
:102D2000CBFC20463EBD0000B93600080048704785
:102D3000BC01002030B528B1144C031F00202168CD
:102D40000A4605E0084630BD9A4203D8104652684C
:102D5000002AF9D1002800D041680BD00468A3EB09
:102D60000005A54204D11B681C440346046002E030
:102D7000436000E023603AB11C68D51AA54203D134
:102D800015682C441C6052685A6030BDB4010020A4
:102D90002DE9F04782460F4C10480D4E0E4F001B98
:102DA0004FF0000820F007054FF0010900221146FE
:102DB000504603F093F8002802D1306810B100208B
:102DC000BDE8F0873C60C4E90058C6F80090EDE724
:102DD000B80100207C200020B401002078280020C9
:102DE00002E008C8121F08C1002AFAD170477047D4
:102DF000002001E001C1121F002AFBD17047000032
:102E00002DE9FF5FDDE90220010DDDF838B0024356
:102E100018D044F61050A1F2FF3141430D140F9821
:102E2000012820D0A5EB0B00401C5FEA000A4FF000
:102E30000004474EDFF81C91A046504616D5CAF153
:102E4000000728E00F98012443A2012808D00021A0
:102E500000980F9BC0E90021C0E90243BDE8FF9F35
:102E60006FEA0B01F4E7CBF10000DEE7074612E062
:102E7000F80707D02246334640464946FDF773FC23
:102E8000804689462246334610461946FDF76BFCBC
:102E900004460E467F10002FEAD1DDE90201BAF1A7
:102EA000000F42464B4602DAFDF75DFC01E0FDF7FC
:102EB000F2FE04460E460022284BFDF7FDFC03D827
:102EC0004FF0FF30014607E00022254B20463146F7
:102ED000FDF7A2FBFDF75AFF102409E0002C0ADBE6
:102EE0000A220023FDF716FD019B30321A55641E9D
:102EF00050EA0102F2D1641C019AC4F11103144496
:102F00000F9A012A03D0012208430DD10AE0084399
:102F100004D000204FF0110B0F9080E7A3EB0B05BE
:102F20006D1E0DE05B4504DD4FF0000205F101056B
:102F300004E003DA4FF00002A5F10105002AECD00D
:102F400000980F99C0E90231C0E9004586E700000A
:102F5000000024400000F03F300000000000F0437B
:102F60000000E03F30380A2801D2012070470020DD
:102F7000704700002DE9FF4F95B09B4689460646F5
:102F800000250FE2252877D100242746F84A0121A1
:102F9000059400E0044316F8013F203B01FA03F0DA
:102FA0001042F7D130782A2811D06FF02F033078F3
:102FB000A0F13002092A16D8059A44F0020402EB67
:102FC000820203EB42021044761C0590EFE759F8A9
:102FD000042B0592002A03DA504244F40054059071
:102FE00044F00204761C30782E2816D116F8010F12
:102FF00044F004042A280DD06FF02F023078A0F19D
:103000003003092B09D807EB870302EB4303C718EA
:10301000761CF3E759F8047B761C30786C280FD0C7
:1030200006DC4C2817D068280DD06A2814D104E09B
:10303000742810D07A280FD10DE044F400140AE06F
:1030400044F4801401E044F440147278824202D1C6
:1030500004F58014761C761C307866280BD013DCBF
:10306000582877D009DC002875D04528F6D04628A6
:10307000F4D047281AD19DE118E0632835D06428A0
:1030800079D0652812D195E1702873D008DC6728C3
:10309000F1D069286FD06E280DD06F2806D1B5E029
:1030A00073282CD0752875D0782874D05A46179973
:1030B00090476D1C75E1C4F30250022809D0032823
:1030C0000DD0D9F8001004280DD00D6009F10409C5
:1030D00067E1D9F80010EA17C1E90052F6E7D9F81C
:1030E00000100D80F2E70D70F0E719F8041B8DF861
:1030F000001000208DF80100EA46012003E059F895
:1031000004AB4FF0FF3061074FF0000102D40DE037
:1031100008F101018846B9420FDA8045F8DB1AF858
:1031200008100029F4D108E008F101018846814225
:10313000FADB1AF808100029F6D105985B46A0EBD7
:10314000080721463846179A00F094FA284400EB05
:10315000080507E04DE029E10DE01AF8010B5A4699
:1031600017999047B8F10108F7D25B4621463846D7
:10317000179A13E142E00A220092C4F302524FF080
:10318000000A022A08D059F804CB032A4FEAEC714E
:103190000AD00DE029E02AE009F1070121F0070239
:1031A000F2E802C1914609E00FFA8CFC4FEAEC719B
:1031B000042A03D14FFA8CFC4FEAEC71002907DA9C
:1031C0000A460021DCF1000C61EB02012D2202E035
:1031D000220504D52B228DF80420012203E0E2070A
:1031E00001D02022F7E7904659E00A2102E01022A0
:1031F0000DE010214FF0000A00910BE010224FF07B
:10320000000A44F004040827009203E008224FF06B
:10321000000A0092C4F30252022A05D059F804CBE6
:103220000021032A08D009E009F1070121F0070273
:10323000F2E802C1914605E01FFA8CFC042A01D194
:103240000CF0FF0C4FF00008220728D5702806D09C
:10325000009B83F0100353EA0A0305D00EE04022DE
:103260008DF80420012208E05CEA010206D0302239
:103270008DF804208DF8050002229046009B83F013
:10328000080353EA0A030AD15CEA010201D162078A
:1032900005D530228DF804204FF001087F1E5828F4
:1032A00004D034A003900EA802900DE036A0F9E7F8
:1032B00053466046009AFDF72DFB84460398825CD6
:1032C0000298401E029002705CEA0100F0D1029860
:1032D00006A9081A00F1200A600702D524F48034F8
:1032E00000E00127574502DDA7EB0A0000E00020BF
:1032F00000EB0A01009005984144401A0590E00354
:1033000006D45B462146179A059800F0B3F90544A8
:10331000002706E001A85A46C05D179990476D1C2A
:103320007F1C4745F6DBE0030CD55B462146179A28
:10333000059800F09FF9054404E030205A4617999B
:1033400090476D1C0099481E00900029F5DC08E0AC
:10335000029802995A460078491C029117999047A1
:103360006D1CBAF10001AAF1010AF1DC65E100006F
:10337000092801003031323334353637383961624B
:10338000636465660000000030313233343536370F
:1033900038394142434445460000000000F058F9E6
:1033A0000544761C307800287FF4ECAD19B028462F
:1033B000BDE8F08F620700D4062709F1070222F06A
:1033C000070CFCE80223E14603F000485FEA080C22
:1033D00002D00FF2702C0DE05FEA045C02D50FF210
:1033E000682C07E05FEAC47C02D00FF2602C01E099
:1033F000AFF2700C4FF0FF3823F00043CDF850C00F
:1034000065280CD006DC452809D046281DD0472861
:103410003DD13DE0662818D067287ED138E00021F4
:10342000112F01DB112000E0781CCDE9000106A975
:103430000EA8FFF7E5FCDDE90F010E9A03910021CC
:10344000009207F1010A04914DE04FF0004000970F
:10345000CDE9011006A90EA8FFF7D2FCDDE90F02A5
:1034600003920E9B11990022DDF80CA000930492A8
:1034700011B9791C00EB010AB7EB0A0004D4C0F1C2
:10348000FF3007F1010A0490AAEB0700019044E025
:10349000012F00DA01270021112F01DD112000E0AA
:1034A0003846CDE9000106A90EA8FFF7A9FCDDE921
:1034B0000F010E9A0391002104910092BA46210750
:1034C0000CD40399514500DA8A46BAF1010F05DDA3
:1034D000009AAAF10101515C302908D0B84202DA01
:1034E00010F1040F06DA0121CDE9011015E0AAF16F
:1034F0000101E9E7002805DC049901440491AAEBE5
:10350000000102E0411C514500DD8A460499401A41
:10351000401C01904FF000400290200704D4019815
:10352000504501DBCDF8048000208DF84F00029853
:103530000DF14F07B0F1004F25D02B200E900298CF
:103540004FF0020800280CDA404202902D200E9025
:1035500007E00A210298FDF7C7F93031029007F819
:10356000011DB8F10001A8F10108F2DC0298002861
:10357000EFD1791E0E980870307800F0200040F0EE
:10358000450007F8020D12A8C01B00F107081498A7
:10359000007800B1012000EB0A01019801EBE07115
:1035A00005984144401A401E0590E00306D45B464E
:1035B0002146179A059800F05DF8054414980078A4
:1035C00018B15A46179990476D1CE00324D55B4605
:1035D0002146179A059800F04DF805441CE0049820
:1035E000002807DBDDE90301884203DD0098405C29
:1035F000179901E0179930205A469047049805F131
:103600000105401C04900198401E019004D12E2019
:103610005A46179990476D1CBAF10001AAF1010AA8
:10362000DDDC05E017F8010B5A46179990476D1C31
:10363000B8F10001A8F10108F4DC5B462146179AB5
:103640000598ABE62D0000002B00000020000000D4
:103650002DE9F041044600251E461746880404D48F
:1036600005E039462020B0476D1C641EF9D5284678
:10367000BDE8F0812DE9F041044600251E46904644
:10368000C80301D5302700E02027880404D505E0D1
:1036900041463846B0476D1C641EF9D52846BDE842
:1036A000F0814A68002A06D00A68531C0B6010702B
:1036B0004868401E486070470A68531C0B601070D1
:1036C000704700002DE9F043ADF5017D00274FF470
:1036D000007101A8FCF745FD002000908046002401
:1036E00000250026414842F210736A4601A9D0F82D
:1036F0006CC03F480078E0470746022F04D13846A7
:103700000DF5017DBDE8F0834FF499613948FCF770
:1037100028FDBDF8002001A93648FCF709FD0A2361
:10372000042235493548FEF7FFFBBDF8000031495A
:10373000C1F8C80408460A232F4AD0F8C814FDF778
:10374000AAFE2C4800F01CFC8046B8F1000F14D1F2
:1037500000F0ECFB8146494629A0FEF723F94046DC
:1037600000F0B8FB204600F0B5FB284600F0B2FBA5
:10377000304600F0AFFB0220C2E727A1404600F030
:10378000DDFB064628A1404600F0D8FB044629A1EF
:10379000404600F0D3FB05462B692269316928A019
:1037A000FEF700F9316932223548FCF7C1FC216986
:1037B0001E2233483230FCF7BBFC29691E223048F8
:1037C0005030FCF7B5FC012211462E48FCF7C2FC34
:1037D000404600F07FFB204600F07CFB284600F0CE
:1037E00079FB304600F076FB012089E7E4000020F9
:1037F000A0010020B4100020881F00208F010020AD
:103800006A736F6E207061727365206572726F7279
:103810002C25730D0A0000006465766963655365A5
:10382000637265740000000070726F647563744B9E
:10383000657900006465766963654E616D650000B9
:10384000BBF1C8A1CAFDBEDDB3C9B9A6646576697E
:1038500063655365637265743A25732C6A736F6E82
:103860005F70726F647563744B65793A25732C646D
:1038700065766963654E616D653A25730D0A0000D2
:10388000B416002080010020014609B1086808B97B
:103890000020704719B1D1E90120904201D30846B8
:1038A000F7E702E08868401C886041B1D1E9012057
:1038B000904204D28A680868805C2028F2DDD1E951
:1038C0000120904202D18868401E88600846E0E7E7
:1038D0000FB438B5DDE9114500200090FE4908809D
:1038E0005421BDF80020501C80B20090A1545221F8
:1038F000BDF80020501C80B20090A1540121BDF8F9
:103900000020501C80B20090A154BDF80020501C33
:1039100080B20090A1546B462246652007F04EF914
:103920009DF81210BDF80020501C80B20090A154E8
:103930006B4622460421672007F040F90598010EE6
:10394000BDF80020501C80B20090A1540598C0F32F
:103950000741BDF80020501C80B20090A15405988A
:10396000C0F30721BDF80020501C80B20090A15484
:103970000598C1B2BDF80020501C80B20090A1543F
:103980006B4622460421682007F018F90698010EBC
:10399000BDF80020501C80B20090A1540698C0F3DE
:1039A0000741BDF80020501C80B20090A154069839
:1039B000C0F30721BDF80020501C80B20090A15434
:1039C0000698C1B2BDF80020501C80B20090A154EE
:1039D0006B4622460421692007F0F0F80798010E93
:1039E000BDF80020501C80B20090A1540798C0F38D
:1039F0000741BDF80020501C80B20090A1540798E8
:103A0000C0F30721BDF80020501C80B20090A154E3
:103A10000798C1B2BDF80020501C80B20090A1549C
:103A20006B46224602216A2007F0C8F8BDF8200044
:103A3000010ABDF80020501C80B20090A154BDF8CE
:103A40002000C1B2BDF80020501C80B20090A154EB
:103A50006B46224601216B2007F0B0F89DF822103A
:103A6000BDF80020501C80B20090A1546B46224645
:103A700001216C2007F0A2F89DF82310BDF800206A
:103A8000501C80B20090A1546B46224601216D204B
:103A900007F094F89DF82410BDF80020501C80B267
:103AA0000090A1546B46224601216E2007F086F853
:103AB0009DF82510BDF80020501C80B20090A15444
:103AC0006B46224602216F2007F078F8BDF82600E9
:103AD000010ABDF80020501C80B20090A154BDF82E
:103AE0002600C1B2BDF80020501C80B20090A15445
:103AF0006B4622460221702007F060F8BDF82800CE
:103B0000010ABDF80020501C80B20090A154BDF8FD
:103B10002800C1B2BDF80020501C80B20090A15412
:103B20006B4622460121712007F048F89DF82A10C3
:103B3000BDF80020501C80B20090A1546B46224674
:103B40000121722007F03AF89DF82B10BDF80020F3
:103B5000501C80B20090A1549DF82C0001280CD17B
:103B60006B4622460121732007F028F80121BDF899
:103B70000020501C80B20090A1549DF82D00012817
:103B80000CD16B4622460121732007F017F8022161
:103B9000BDF80020501C80B20090A1549DF82E006A
:103BA00001280CD16B4622460121732007F006F84C
:103BB0000321BDF80020501C80B20090A1549DF854
:103BC0002F0001280CD16B4622460121732006F0FC
:103BD000F5FF0421BDF80020501C80B20090A154D4
:103BE0009DF8300001280CD16B462246012173203C
:103BF00006F0E4FF0521BDF80020501C80B20090C3
:103C0000A1549DF8310001280CD16B4622460121B8
:103C1000732006F0D3FF0621BDF80020501C80B2AF
:103C20000090A1549DF8320001280CD16B46224629
:103C30000121732006F0C2FF0721BDF80020501CAF
:103C400080B20090A1549DF8330001280CD16B463E
:103C500022460121732006F0B1FF0821BDF80020A3
:103C6000501C80B20090A1549DF8340001280CD162
:103C70006B4622460121732006F0A0FF0921BDF802
:103C80000020501C80B20090A1549DF835000128FE
:103C90000CD16B4622460121742006F08FFF0121D2
:103CA000BDF80020501C80B20090A1549DF8360051
:103CB00001280CD16B4622460121742006F07EFFBC
:103CC0000221BDF80020501C80B20090A1549DF844
:103CD000370001280FD101E0E00000206B462246AA
:103CE0000121742006F06AFF0321BDF80020501C5A
:103CF00080B20090A1546B4622460121752006F047
:103D00005DFF9DF8380030B90021BDF80020501C3F
:103D100080B20090A1549DF83800012806D10121FD
:103D2000BDF80020501C80B20090A1549DF83800CE
:103D3000022806D10221BDF80020501C80B200905C
:103D4000A1549DF83800032806D10321BDF80020B6
:103D5000501C80B20090A1549DF83800042806D170
:103D60000421BDF80020501C80B20090A1546B4685
:103D700022460121762006F021FF9DF83910BDF87A
:103D80000020501C80B20090A1546B4622460221B4
:103D9000772006F013FFBDF83A00010ABDF80020B5
:103DA000501C80B20090A154BDF83A00C1B2BDF8D9
:103DB0000020501C80B20090A1546B462246042182
:103DC000782006F0FBFE0F98010EBDF80020501C75
:103DD00080B20090A1540F98C0F30741BDF80020B5
:103DE000501C80B20090A1540F98C0F30721BDF879
:103DF0000020501C80B20090A1540F98C1B2BDF8B1
:103E00000020501C80B20090A1546B462246012134
:103E1000792006F0D3FE9DF84010BDF80020501C1C
:103E200080B20090A1546B46224601217A2006F010
:103E3000C5FE9DF84110BDF80020501C80B20090D6
:103E4000A1546B46224601217B2006F0B7FE9DF867
:103E50004210BDF80020501C80B20090A154BDF863
:103E600000002880BDF8001002A0FDF783FD38BCDB
:103E70005DF814FBB7A2CBCDB3C9B9A6A3BA25731D
:103E80000D0A0000F0B50446154600201EE0265C31
:103E90003211265C06F00F033032392A03DDD61DBD
:103EA00001F8106001E001F8102003F13006F3B2D0
:103EB000392B05DDDE1D012707EB4007CE5503E05A
:103EC000012606EB40068B55461C30B2A842DEDBCD
:103ED000F0BD000070B50446002522E02568A089E9
:103EE00000F4807020B9A06810B1A068FFF7F2FF5D
:103EF000A08900F4807028B9206918B10A4A2069A5
:103F000051688847A08900F4007028B9206A18B168
:103F1000054A206A51688847034841682046884717
:103F20002C46002CDAD170BDC40000200248006885
:103F30000149496808447047BC00002070B5044638
:103F40000D4600222946204601F012FF70BD70B5D3
:103F500004460D4629462046FFF7F0FF08B1012030
:103F600070BD0020FCE770B5044628202168884712
:103F700005461DB128212846FCF7F3F8284670BDF8
:103F800010B5044600221146204600F06BF810BD23
:103F90002DE9F0478AB004460E46154698461C2186
:103FA00003A8FCF7DEF8002700202C4908604860D1
:103FB00004B106B932E00394049600200590284A23
:103FC00007CA07AB07C32648FFF7CDFF074607B967
:103FD00024E003A806F05CFE8246FFF755FC81460C
:103FE0004946384606F0EAFA00B917E0B8F1000F82
:103FF0000BD003A8FFF748FCDDE90410884203D288
:1040000005990398405C00B108E01DB1059903983B
:104010000844286038460AB0BDE8F08717B1384632
:10402000FFF758FFC4B1019400200290DDE90410AD
:10403000884202D20598029004E0049810B10498D6
:10404000401E02901DB1DDE90101084428600348CB
:10405000DDE9011206C000BF0020DCE7BC00002043
:10406000C40000202DE9F04104460D46164614B95F
:104070000020BDE8F0812046FCF79CF8471C334641
:104080002A4639462046FFF783FFF2E770B504461B
:104090000D4604B10DB9012070BDAC4201D1002024
:1040A000FAE705E0207808B90020F5E7641C6D1CEC
:1040B0002078FCF737F806462878FCF733F8864274
:1040C000F0D02078FCF72EF806462878FCF72AF87E
:1040D000301AE1E70C2803D808700023138015E09C
:1040E0000D2808D3B0F5867F05D80D230B70A0F1FD
:1040F0000D0313800AE0B0F5867F07D9044B984280
:1041000004D80E230B70A0F1FF031380704700004A
:10411000F5FF09000C2803D808700023138015E070
:104120000D2808D3B0F5867F05D80D230B70A0F1BC
:104130000D0313800AE0B0F5867F07D9044B98423F
:1041400004D80E230B70A0F1FF031380704700000A
:10415000F5FF090070B5044600252046FCF72AF853
:104160000646751E02E0002060556D1E605D002849
:1041700002DD605D1028F6DB70BD70B504460025D9
:104180002046FCF717F80646751E02E00020605531
:104190006D1E605D002802DD605D1028F6DB70BDDD
:1041A00000B5034603E04FF47A7000F005F81800FC
:1041B000A3F10103F7D100BD00EBC001C9004FF02E
:1041C000E0225161002191610521116100BF4FF092
:1041D000E021096901F480310029F8D004214FF071
:1041E000E0221161704700002DE9F04705460026E6
:1041F0001D244FF4FA77204606F0E4FF10B90220A0
:10420000BDE8F08701F0A6FD50B92A462AA12F4843
:10421000FEF766FDE1B22D4806F090FC064648E048
:1042200001F098FD012804D029A0FDF7BBFB022670
:104230003FE001F095FDB84206D92CA0FDF7B2FB96
:1042400005F062FE064634E0FCF7B6FE80462CA17F
:10425000FBF79EFF98B1FCF7B3FE804641462AA0CB
:10426000FDF7A0FBFCF7ACFE8046FCF7A5FE8146FF
:104270004146FDF7C5FB06F0C9FD064619E0FCF70F
:104280009BFE804624A1FBF783FF90B1FCF798FECC
:10429000804641461CA0FDF785FBFCF791FE804659
:1042A000FCF78AFE81464146FDF7AAFB01F0DCFCE3
:1042B00006463046A4E7000041542B5149434C4F79
:1042C00053453D25640D0D0A00000000B415002083
:1042D000B7B5BBD8BDE1B9FBB9FDC6DAA3ACC7EB36
:1042E000D6D8D6C3D7B4CCAC0D0A00004154D6B84A
:1042F000C1EEB7B5BBD8B3ACCAB10D0A000000001F
:104300004F4B0D0A000000004154B7B5BBD83A200E
:1043100025640D0A000000004552524F520D0A005C
:1043200070B50546002408E02846FFF75DFF044607
:104330001CB104498868804700E0F5E700BF2046CB
:1043400070BD0000E400002010B520210148FDF7F9
:104350000CFA10BD0018014010B520210148FDF7EE
:1043600002FA10BD001801402DE9F04F89B0054652
:104370000E4617469846DDE912A90020089013243E
:1043800040F6B8300790204606F01CFF18B902200E
:1043900009B0BDE8F08F01F0DDFC80B900203346A4
:1043A0002A464EA1CDE9020ACDE900785548FEF72C
:1043B00097FCE1B2534806F0C1FB08908CE001F095
:1043C000C9FC012806D050A0FDF7ECFA01F04CFC26
:1043D000089081E001F0C4FC0799884206D951A0F9
:1043E000FDF7E0FA05F090FD089075E0FCF7E4FDBC
:1043F000834651A1FBF7CCFE002853D0FCF7E0FD2B
:10440000014603904FA0FDF7CDFAFCF7D9FD0390CC
:10441000FCF7D2FD02900399FDF7F2FA0020069016
:104420000FF2FC0BFCF7C8FD06AA59460390FBF7F8
:10443000EFFE06AA59460020FBF7EAFE059006AA01
:1044400059460020FBF7E4FE049042A10598FBF7D3
:10445000B8FE18BB002003903FA0029003AA029967
:104460000498FBF7D5FE03AA00200299FBF7D0FEC3
:104470000090FCF7C4F8C0B2019003AA0020029992
:10448000FBF7C6FE0090FCF7BAF8A9F80000B9F8EF
:10449000002033A00199FDF785FA00BF06F0B6FCB5
:1044A000089019E0FCF788FD834632A1FBF770FE07
:1044B00090B1FCF785FD8346594622A0FDF772FABC
:1044C000FCF77EFD8346FCF777FD59460690FDF725
:1044D00097FA01F0C9FB0890089859E741542B510D
:1044E000494F50454E3D312C25642C222573222CFA
:1044F000222573222C25642C25642C25640D0D0A9D
:1045000000000000B4150020B7B5BBD8BDE1B9FB71
:10451000B9FDC6DAA3ACC7EBD6D8D6C3D7B4CCACFA
:104520000D0A00004154D6B8C1EEB7B5BBD8B3AC44
:10453000CAB10D0A000000002B51494F50454E3AB8
:10454000200000004154B7B5BBD83A2025640D0ABD
:10455000000000004F4B00003A202C220000000019
:10456000726573756C743A2025642C2025640D0ADD
:10457000000000004552524F520D0A002DE9FC4741
:1045800005460E4617469846DDE90A9A00240DE0D6
:1045900043463A4631462846CDE9009AFFF7E4FE05
:1045A00004461CB104498868804700E0F0E700BF7A
:1045B0002046BDE8FC870000E40000202DE9F0471C
:1045C00005460026452440F6B837204606F0FAFD99
:1045D00010B90220BDE8F08701F0BCFB50B92A46B3
:1045E0001CA12048FEF77CFBE1B21E4806F0A6FAAB
:1045F00006462DE001F0AEFB012804D01AA0FDF71D
:10460000D1F9022624E001F0ABFBB84206D91DA087
:10461000FDF7C8F905F078FC064619E0FCF7CCFC7C
:1046200080461DA1FBF7B4FD90B1FCF7C9FC8046A4
:1046300041461DA0FDF7B6F9FCF7C2FC8046FCF729
:10464000BBFC81464146FDF7DBF906F0DFFB064681
:104650003046BFE741542B51504F57443D25640D20
:104660000D0A0000B4150020B7B5BBD8BDE1B9FBF9
:10467000B9FDC6DAA3ACC7EBD6D8D6C3D7B4CCAC99
:104680000D0A00004154D6B8C1EEB7B5BBD8B3ACE3
:10469000CAB10D0A00000000504F57455245442052
:1046A000444F574E0D0A00004154B7B5BBD83A20CD
:1046B00025640D0A0000000070B50546002408E0DE
:1046C0002846FFF77BFF04461CB1044988688047F1
:1046D00000E0F5E700BF204670BD0000E4000020C8
:1046E0002DE9F04F87B004460D4616461F464FF0A1
:1046F00000094FF047084FF4FA700690404606F064
:1047000061FD18B9022007B0BDE8F08F01F022FB6F
:1047100050B972A17848FEF7E3FA08F0FF01764835
:1047200006F00CFA8146D7E001F014FB012806D010
:1047300072A0FDF737F901F097FA8146CCE001F05D
:104740000FFB0699884208D973A0FDF72BF90420C6
:1047500006F092FA4FF00209BEE0FCF72DFC82460B
:1047600072A1FBF715FD00287ED0FCF729FC01465D
:10477000029070A0FDF716F9FCF722FC0290FCF7FE
:104780001BFC01900299FDF73BF9002005900FF208
:10479000841AFCF711FC05AA51460290FBF738FD7C
:1047A00005AA51460020FBF733FD0490002003903A
:1047B0000FF2901B03AA59460498FBF729FD03AAA0
:1047C00059460020FBF724FD03AA59460020FBF7B9
:1047D0001FFD03AA59460020FBF71AFD03AA5946FC
:1047E0000020FBF715FD03AA59460020FBF710FD3A
:1047F00003AA59460020FBF70BFD03AA59460020E7
:10480000FBF706FD03AA59460020FBF701FD03AAAA
:1048100059460020FBF7FCFC03AA59460020FBF791
:10482000F7FC03AA59460020FBF7F2FC03AA5946FD
:104830000020FBF7EDFC03AA59460020FBF7E8FC3B
:1048400003AA59460020FBF7E3FC0290FBF7D7FED2
:10485000206003AA59460020FBF7DAFC0290FBF720
:10486000CEFE286003AA00E01CE059460020FBF7BA
:10487000CFFC0290FBF7C3FE306003AA594600202C
:10488000FBF7C6FC0290FBF7BAFE38603868009070
:1048900033682A682DA02168FDF784F806F0B6FA7F
:1048A000814619E0FCF788FB824633A1FBF770FCD8
:1048B00090B1FCF785FB824651461EA0FDF772F8C9
:1048C000FCF77EFB8246FCF777FB83465146FDF7FB
:1048D00097F801F0C9F98146484614E741542B5135
:1048E000454E473D2273657276696E6763656C6CF1
:1048F000220D0D0A00000000B4150020B7B5BBD88A
:10490000BDE1B9FBB9FDC6DAA3ACC7EBD6D8D6C3B7
:10491000D7B4CCAC0D0A00004154D6B8C1EEB7B53F
:10492000BBD8B3ACCAB10D0A000000004F4B0D0A52
:10493000000000004154B7B5BBD83A2025640D0AE9
:10494000000000003A202C22000000005253525078
:104950003A2025642C20525352513A2025642C20B1
:10496000525353493A2025642C2053494E523A2041
:1049700025640D0A000000004552524F520D0A00F6
:104980002DE9F04105460E461746984600240BE0F7
:1049900043463A4631462846FFF7A2FE04461CB17C
:1049A00004498868804700E0F2E700BF2046BDE880
:1049B000F0810000E40000202DE9F04F87B00446AC
:1049C0000D4616461F464FF000094FF009084FF4F8
:1049D000FA700690404606F0F5FB18B9022007B0C1
:1049E000BDE8F08F01F0B6F950B953A15648FEF773
:1049F00077F908F0FF01544806F0A0F8814698E0E6
:104A000001F0A8F9012806D050A0FCF7CBFF01F077
:104A10002BF981468DE001F0A3F90699884208D967
:104A200051A0FCF7BFFF042006F026F94FF0020961
:104A30007FE0FCF7C1FA824650A1FBF7A9FB0028F2
:104A40005DD0FCF7BDFA014602904EA0FCF7AAFF2C
:104A5000FCF7B6FA0290FCF7AFFA01900299FCF766
:104A6000CFFF002005900FF2FC0AFCF7A5FA05AA7B
:104A700051460290FBF7CCFB05AA51460020FBF7FC
:104A8000C7FB0490002003900FF2081B03AA5946AD
:104A90000498FBF7BDFB03AA59460020FBF7B8FBBF
:104AA0000290FBF7ACFD207003AA59460020FBF7EB
:104AB000AFFB0290FBF7A3FD287003AA5946002024
:104AC000FBF7A6FB102200210290FBF75FFD308070
:104AD00003AA59460020FBF79BFB102200210290FD
:104AE000FBF754FD38603868009033882A782178C5
:104AF0002AA0FCF757FF06F089F9814619E0FCF778
:104B00005BFA82462FA1FBF743FB90B1FCF758FA02
:104B1000824651461BA0FCF745FFFCF751FA82463E
:104B2000FCF74AFA83465146FCF76AFF01F09CF80D
:104B30008146484653E7000041542B4347524547BE
:104B40003F0D0D0A00000000B4150020B7B5BBD81A
:104B5000BDE1B9FBB9FDC6DAA3ACC7EBD6D8D6C365
:104B6000D7B4CCAC0D0A00004154D6B8C1EEB7B5ED
:104B7000BBD8B3ACCAB10D0A000000004F4B0D0A00
:104B8000000000004154B7B5BBD83A2025640D0A97
:104B9000000000003A202C22000000006D6F6465C8
:104BA0003A2025642C20737461743A2025642C20EB
:104BB0006C61633A2025642C2063693A2025640DDA
:104BC0000A0000004552524F520D0A002DE9F041F3
:104BD00005460E461746984600240BE043463A46E3
:104BE00031462846FFF7E8FE04461CB104498868B0
:104BF000804700E0F2E700BF2046BDE8F0810000FA
:104C0000E40000202DE9FE4F054600264B244FF41A
:104C1000FA77204606F0D6FA10B90220BDE8FE8FDA
:104C200001F098F848B940A14248FEF759F8E1B2BE
:104C3000404805F083FF064674E001F08BF8012838
:104C400006D03DA0FCF7AEFE01F00EF8064669E086
:104C500001F086F8B84207D93EA0FCF7A3FE042075
:104C600006F00AF802265DE0FCF7A6F980463EA1B0
:104C7000FBF78EFA00283BD0FCF7A2F9824651469A
:104C80003BA0FCF78FFEFCF79BF98246FCF794F9FA
:104C900083465146FCF7B4FE002002900FF2B008A4
:104CA000FCF78AF9824602AA4146FBF7B1FA02AA4A
:104CB00041460020FBF7ACFA0190002000900FF273
:104CC000C0096A4649460198FBF7A2FA6A46494676
:104CD0000020FBF79DFA824651462846FBF77FFAF3
:104CE000294629A0FCF75EFE06F090F8064619E07A
:104CF000FCF762F9804627A1FBF74AFA90B1FCF76E
:104D00005FF9804641461AA0FCF74CFEFCF758F9C3
:104D10008046FCF751F981464146FCF771FE00F0F0
:104D2000A3FF0646304679E741542B51434349449B
:104D30000D0D0A00B4150020B7B5BBD8BDE1B9FB15
:104D4000B9FDC6DAA3ACC7EBD6D8D6C3D7B4CCACC2
:104D50000D0A00004154D6B8C1EEB7B5BBD8B3AC0C
:104D6000CAB10D0A000000004F4B0D0A0000000000
:104D70004154B7B5BBD83A2025640D0A00000000A5
:104D80003A202C220000000049434349443A2025A0
:104D9000730D0A004552524F520D0A0070B5054678
:104DA000002408E02846FFF72DFF04461CB1044903
:104DB0008868804700E0F5E700BF204670BD00002E
:104DC000E40000202DE9FF5F0546002601244FF492
:104DD000FA77204606F0F6F918B9022004B0BDE8CB
:104DE000F09F00F0B7FF48B93DA14148FDF778FFBB
:104DF000E1B23F4805F0A2FE064614E000F0AAFF2B
:104E0000012806D03BA0FCF7CDFD00F02DFF0646A3
:104E100009E000F0A5FFB84205D93DA0FCF7C2FDAE
:104E200005F072F80646FCF7C7F880463DA1FBF78F
:104E3000AFF9002837D0FCF7C3F8834659463BA0AA
:104E4000FCF7B0FDFCF7BCF88346FCF7B5F8594613
:104E50000090FCF7D5FD002003900FF2E008FCF76E
:104E6000ABF8834603AA4146FBF7D2F9824603AA70
:104E700041460020FBF7CCF90290002001900FF290
:104E8000C00901AA49460298FBF7C2F901AA49469E
:104E90000020FBF7BDF98346FBF7B1FB287005F056
:104EA000B5FF064619E0FCF787F8804625A1FBF719
:104EB0006FF990B1FCF784F8804641461BA0FCF7DF
:104EC00071FDFCF77DF88046FCF776F88146414697
:104ED000FCF796FD00F0C8FE064630467EE700006F
:104EE00041542B5153434C4B3F0D0D0A0000000021
:104EF000B4150020B7B5BBD8BDE1B9FBB9FDC6DA22
:104F000031A3ACC7EBD6D8D6C3D7B4CCAC0D0A000E
:104F10004154D6B8C1EEB7B5BBD8B3ACCAB10D0ACF
:104F2000000000004F4B0D0A000000004154B7B5CF
:104F3000BBD83A2025640D0A000000000D0A0000CD
:104F40003A2000004552524F520D0A0070B50546F6
:104F5000002408E02846FFF735FF04461CB1044949
:104F60008868804700E0F5E700BF204670BD00007C
:104F7000E40000202DE9FE4F06460C4600270925D7
:104F80004FF4FA78284606F01DF910B90220BDE862
:104F9000FE8F00F0DFFE50B9324650A15448FDF7B5
:104FA0009FFEE9B2524805F0C9FD074694E000F0C3
:104FB000D1FE012806D04FA0FCF7F4FC00F054FE0F
:104FC000074689E000F0CCFE404506D950A0FCF72A
:104FD000E9FC04F099FF07467EE0FBF7EDFF814610
:104FE00050A1FBF7D5F800285CD0FBF7E9FF82461B
:104FF00051464EA0FCF7D6FCFBF7E2FF8246FBF7DA
:10500000DBFF83465146FCF7FBFC002002900FF2C9
:10501000DC09FBF7D1FF824602AA4946FBF7F8F804
:1050200002AA49460020FBF7F3F8019043A101983A
:10503000FBF7C7F810B9002020702BE0002000908B
:105040000FF2FC0A6A4651460198FBF7E1F86A46FE
:1050500051460020FBF7DCF86A4651460020FBF77A
:10506000D7F86A4651460020FBF7D2F86A46514607
:105070000020FBF7CDF86A4651460020FBF7C8F840
:105080006A4651460020FBF7C3F88346FBF7B7FAA0
:10509000207000BF21782CA0FCF784FC05F0B6FE40
:1050A000074619E0FBF788FF81462BA1FBF770F854
:1050B00090B1FBF785FF814649461CA0FCF772FCC6
:1050C000FBF77EFF8146FBF777FF82464946FCF7F8
:1050D00097FC00F0C9FD0746384658E741542B516C
:1050E0004953544154453D312C25640D0D0A0000AF
:1050F000B4150020B7B5BBD8BDE1B9FBB9FDC6DA20
:10510000A3ACC7EBD6D8D6C3D7B4CCAC0D0A00003D
:105110004154D6B8C1EEB7B5BBD8B3ACCAB10D0ACD
:10512000000000004F4B0D0A000000004154B7B5CD
:10513000BBD83A2025640D0A000000004F4B000048
:105140003A202C2200000000726573756C743A20BE
:1051500025640D0A000000004552524F520D0A000E
:1051600070B505460E46002409E031462846FFF793
:1051700001FF04461CB104498868804700E0F4E759
:1051800000BF204670BD0000E400002070B5002480
:10519000FBF712FF05460CA1FAF7FAFF90B1FBF7F7
:1051A0000FFF054629460AA0FCF7FCFBFBF708FFAA
:1051B0000546FBF701FF06462946FCF721FC0124C2
:1051C000FBF7ACFE204670BD0D0A5244590D0A0093
:1051D0004154B7B5BBD83A2025640D0A0000000041
:1051E0002DE9F04F8BB004460E4615460120FBF723
:1051F000DDFE4FF0000A0B2C06DD3FA0FCF7D2FBD2
:1052000002200BB0BDE8F08F224641A106A8FDF7B1
:1052100067FDFBF7D1FE074606A9FAF7B9FF00289C
:1052200067D0FBF7CDFE07463E480088874206DD83
:105230003C48078000F0C6FD3B49086058E03A480A
:10524000006800F0C5FD0A2852D93748006800F010
:10525000BFFD0190FBF7B4FE0090014633A0019A18
:10526000FCF7A0FB0020059037A00490FBF7A4FEFC
:1052700005AA01900499FAF7CBFF80464046FAF759
:1052800099FF00F0FF094246494630A0FCF78AFB2F
:10529000002003900FF2C40B03AA59464046FAF7C8
:1052A000B7FF03AA59460020FAF7B2FF03AA5946EE
:1052B0000020FAF7ADFF0A2200210190FBF766F902
:1052C000288009F104000290FBF776FE0299084459
:1052D00001902A8801463046FAF72AFF002011493A
:1052E0000880114908604FF0010AFBF717FE00BF64
:1052F00000BF504685E700007265637620706172DA
:10530000616D73206572726F72210D0A00000000DA
:105310002B51495552433A202272656376222C253F
:1053200064000000780100207C0100204154B7B5E2
:10533000BBD83A2025642C2074696D655F6469666A
:10534000663A2025640D0A000D0A00004C696E655E
:1053500031282564293A2025730D0A002C0000000D
:105360002DE9F0470746884691461C4600253B2616
:10537000A246304605F026FF10B90220BDE8F087AE
:1053800000F0E8FC18B9012005F076FC1FE000F001
:10539000E1FC012804D00FA0FCF704FB022516E075
:1053A00000F0DEFC504506D911A0FCF7FBFA04F032
:1053B000ABFD05460BE012484A464146436E38466F
:1053C00098470546012D02D105F020FD05462846E7
:1053D000D4E70000B7B5BBD8BDE1B9FBB9FDC6DA6B
:1053E000A3ACC7EBD6D8D6C3D7B4CCAC0D0A00005B
:1053F000B5C8B4FDCAB1BCE4B3ACCAB10D0A000073
:10540000E40000202DE9F04105460E461746984677
:1054100000240BE043463A4631462846FFF7A0FFFA
:1054200004461CB104498868804700E0F2E700BFE9
:105430002046BDE8F0810000E400002010B5002007
:1054400005F01AFC002005F0B3FB002005F01AFC63
:10545000FBF752FD10BD00002DE9F05F06460F4638
:1054600014464FF00008312542F21079284605F025
:10547000A9FE10B90220BDE8F09F00F06BFC58B9FE
:105480002346324647A14C48FDF72AFCE9B24A4878
:1054900005F054FB804682E000F05CFC012805D05A
:1054A00046A0FCF77FFA4FF0020878E000F058FCC5
:1054B000484506D948A0FCF775FA04F025FD80465A
:1054C0006DE0FBF779FD824648A1FAF761FEB0B1C5
:1054D000FBF776FD8246514645A0FCF763FAFBF7E1
:1054E0006FFD8246FBF768FD83465146FCF788FA5C
:1054F0002146384605F054FBFBF710FD4FE0FBF763
:105500005BFD82463EA1FAF743FE98B1FBF758FDDA
:105510008246514636A0FCF745FAFBF751FD82461C
:10552000FBF74AFD83465146FCF76AFA05F06EFC2C
:10553000804634E0FBF740FD824634A1FAF728FEAE
:1055400098B1FBF73DFD8246514629A0FCF72AFAA7
:10555000FBF736FD8246FBF72FFD83465146FCF7ED
:105560004FFA00F081FB804619E0FBF725FD8246EB
:1055700029A1FAF70DFE90B1FBF722FD82465146B4
:105580001BA0FCF70FFAFBF71BFD8246FBF714FD8F
:1055900083465146FCF734FA00F066FB80464046ED
:1055A00069E7000041542B514953454E443D256461
:1055B0002C25640D0D0A0000B4150020B7B5BBD82A
:1055C000BDE1B9FBB9FDC6DAA3ACC7EBD6D8D6C3EB
:1055D000D7B4CCAC0D0A00004154D6B8C1EEB7B573
:1055E000BBD8B3ACCAB10D0A000000003E200000D9
:1055F0004154B7B5BBD83A2025640D0A000000001D
:1056000053454E44204F4B0D0A00000053454E4475
:105610002046414C4C0D0A004552524F520D0A0093
:105620002DE9F04105460E46174600240AE03A46A9
:1056300031462846FFF710FF04461CB1044988682C
:10564000804700E0F3E700BF2046BDE8F08100009E
:10565000E40000202DE9F04704464FF0000804263E
:1056600014B94FF47A750AE0012C02D141F2883561
:1056700005E040A0FCF796F90220BDE8F087F0B203
:1056800005F0A0FD08B90220F7E700F063FB50B970
:1056900022463FA14248FDF723FBF1B2404805F006
:1056A0004DFA804663E000F055FB012806D03DA08E
:1056B000FCF778F900F0D8FA804658E000F050FB8B
:1056C000A84206D93EA0FCF76DF904F01DFC804607
:1056D0004DE0FBF771FC07463EA1FAF759FD60B3B8
:1056E000FBF76EFC07463D480088874206DD3B48D5
:1056F000078000F067FB3A4908601DE03848006801
:1057000000F066FB0A2817D9FBF75AFC8146494688
:1057100034A0FCF747F9FBF753FC8146FBF74CFC40
:1057200082464946FCF76CF900202C4908802C4938
:10573000086005F06BFB804619E0FBF73DFC07466F
:105740002CA1FAF725FD90B1FBF73AFC0746394644
:1057500024A0FCF727F9FBF733FC0746FBF72CFCEA
:1057600081463946FCF74CF900F07EFA8046404607
:1057700083E700007365745F6366756E2070617205
:10578000616D73206572726F72210D0A0000000056
:1057900041542B4346554E3D25640D0D0A00000033
:1057A000B4150020B7B5BBD8BDE1B9FBB9FDC6DA69
:1057B000A3ACC7EBD6D8D6C3D7B4CCAC0D0A000087
:1057C0004154D6B8C1EEB7B5BBD8B3ACCAB10D0A17
:1057D000000000004F4B0D0A000000007001002087
:1057E000740100204154B7B5BBD83A2025640D0A96
:1057F000000000004552524F520D0A0070B5054698
:10580000002408E02846FFF725FF04461CB10449A0
:105810008868804700E0F5E700BF204670BD0000C3
:10582000E40000202DE9F0470446002606254FF449
:10583000FA77022C05DD33A0FCF7B4F80220BDE8AE
:10584000F087E8B205F0BEFC08B90220F7E700F0E7
:1058500081FA50B9224632A13548FDF741FAE9B242
:10586000334805F06BF906464AE000F073FA012868
:1058700006D030A0FCF796F800F0F6F906463FE0B7
:1058800000F06EFAB84206D931A0FCF78BF804F0AC
:105890003BFB064634E0FBF78FFB804631A1FAF76D
:1058A00077FC98B1FBF78CFB804641462FA0FCF7B4
:1058B00079F8FBF785FB8046FBF77EFB8146414686
:1058C000FCF79EF805F0A2FA064619E0FBF774FB18
:1058D00080462AA1FAF75CFC90B1FBF771FB804689
:1058E000414622A0FCF75EF8FBF76AFB8046FBF717
:1058F00063FB81464146FCF783F800F0B5F90646A4
:1059000030469CE77365745F6367726567207061FA
:1059100072616D73206572726F72210D0A00000052
:1059200041542B43475245473D25640D0D0A000065
:10593000B4150020B7B5BBD8BDE1B9FBB9FDC6DAD7
:10594000A3ACC7EBD6D8D6C3D7B4CCAC0D0A0000F5
:105950004154D6B8C1EEB7B5BBD8B3ACCAB10D0A85
:10596000000000004F4B0D0A000000004154B7B585
:10597000BBD83A2025640D0A000000004552524F62
:10598000520D0A0070B50546002408E02846FFF7CE
:1059900049FF04461CB104498868804700E0F5E7E8
:1059A00000BF204670BD0000E40000202DE9F04754
:1059B000054600262D244FF4FA77204605F002FC18
:1059C00010B90220BDE8F08700F0C4F950B92A46AA
:1059D0002AA12E48FDF784F9E1B22C4805F0AEF873
:1059E000064648E000F0B6F9012804D028A0FBF7ED
:1059F000D9FF02263FE000F0B3F9B84206D92BA048
:105A0000FBF7D0FF04F080FA064634E0FBF7D4FA47
:105A100080462BA1FAF7BCFB98B1FBF7D1FA804680
:105A2000414629A0FBF7BEFFFBF7CAFA8046FBF709
:105A3000C3FA81464146FBF7E3FF05F0E7F9064666
:105A400019E0FBF7B9FA804623A1FAF7A1FB90B160
:105A5000FBF7B6FA804641461BA0FBF7A3FFFBF716
:105A6000AFFA8046FBF7A8FA81464146FBF7C8FF2C
:105A700000F0FAF806463046A4E7000041542B51E6
:105A8000495344453D25640D0D0A0000B41500201E
:105A9000B7B5BBD8BDE1B9FBB9FDC6DAA3ACC7EB5E
:105AA000D6D8D6C3D7B4CCAC0D0A00004154D6B872
:105AB000C1EEB7B5BBD8B3ACCAB10D0A0000000047
:105AC0004F4B0D0A000000004154B7B5BBD83A2037
:105AD00025640D0A000000004552524F520D0A0085
:105AE00070B50546002408E02846FFF75FFF04462E
:105AF0001CB104498868804700E0F5E700BF2046F4
:105B000070BD0000E40000202DE9F04705460026A6
:105B100002244FF4FA77204605F054FB10B9022016
:105B2000BDE8F08700F016F950B92A462BA12F489E
:105B3000FDF7D6F8E1B22D4805F000F806464AE038
:105B400000F008F9012806D029A0FBF72BFF00F090
:105B50008BF806463FE000F003F9B84206D92BA0C7
:105B6000FBF720FF04F0D0F9064634E0FBF724FAF7
:105B700080462BA1FAF70CFB98B1FBF721FA80467F
:105B8000414629A0FBF70EFFFBF71AFA8046FBF708
:105B900013FA81464146FBF733FF05F037F9064615
:105BA00019E0FBF709FA804623A1FAF7F1FA90B160
:105BB000FBF706FA804641461BA0FBF7F3FEFBF716
:105BC000FFF98046FBF7F8F981464146FBF718FFDD
:105BD00000F04AF806463046A2E7000041542B5137
:105BE00053434C4B3D25640D0D0A0000B4150020B5
:105BF000B7B5BBD8BDE1B9FBB9FDC6DAA3ACC7EBFD
:105C0000D6D8D6C3D7B4CCAC0D0A00004154D6B810
:105C1000C1EEB7B5BBD8B3ACCAB10D0A00000000E5
:105C20004F4B0D0A000000004154B7B5BBD83A20D5
:105C300025640D0A000000004552524F520D0A0023
:105C400070B50546002408E02846FFF75DFF0446CE
:105C50001CB104498868804700E0F5E700BF204692
:105C600070BD0000E400002010B5032005F004F82A
:105C7000022010BD2DE9F041064600253046FAF716
:105C800099FA0446E11704EB11710911A4EB011113
:105C900039B13046FAF78EFA00F00F00C0F1100566
:105CA00000E010253046FAF785FA87192A4629467A
:105CB0003846FAF74FFA2C442046BDE8F0812DE92A
:105CC000F04107460C4600262546E91705EB117101
:105CD0000911A5EB011149B12046E11704EB11713F
:105CE0000911A4EB0111C1F1100600E010263819CA
:105CF00032463146FAF72EFA35442846BDE8F0819F
:105D00002DE9F041064600253046FAF753FA0446DD
:105D1000E11704EB11710911A4EB011181B13046B7
:105D2000FAF748FA00F00F00C0F110053046FAF714
:105D300041FA87192A4629463846FAF70BFA2C44C5
:105D40002046BDE8F08100000148807870470000DF
:105D5000E40000200148007870470000E4000020C3
:105D60000148406870470000E40000202E20704782
:105D70002DE9F04105460E461746002405B116B937
:105D80000020BDE8F081AC685FB100E024688CB110
:105D9000206A78B13046216AFAF713FA0028F5D163
:105DA00008E000E024682CB13046216AFEF76EF965
:105DB0000028F7D10CB1206A08B90020E1E720469D
:105DC000DFE7000001480068704700001C00002069
:105DD000014607480068884203D305480068401A16
:105DE0007047C1F1FF30024A12681044F8E7000022
:105DF0001C00002010B50446214607A0FBF7D2FD89
:105E000003200B49087021460948401CFAF7E7F9BE
:105E1000182000F00FF810BD535445503A20CAFD29
:105E2000BEDDB7A2CBCDCAA7B0DC2C25730D0A000E
:105E3000C407002010B5044602498868804702481C
:105E4000047010BDE40000202400002070B504465A
:105E50000D460420FFF7EEFF02480560024804707B
:105E600070BD0000A40000202500002010B50446ED
:105E7000214607A0FBF796FD02200B49087021463A
:105E80000948401CFAF7ABF91720FFF7D3FF10BD04
:105E9000535445503A20CAFDBEDDB7A2CBCDB3C99D
:105EA000B9A62C25730D0A00C407002010B50446BE
:105EB000214602480078FFF7C9FF10BD24000020EA
:105EC00078B504460D46164600232A462146024868
:105ED0000096FBF741FD78BDC40500202DE9F04197
:105EE0000B3020F00706104D19E02068B04215D3A2
:105EF000B0420AD9871B201DD4F80480FAF718F99C
:105F0000A019C0E90078286004E060682860201DBE
:105F1000FAF70EF9201D2660BDE8F081251D2C68DA
:105F2000002CE2D10020F7E7B4010020F0B5C3B0A7
:105F300005460C464FF6FF70354908600846016873
:105F400034A0FBF72FFDFBF7DDF80020FBF714FA78
:105F50000220FBF7F1F82E49098888B2FBF7F2F826
:105F600035490320FBF7B0F9344801880720FBF7D7
:105F700091F933A10B20FBF7A7F932210C20FBF795
:105F800089F932211120FBF785F964212E48FAF7AF
:105F9000E8F82E482E492F4B2F4ACDE900102FA1AB
:105FA0002948FCF79DFE32213648FAF7DAF83648E0
:105FB000FAF700F906462448FAF7FCF80746324B90
:105FC000304A39462048009605F07FF84FF480713A
:105FD00003A8FAF7C6F81D481E491D4A294BCDE90A
:105FE000002102901C4A294903A8FCF779FE03A866
:105FF000FBF7A4F9FBF750F82080FBF753F80646AF
:10600000228831462846FAF793F843B0F0BD0000E5
:1060100084000020535445503A20C6B4BDD3C8CFA5
:10602000D6A4B1A8CEC42C7365714F66667365742F
:106030003D25640D0A000000C908002082000020F0
:106040006175746800000000100C002077000020CB
:10605000270000203B0000208D080020636C69654C
:106060006E74496425736465766963654E616D6518
:10607000257370726F647563744B657925737365EE
:1060800071257300740C00204F000020E4D8000834
:106090002DE9F047F6B005460E4617461C46574810
:1060A0000068401C554908600846016854A0FBF789
:1060B00079FC502162A8FAF754F8642149A8FAF74C
:1060C00050F85848584B59A26421009049A8FCF751
:1060D000F3FD49A957A0FBF765FC49A8FAF76AF850
:1060E000824662AA514649A805F054F81021564844
:1060F000FAF737F8102264A95348FAF719F8FBF7B2
:1061000001F80020FBF738F90220FBF715F83B49AE
:10611000098888B2FBF716F84C490320FBF7D4F83E
:106120004B4801880720FBF7B5F84AA10B20FBF785
:10613000CBF84AA10B20FBF7C7F849490B20FBF726
:10614000C3F848490B20FBF7BFF847A10B20FBF72A
:10615000BBF847A10B20FBF7B7F847A10B20FBF7D3
:10616000B3F832210C20FBF795F832211120FBF710
:1061700091F8434940F62800FBF7A6F80020469026
:1061800047904890142141A8F9F7EBFF0A2246A94D
:106190001A48006803F03AFE41AB46AA39492A483A
:1061A00004F009FF814641A940F62900FBF78CF86D
:1061B0004FF4807101A8F9F7D4FF01A833462A46AD
:1061C00030490090204804F03CFF804641462EA014
:1061D000FBF7E8FB1FFA88F101A8FBF795F8FAF73F
:1061E0005BFF2080FAF75EFF8246228851463846E0
:1061F000F9F79EFF76B0BDE8F0870000840000202C
:10620000535445503A20C6B4BDD3CAFDBEDDB1A833
:10621000CEC42C7365714F66667365743D25640D3D
:106220000A000000050900204F00002025732C25DE
:10623000730000007368613235365F736F75726387
:10624000653A2025730D0A004B0B0020C908002079
:1062500082000020746F706963000000737973001E
:10626000270000203B0000207468696E6700000072
:106270006D6F64656C00000075705F72617700007F
:10628000190900208A0000207061796C6F61645FD9
:106290006C656E6774683A2025640D0A0000000082
:1062A00010B50448F9F786FF08B1012010BD0020A1
:1062B000FCE7000019090020FCF706F8FCF746FC93
:1062C000FCF7A0FCFBF7AAF904F0F4FB01E004F0F2
:1062D00013FAFCE72DE9FF5F83468A461646984687
:1062E000DDE90E756FF06D0900BF00BF00BF00BF94
:1062F00000BF00BF00BF00BF00BF00BF06F00F001F
:1063000020B16FF0210004B0BDE8F09FBAF1000F9A
:1063100025D121E0102239466846F9F709FF2B46BE
:106320003A465146584600F03FF88146B9F1000F11
:1063300000D037E0002405E0285D18F8041048403C
:106340002855641C102CF7DB102269464046F9F7EB
:10635000EFFE10371035103E002EDBD11FE01CE0A1
:10636000002405E0385D18F8041048402855641CE6
:10637000102CF7DB2B462A465146584600F014F8FD
:106380008146B9F1000F00D00CE0102229464046AA
:10639000F9F7CEFE10371035103E002EE0D14FF049
:1063A000000900BF4846AEE72DE9F04107460C461C
:1063B00015461E4600BF00BF00BF00BF00BF00BFA4
:1063C00000BF00BF012C06D132462946384600F0F6
:1063D000D7FBBDE8F08132462946384600F08AF9FD
:1063E000F7E710B5044604B910BD4FF48C71204690
:1063F00003F05AFA00BFF7E710B5044600BF00BF2C
:106400004FF48C712046F9F7ACFE10BD2DE9F04F2A
:10641000C7B006468A46934600BF00BF00BF00BF14
:1064200001A8FFF7E9FF06F1080575605A465146D5
:1064300001A800F05FF85FEA000900D048E0019889
:106440003060DDE9011000EB011401CC01C501CC85
:1064500001C501CC01C501CC01C53068471E203CF7
:106460002BE04FF0000823E020781D49085C1D490F
:1064700051F820002188C1F30721194A515C1A4ABA
:1064800052F8211048402168C1F30741144A515C79
:10649000164A52F8211048402168090E104A515CF2
:1064A000134A52F82110484001C508F10108241D83
:1064B000B8F1040FD8DB7F1E203C002FD1DC01CCCB
:1064C00001C501CC01C501CC01C501CC01C500BF8E
:1064D00001A8FFF786FF484647B0BDE8F08F0000EF
:1064E00034B5000834C7000834CB000834CF0008A6
:1064F00034D30008F0B503460C46154600BF00BF74
:1065000000BF00BF802D05D0C02D06D0B5F5807F1F
:1065100009D105E00A20186008E00C20186005E0A9
:106520000E20186002E06FF01F00F0BD00BF03F105
:1065300008015960002216E014F82200012606EB3B
:106540008206A65D40EA0620022606EB8206A65DCC
:1065500040EA0640032606EB8206A65D40EA066096
:1065600041F82200521CB2EB551FE5D318680A28E7
:1065700004D00C2830D00E282DD163E0002228E072
:106580005A4E56F82260086870408E89C6F3072676
:10659000574FBE5D7040CE68C6F30746BE5D80EAC9
:1065A0000626C868000E385C86EA00400E7BBE5D99
:1065B00080EA066008610E694868704048614E696B
:1065C0008868704088618E69C8687040C861521CD4
:1065D00010310A2AD4D386E0002230E0434E56F828
:1065E0002260086870408E8AC6F30726404FBE5D61
:1065F00070404E69C6F30746BE5D80EA06264869CC
:10660000000E385C86EA00400E7DBE5D80EA0660C2
:1066100088618E6948687040C861CE69886870403A
:1066200008620E6AC868704048624E6A0869704025
:1066300088628E6A48697040C862521C1831082A04
:10664000CCD350E000224BE0284E56F82260086878
:1066500070408E8BC6F30726254FBE5D7040CE6915
:10666000C6F30746BE5D80EA0626C869000E385CA0
:1066700086EA00400E7FBE5D80EA066008620E6A10
:106680004868704048624E6A8868704088628E6AC6
:10669000C8687040C86291F82C60BE5D086970409F
:1066A0008E8DC6F30726BE5D80EA0620CE6AC6F34D
:1066B0000746BE5D80EA0646C86A000E385C86EA78
:1066C000006008630E6B4869704048634E6B8869D0
:1066D000704088638E6BC8697040C863521C20315B
:1066E000072AB1D300BF00BF00201EE734D700083F
:1066F00034B500082DE9F04188B007460D4616462E
:106700007C682878697840EA0120A97840EA01404D
:10671000E97840EA0160009001CC0099484000907F
:106720002879697940EA0120A97940EA0140E979AC
:1067300040EA0160019001CC019948400190287A1B
:10674000697A40EA0120A97A40EA0140E97A40EA00
:106750000160029001CC029948400290287B697B3D
:1067600040EA0120A97B40EA0140E97B40EA016060
:10677000039001CC03994840039001213868C1EB94
:106780006008E8E000BF01CC0099C9B2F74A52F8AE
:10679000211048400399C1F30721F54A52F821100E
:1067A00048400299C1F30741F24A52F8211048408B
:1067B0000199090EF04A52F821104840049001CC8A
:1067C0000199C9B2E94A52F8211048400099C1F331
:1067D0000721E74A52F8211048400399C1F30741C5
:1067E000E44A52F8211048400299090EE24A52F850
:1067F00021104840059001CC0299C9B2DB4A52F8F9
:10680000211048400199C1F30721D94A52F82110BB
:1068100048400099C1F30741D64A52F82110484038
:106820000399090ED44A52F821104840069001CC31
:106830000399C9B2CD4A52F8211048400299C1F3D8
:106840000721CB4A52F8211048400199C1F3074172
:10685000C84A52F8211048400099090EC64A52F819
:1068600021104840079000BF00BF01CC0499C9B275
:10687000BE4A52F821104840BDF81C10C1F3072150
:10688000BB4A52F8211048400699C1F30741B94A62
:1068900052F8211048400599090EB74A52F82110C4
:1068A0004840009001CC9DF81410B04A52F82110D5
:1068B00048400499C1F30721AD4A52F821104840DD
:1068C0000799C1F30741AB4A52F821104840069995
:1068D000090EA94A52F821104840019001CC9DF8B8
:1068E0001810A24A52F821104840BDF81410C1F304
:1068F00007219F4A52F8211048400499C1F30741EB
:106900009C4A52F8211048400799090E9A4A52F8B9
:1069100021104840029001CC9DF81C10934A52F877
:1069200021104840BDF81810C1F30721904A52F8D1
:10693000211048400599C1F307418E4A52F82110B1
:1069400048400499090E8C4A52F82110484003909F
:1069500000BFA8F10108B8F1000F3FF713AF00BF67
:1069600001CC0099C9B2814A52F8211048400399DC
:10697000C1F307217E4A52F8211048400299C1F321
:1069800007417C4A52F8211048400199090E7A4A81
:1069900052F821104840049001CC0199C9B2734AC1
:1069A00052F8211048400099C1F30721704A52F86B
:1069B000211048400399C1F307416E4A52F8211053
:1069C00048400299090E6C4A52F82110484005903F
:1069D00001CC0299C9B2654A52F821104840019988
:1069E000C1F30721624A52F8211048400099C1F3CF
:1069F0000741604A52F8211048400399090E5E4A47
:106A000052F821104840069001CC0399C9B2574A68
:106A100052F8211048400299C1F30721544A52F814
:106A2000211048400199C1F30741524A52F8211000
:106A300048400099090E504A52F8211048400790EA
:106A400000BF01CC0499C9B24C4A515C4840BDF822
:106A50001C10C1F30721515C80EA01210698C0F3A4
:106A60000740105C81EA00410598000E105C81EA45
:106A70000060009001CC9DF81410515C48400499CE
:106A8000C1F30721515C80EA01210798C0F3074058
:106A9000105C81EA00410698000E105C81EA0060FB
:106AA000019001CC9DF81810515C4840BDF81410BD
:106AB000C1F30721515C80EA01200499C1F3074129
:106AC000515C80EA01410798000E105C81EA006089
:106AD000029001CC9DF81C10515C4840BDF8181084
:106AE000C1F30721515C80EA01210598C0F30740FA
:106AF000105C81EA00410498000E105C81EA00609D
:106B00000390009830700098000A70700098000C94
:106B1000B0700098000EF070019830710198000A72
:106B200070710198000CB0710198000EF07102981C
:106B300030720298000A70720298000CB0720298CB
:106B4000000EF072039830730398000A7073039874
:106B5000000CB0730398000EF0732021684602F019
:106B6000A3FE002008B0BDE8F081000034C7000893
:106B700034CB000834CF000834D3000834C60008F2
:106B80002DE9F04188B007460D4616467C68287806
:106B9000697840EA0120A97840EA0140E97840EAB2
:106BA0000160009001CC00994840009028796979F3
:106BB00040EA0120A97940EA0140E97940EA016010
:106BC000019001CC019948400190287A697A40EA05
:106BD0000120A97A40EA0140E97A40EA0160029086
:106BE00001CC029948400290287B697B40EA012051
:106BF000A97B40EA0140E97B40EA0160039001CCB7
:106C000003994840039001213868C1EB6008E8E02F
:106C100000BF01CC0099C9B2F74A52F82110484090
:106C20000199C1F30721F54A52F821104840029911
:106C3000C1F30741F24A52F8211048400399090E66
:106C4000F04A52F821104840049001CC0199C9B291
:106C5000E94A52F8211048400299C1F30721E74A56
:106C600052F8211048400399C1F30741E44A52F811
:106C7000211048400099090EE24A52F8211048407C
:106C8000059001CC0299C9B2DB4A52F82110484064
:106C90000399C1F30721D94A52F8211048400099BD
:106CA000C1F30741D64A52F8211048400199090E14
:106CB000D44A52F821104840069001CC0399C9B239
:106CC000CD4A52F8211048400099C1F30721CB4A20
:106CD00052F8211048400199C1F30741C84A52F8BF
:106CE000211048400299090EC64A52F82110484026
:106CF000079000BF00BF01CC0499C9B2BE4A52F848
:106D000021104840BDF81410C1F30721BB4A52F8C6
:106D1000211048400699C1F30741B94A52F82110A1
:106D200048400799090EB74A52F821104840009090
:106D300001CC9DF81410B04A52F821104840BDF81B
:106D40001810C1F30721AD4A52F8211048400799A5
:106D5000C1F30741AA4A52F8211048400499090E8C
:106D6000A84A52F821104840019001CC9DF8181013
:106D7000A14A52F821104840BDF81C10C1F3072168
:106D80009E4A52F8211048400499C1F307419C4A99
:106D900052F8211048400599090E9A4A52F82110DC
:106DA0004840029001CC9DF81C10934A52F82110E3
:106DB00048400499C1F30721904A52F821104840F5
:106DC0000599C1F307418E4A52F8211048400699AF
:106DD000090E8C4A52F821104840039000BFA8F1D8
:106DE0000108B8F1000F3FF713AF00BF01CC0099C5
:106DF000C9B2814A52F8211048400199C1F30721D4
:106E00007E4A52F8211048400299C1F307417C4A5A
:106E100052F8211048400399090E7A4A52F821107D
:106E20004840049001CC0199C9B2734A52F821102C
:106E300048400299C1F30721704A52F82110484096
:106E40000399C1F307416E4A52F821104840009956
:106E5000090E6C4A52F821104840059001CC029965
:106E6000C9B2654A52F8211048400399C1F307217D
:106E7000624A52F8211048400099C1F30741604A24
:106E800052F8211048400199090E5E4A52F821102B
:106E90004840069001CC0399C9B2574A52F82110D4
:106EA00048400099C1F30721544A52F82110484044
:106EB0000199C1F30741524A52F821104840029902
:106EC000090E504A52F821104840079000BF01CCEB
:106ED0000499C9B24C4A515C4840BDF81410C1F342
:106EE0000721515C80EA01210698C0F30740105C3D
:106EF00081EA00410798000E105C81EA0060009072
:106F000001CC9DF81410515C4840BDF81810C1F335
:106F10000721515C80EA01210798C0F30740105C0B
:106F200081EA00410498000E105C81EA0060019043
:106F300001CC9DF81810515C4840BDF81C10C1F3FD
:106F40000721515C80EA01200499C1F30741515C9B
:106F500080EA01410598000E105C81EA0060029011
:106F600001CC9DF81C10515C48400499C1F30721E5
:106F7000515C80EA01210598C0F30740105C81EA6A
:106F800000410698000E105C81EA006003900098B2
:106F900030700098000A70700098000CB070009873
:106FA000000EF070019830710198000A707101981C
:106FB000000CB0710198000EF071029830720298C6
:106FC000000A70720298000CB0720298000EF07203
:106FD000039830730398000A70730398000CB07321
:106FE0000398000EF0732021684602F05DFC00203B
:106FF00008B0BDE8F081000034B6000834BA0008DB
:1070000034BE000834C2000834B5000830B597B06B
:1070100005460C4600BF00BF00BF00BF2078000639
:10702000617840EA0140A17840EA0120E178084314
:10703000029020790006617940EA0140A17940EA96
:107040000120E17908430390207A0006617A40EA42
:107050000140A17A40EA0120E17A08430490207BB4
:107060000006617B40EA0140A17B40EA0120E17B10
:1070700008430590207C0006617C40EA0140A17C29
:1070800040EA0120E17C08430690207D0006617DF6
:1070900040EA0140A17D40EA0120E17D08430790DC
:1070A000207E0006617E40EA0140A17E40EA012088
:1070B000E17E08430890207F0006617F40EA01409E
:1070C000A17F40EA0120E17F0843099094F8200065
:1070D000000694F8211040EA014094F8221040EA9A
:1070E000012094F8231008430A9094F82400000625
:1070F00094F8251040EA014094F8261040EA012057
:1071000094F8271008430B9094F82800000694F890
:10711000291040EA014094F82A1040EA012094F82E
:107120002B1008430C9094F82C00000694F82D10B6
:1071300040EA014094F82E1040EA012094F82F1004
:1071400008430D9094F83000000694F8311040EA9E
:10715000014094F8321040EA012094F833100843BB
:107160000E9094F83400000694F8351040EA01407F
:1071700094F8361040EA012094F8371008430F9035
:1071800094F83800000694F8391040EA014094F869
:107190003A1040EA012094F83B100843109094F80C
:1071A0003C00000694F83D1040EA014094F83E107F
:1071B00040EA012094F83F1008431190A86812900B
:1071C000E86813902869149068691590A86916906A
:1071D00000BF12984001129940EAD161DDE9140222
:1071E0005040139A1040159A50400844FE490844F4
:1071F0000299084416990844169013988007139929
:1072000040EA9100139000BF00BF16984001169904
:1072100040EAD161DDE913025040129A1040149AFD
:1072200050400844F0490144039808441599084423
:10723000159012988007129940EA9100129000BFB1
:1072400000BF15984001159940EAD161DDE91202AD
:107250005040169A1040139A50400844E2490144A5
:1072600004980844149908441490169880071699B5
:1072700040EA9100169000BF00BF14984001149995
:1072800040EAD161129A16985040159A1040129A0D
:1072900050400844D44901440598084413990844CF
:1072A000139015988007159940EA9100159000BF3A
:1072B00000BF13984001139940EAD161DDE915023E
:1072C0005040149A1040169A50400844C649014450
:1072D000069808441299084412901498800714994B
:1072E00040EA9100149000BF00BF1298400112992B
:1072F00040EAD161DDE914025040139A1040159A1A
:1073000050400844B8490144079808441699084475
:10731000169013988007139940EA9100139000BFCC
:1073200000BF16984001169940EAD161DDE91302C9
:107330005040129A1040149A50400844AA490144FF
:1073400008980844159908441590129880071299D6
:1073500040EA9100129000BF00BF159840011599B6
:1073600040EAD161DDE912025040169A1040139AAA
:10737000504008449C490144099808441499084421
:10738000149016988007169940EA9100169000BF55
:1073900000BF14984001149940EAD161129A1698DE
:1073A0005040159A1040129A504008448E490144AA
:1073B0000A98084413990844139015988007159962
:1073C00040EA9100159000BF00BF13984001139947
:1073D00040EAD161DDE915025040149A1040169A36
:1073E00050400844804901440B98084412990844CD
:1073F000129014988007149940EA9100149000BFED
:1074000000BF12984001129940EAD161DDE91402EF
:107410005040139A1040159A504008447249014454
:107420000C980844169908441690139880071399ED
:1074300040EA9100139000BF00BF169840011699D2
:1074400040EAD161DDE913025040129A1040149ACB
:1074500050400844644901440D9808441599084473
:10746000159012988007129940EA9100129000BF7F
:1074700000BF15984001159940EAD161DDE912027B
:107480005040169A1040139A5040084456490144FF
:107490000E98084414990844149016988007169979
:1074A00040EA9100169000BF00BF14984001149963
:1074B00040EAD161129A16985040159A1040129ADB
:1074C00050400844484901440F980844139908441F
:1074D000139015988007159940EA9100159000BF08
:1074E00000BF13984001139940EAD161DDE915020C
:1074F0005040149A1040169A504008443A490144AA
:10750000109808441299084412901498800714990E
:1075100040EA9100149000BF00BF129840011299F8
:1075200040EAD161DDE914025040139A1040159AE7
:10753000504008442C4901441198084416990844C5
:10754000169013988007139940EA9100139000BF9A
:1075500000BF16984001169940EAD161DDE9130297
:107560005040129A1040149A504008441E49421844
:107570000A990F9848400499484002994840019060
:1075800001984000019940EAD17002901044159989
:107590000844159012988007129940EA91001290C1
:1075A00000BF00BF15984001159940EAD161DDE99F
:1075B00012025040169A1040139A504008440A494B
:1075C000421810990B984840059948400399484043
:1075D000019001984000019940EAD171501803913F
:1075E00014990844149001E09979825A16988007FA
:1075F000169940EA9100169000BF00BF1498400110
:10760000149940EAD161129A16985040159A104088
:10761000129A50400844FE4942180C99119848406B
:10762000069948400499484001900198400001990A
:1076300040EAD17150180491139908441390159899
:107640008007159940EA9100159000BF00BF13987C
:107650004001139940EAD161DDE915025040149AC6
:107660001040169A50400844E94942180D99029872
:1076700048400799484005994840019001984000CA
:10768000019940EAD171501805911299084412905D
:1076900014988007149940EA9100149000BF00BF2D
:1076A00012984001129940EAD161DDE9130250407D
:1076B000159A50400844D749421803990E984840FB
:1076C0000899484006994840019001984000019966
:1076D00040EAD171501806911699084416901398F3
:1076E0008007139940EA9100139000BF00BF1698DD
:1076F0004001169940EAD161DDE912025040149A26
:1077000050400844C34942180F99049848400999C9
:10771000484007994840019001984000019940EA8B
:10772000D171501807911599084415901298800747
:10773000129940EA9100129000BF00BF15984001D5
:10774000159940EAD161129A16985040139A504008
:107750000844B04942181099059848400A99484091
:1077600008994840019001984000019940EAD17180
:107770005018089114990844149016988007169987
:1077800040EA9100169000BF00BF14984001149980
:1077900040EAD161DDE915025040129A5040084498
:1077A0009C4942181199069848400B9948400999FC
:1077B0004840019001984000019940EAD171501869
:1077C000099113990844139015988007159940EA78
:1077D0009100159000BF00BF13984001139940EA33
:1077E000D161DDE914025040169A5040084489499D
:1077F00042180299079848400C9948400A99484015
:10780000019001984000019940EAD17150180A9105
:1078100012990844129014988007149940EA910034
:10782000149000BF00BF12984001129940EAD16144
:10783000DDE913025040159A50400844754942183A
:107840000899039848400D9948400B994840019089
:1078500001984000019940EAD17150180B91169996
:107860000844169013988007139940EA91001390EA
:1078700000BF00BF16984001169940EAD161DDE9CA
:1078800012025040149A5040084462494218049928
:10789000099848400E9948400C9948400190019839
:1078A0004000019940EAD17150180C911599084493
:1078B000159012988007129940EA9100129000BF2B
:1078C00000BF15984001159940EAD161129A1698A7
:1078D0005040139A504008444E49421805990A985E
:1078E00048400F9948400D99484001900198400048
:1078F000019940EAD17150180D91149908441490DF
:1079000016988007169940EA9100169000BF00BFB4
:1079100014984001149940EAD161DDE91502504004
:10792000129A504008443B49421806990B98484027
:10793000109948400E9948400190019840000199E3
:1079400040EAD17150180E9113990844139015987C
:107950008007159940EA9100159000BF00BF139869
:107960004001139940EAD161DDE914025040169AB2
:10797000504008442749421807990C9848401199EB
:1079800048400F994840019001984000019940EA11
:10799000D17150180F9112990844129014988007D1
:1079A000149940EA9100149000BF00BF1298400162
:1079B000129940EAD161DDE913025040159A504016
:1079C00008441449421808990D98484002994840C3
:1079D00010994840019001984000019940EAD17106
:1079E000501810911699084416901398800713990F
:1079F00040EA9100139000BF00BF1698400116990D
:107A000040EAD161DDE912025040149A504003E08F
:107A10009979825AA1EBD96E0844FE4942180E9911
:107A200009984840039948401199484001900198AD
:107A30004000019940EAD1715018119115990844FC
:107A4000159012988007129940EA9100129000BF99
:107A500000BF15984001159940EAD161129A169815
:107A60005040139A50400844EA4942180A990F9826
:107A700048400499484002994840019001984000CC
:107A8000019940EAD170029010441499084414906E
:107A900016988007169940EA9100169000BF00BF23
:107AA00014984001149940EAD161DDE91502504073
:107AB000129A50400844D74942180B9910984840F0
:107AC0000599484003994840019001984000019968
:107AD00040EAD171501803911399084413901598F6
:107AE0008007159940EA9100159000BF00BF1398D8
:107AF0004001139940EAD161DDE914025040169A21
:107B000050400844C349421811990C9848400699BE
:107B1000484004994840019001984000019940EA8A
:107B2000D17150180491129908441290149880074A
:107B3000149940EA9100149000BF00BF12984001D0
:107B4000129940EAD161DDE913025040159A504084
:107B50000844B04942180D99029848400799484096
:107B600005994840019001984000019940EAD1717F
:107B70005018059116990844169013988007139988
:107B800040EA9100139000BF00BF1698400116997B
:107B900040EAD161DDE912025040149A5040084495
:107BA0009C4942180E990398484008994840069904
:107BB0004840019001984000019940EAD171501865
:107BC000069115990844159012988007129940EA79
:107BD0009100129000BF00BF15984001159940EA2E
:107BE000D161129A16985040139A5040084489491E
:107BF000421804990F98484009994840079948400D
:107C0000019001984000019940EAD1715018079104
:107C100014990844149016988007169940EA910028
:107C2000169000BF00BF14984001149940EAD1613A
:107C3000DDE915025040129A504008447549421837
:107C40000599109848400A99484008994840019081
:107C500001984000019940EAD17150180891139998
:107C60000844139015988007159940EA91001590E3
:107C700000BF00BF13984001139940EAD161DDE9CC
:107C800014025040169A5040084462494218119913
:107C9000069848400B99484009994840019001983E
:107CA0004000019940EAD171501809911299084495
:107CB000129014988007149940EA9100149000BF24
:107CC00000BFDDE913010840DDE913121143159AE5
:107CD0001140084312994901129A41EAD2610844BD
:107CE0004D4942180299079848400C9948400A9912
:107CF0004840019001984000019940EAD171501824
:107D00000A9116990844169013988007139940EA2F
:107D10009100139000BF00BFDDE912010840DDE9CA
:107D200012121143149A1140084316994901169AE8
:107D300041EAD261084438494218089903984840FA
:107D40000D9948400B9948400190019840000199D5
:107D500040EAD17150180B9115990844159012986A
:107D60008007129940EA9100129000BF00BF12995B
:107D700016980840129A16991143139A1140084315
:107D800015994901159A41EAD261084422494218DD
:107D90000499099848400E9948400C994840019030
:107DA00001984000019940EAD17150180C91149942
:107DB0000844149016988007169940EA910016908E
:107DC00000BF00BFDDE915010840DDE915121143D0
:107DD000129A1140084314994901149A41EAD26158
:107DE00008440D4942180A99059848400F9948409F
:107DF0000D994840019001984000019940EAD171E5
:107E000050180D91139908441390159880071599EF
:107E100004E00000A1EBD96EDCBC1B8F40EA9100AE
:107E2000159000BF00BFDDE914010840DDE9141220
:107E30001143169A1140084313994901139A41EAD4
:107E4000D2610844FE49421806990B98484010999F
:107E500048400E994840019001984000019940EA3D
:107E6000D17150180E9112990844129014988007FD
:107E7000149940EA9100149000BF00BFDDE913019E
:107E80000840DDE913121143159A11400843129975
:107E90004901129A41EAD2610844E94942180C9911
:107EA00007984840119948400F994840019001981F
:107EB0004000019940EAD17150180F911699084479
:107EC000169013988007139940EA9100139000BF11
:107ED00000BFDDE912010840DDE912121143149AD6
:107EE0001140084316994901169A41EAD2610844A3
:107EF000D349421808990D98484002994840109972
:107F00004840019001984000019940EAD171501811
:107F1000109115990844159012988007129940EA1B
:107F20009100129000BF00BF129916980840129A53
:107F300016991143139A1140084315994901159A4E
:107F400041EAD2610844BE4942180E990998484056
:107F500003994840119948400190019840000199C7
:107F600040EAD17150181191149908441490169850
:107F70008007169940EA9100169000BF00BFDDE926
:107F800015010840DDE915121143129A114008430A
:107F900014994901149A41EAD2610844A849421847
:107FA0000A990F9848400499484002994840019026
:107FB00001984000019940EAD17002901044139951
:107FC0000844139015988007159940EA9100159080
:107FD00000BF00BFDDE914010840DDE914121143C0
:107FE000169A1140084313994901139A41EAD26144
:107FF0000844934942180B99109848400599484005
:1080000003994840019001984000019940EAD171DC
:1080100050180391129908441290149880071499EB
:1080200040EA9100149000BF00BFDDE91301084051
:10803000DDE913121143159A1140084312994901C1
:10804000129A41EAD26108447D49421811990C986C
:1080500048400699484004994840019001984000E2
:10806000019940EAD171501804911699084416906C
:1080700013988007139940EA9100139000BF00BF46
:10808000DDE912010840DDE912121143149A114092
:10809000084316994901169A41EAD2610844684991
:1080A00042180D9902984840079948400599484060
:1080B000019001984000019940EAD1715018059152
:1080C00015990844159012988007129940EA91007A
:1080D000129000BF00BF129916980840129A169984
:1080E0001143139A1140084315994901159A41EA21
:1080F000D2610844524942180E99039848400899A1
:10810000484006994840019001984000019940EA92
:10811000D17150180691149908441490169880074C
:10812000169940EA9100169000BF00BFDDE91501E5
:108130000840DDE915121143129A114008431499C1
:108140004901149A41EAD26108443D494218049910
:108150000F98484009994840079948400190019874
:108160004000019940EAD1715018079113990844D1
:10817000139015988007159940EA9100159000BF5B
:1081800000BFDDE914010840DDE914121143169A1D
:108190001140084313994901139A41EAD2610844F6
:1081A000274942181099059848400A99484008996B
:1081B0004840019001984000019940EAD17150185F
:1081C000089112990844129014988007149940EA73
:1081D0009100149000BF00BFDDE913010840DDE904
:1081E00013121143159A1140084312994901129A2A
:1081F00041EAD26108441249421806991198484050
:108200000B99484009994840019001984000019914
:1082100040EAD171501809911699084416901398A4
:108220008007139940EA9100139000BF00BFDDE979
:1082300012010840DDE912121143149A114001E0C5
:10824000DCBC1B8F084316994901169A41EAD2619A
:108250000844FE4942180299079848400C99484042
:108260000A994840019001984000019940EAD17173
:1082700050180A9115990844159012988007129980
:1082800040EA9100129000BF00BF12991698084072
:10829000129A16991143139A1140084315994901EE
:1082A000159A41EAD2610844E849421803990898AE
:1082B00048400D9948400B99484001900198400072
:1082C000019940EAD17150180B9114990844149007
:1082D00016988007169940EA9100169000BF00BFDB
:1082E000DDE915010840DDE915121143129A11402C
:1082F000084314994901149A41EAD2610844D349C8
:1083000042180999049848400E9948400C994840F1
:10831000019001984000019940EAD17150180C91E8
:1083200013990844139015988007159940EA910015
:10833000159000BF00BFDDE914010840DDE914120B
:108340001143169A1140084313994901139A41EABF
:10835000D2610844BD49421805990A9848400F99CE
:1083600048400D994840019001984000019940EA29
:10837000D17150180D9112990844129014988007E9
:10838000149940EA9100149000BF00BF1298400178
:10839000129940EAD161DDE913025040159A50402C
:1083A0000844AB4942180B99069848401099484038
:1083B0000E994840019001984000019940EAD1711E
:1083C00050180E9116990844169013988007139927
:1083D00040EA9100139000BF00BF16984001169923
:1083E00040EAD161DDE912025040149A504008443D
:1083F0009749421807990C984840119948400F999D
:108400004840019001984000019940EAD17150180C
:108410000F9115990844159012988007129940EA17
:108420009100129000BF00BF15984001159940EAD5
:10843000D161129A16985040139A504008448449CA
:1084400042180D99089848400299484010994840B0
:10845000019001984000019940EAD17150181091A3
:1084600014990844149016988007169940EA9100D0
:10847000169000BF00BF14984001149940EAD161E2
:10848000DDE915025040129A5040084470494218E4
:1084900009990E9848400399484011994840019025
:1084A00001984000019940EAD17150181191139937
:1084B0000844139015988007159940EA910015908B
:1084C00000BF00BF13984001139940EAD161DDE974
:1084D00014025040169A504008445D4942180F99C2
:1084E0000A984840049948400299484001900198F0
:1084F0004000019940EAD17002901044129908445A
:10850000129014988007149940EA9100149000BFCB
:1085100000BF12984001129940EAD161DDE91302CF
:108520005040159A50400844494942180B991098F8
:1085300048400599484003994840019001984000FF
:10854000019940EAD1715018039116990844169088
:1085500013988007139940EA9100139000BF00BF61
:1085600016984001169940EAD161DDE912025040A7
:10857000149A504008443649421811990C984840C2
:10858000069948400499484001900198400001999B
:1085900040EAD17150180491159908441590129829
:1085A0008007129940EA9100129000BF00BF159811
:1085B0004001159940EAD161129A16985040139AD9
:1085C000504008442249421802990D9848400799A2
:1085D000484005994840019001984000019940EABF
:1085E000D171501805911499084414901698800779
:1085F000169940EA9100169000BF00BF1498400100
:10860000149940EAD161DDE915025040129A5040B8
:1086100008440F49421803990E9848400899484069
:1086200006994840019001984000019940EAD171B3
:1086300050180691139908441390159880071599BE
:1086400040EA9100159000BF00BF03E0DCBC1B8F27
:10865000D6C162CA13984001139940EAD161DDE99D
:1086600014025040169A50400844DE4942180F99AF
:10867000049848400999484007994840019001985A
:108680004000019940EAD1715018079112990844AD
:10869000129014988007149940EA9100149000BF3A
:1086A00000BF12984001129940EAD161DDE913023E
:1086B0005040159A50400844CA49421810990598EC
:1086C00048400A9948400899484001900198400064
:1086D000019940EAD17150180891169908441690F2
:1086E00013988007139940EA9100139000BF00BFD0
:1086F00016984001169940EAD161DDE91202504016
:10870000149A50400844B7494218119906984840B5
:108710000B994840099948400190019840000199FF
:1087200040EAD17150180991159908441590129892
:108730008007129940EA9100129000BF00BF15987F
:108740004001159940EAD161129A16985040139A47
:1087500050400844A34942180299079848400C9990
:1087600048400A994840019001984000019940EA28
:10877000D17150180A9114990844149016988007E2
:10878000169940EA9100169000BF00BF149840016E
:10879000149940EAD161DDE915025040129A504027
:1087A0000844904942180399089848400D99484058
:1087B0000B994840019001984000019940EAD1711D
:1087C00050180B9113990844139015988007159928
:1087D00040EA9100159000BF00BF13984001139923
:1087E00040EAD161DDE914025040169A5040084435
:1087F0007C4942180999049848400E9948400C99C0
:108800004840019001984000019940EAD171501808
:108810000C9112990844129014988007149940EA18
:108820009100149000BF00BF12984001129940EAD5
:10883000D161DDE913025040159A5040084469495E
:10884000421805990A9848400F9948400D994840A8
:10885000019001984000019940EAD17150180D91A2
:1088600016990844169013988007139940EA9100CE
:10887000139000BF00BF16984001169940EAD161DD
:10888000DDE912025040149A5040084455494218FC
:1088900006990B984840109948400E99484001901D
:1088A00001984000019940EAD17150180E91159934
:1088B0000844159012988007129940EA910012908E
:1088C00000BF00BF15984001159940EAD161129A86
:1088D00016985040139A504008444249421807994C
:1088E0000C984840119948400F99484001900198D0
:1088F0004000019940EAD17150180F911499084431
:10890000149016988007169940EA9100169000BFBF
:1089100000BF14984001149940EAD161DDE91502C5
:108920005040129A504008442E49421808990D9818
:1089300048400299484010994840019001984000F1
:10894000019940EAD171501810911399084413907D
:1089500015988007159940EA9100159000BF00BF57
:1089600013984001139940EAD161DDE914025040A7
:10897000169A504008441B49421809990E984840DD
:10898000039948401199484001900198400001998D
:1089900040EAD1715018119112990844129014981C
:1089A0008007149940EA9100149000BFA8681299BA
:1089B0000844A860E86813990144E960286914999B
:1089C000014429616869159901446961A86916998A
:1089D0000144A961582101A800F066FF002017B0EA
:1089E00030BD0000D6C162CAF0B5CBB006460D4618
:1089F00000BF00BF00BF00BF002407E006F1080071
:108A000050F8241043A840F82410641C082CF5D317
:108A1000002414E015F824000106A000401C285C86
:108A200041EA0041A000801C285C41EA0021A0002E
:108A3000C01C285C084303A941F82400641C102CC6
:108A4000E8D3002471E200BF479881099DF81C011A
:108A500041EA80604799CA0ABDF81C1142EA4151B7
:108A6000484047994A0E42EAC11148404A99421883
:108A700048994998484047990840499948401044C6
:108A8000FE4951F82410014403A850F8240008447A
:108A9000019043988008439940EA8170490B439ABA
:108AA00041EAC2414840910D41EA822180EA010237
:108AB000449943980840449B43991943459B194066
:108AC0000843104402900199469801444691DDE91B
:108AD000010101444A9100BF00BF469881099DF8F9
:108AE000180141EA80604699CA0ABDF8181142EAA5
:108AF0004151484046994A0E42EAC11148404999BD
:108B00004218479948984840469908404899484033
:108B10001118DA4A601C52F820000A1803A8611CD8
:108B200050F82100104401904A9881089DF82801CE
:108B300041EA80704A994A0BBDF8281142EAC141C6
:108B400048404A998A0D42EA812180EA010243990C
:108B50004A980840439B4A991943449B194008434B
:108B6000104402900199459801444591DDE90101C5
:108B70000144499100BF00BF459881099DF8140147
:108B800041EA80604599CA0ABDF8141142EA415190
:108B9000484045994A0E42EAC11148404899421856
:108BA00047994698484045990840479948401118C8
:108BB000B24AA01C52F820000A1803A8A11C50F8C1
:108BC000210010440190499881089DF8240141EA50
:108BD000807049994A0BBDF8241142EAC1414840CE
:108BE00049998A0D42EA812180EA01024A9949980D
:108BF00008404A9B49991943439B19400843104434
:108C000002900199449801444491DDE90101014435
:108C1000489100BF00BF449881099DF8100141EAC6
:108C200080604499CA0ABDF8101142EA4151484097
:108C300044994A0E42EAC111484047994218469960
:108C400045984840449908404699484011188B4A35
:108C5000E01C52F820000A1803A8E11C50F821007B
:108C600010440190489881089DF8200141EA8070E5
:108C700048994A0BBDF8201142EAC1414840489941
:108C80008A0D42EA812180EA010249994898084008
:108C9000499B489919434A9B194008431044029044
:108CA0000199439808444390DDE90101014447914B
:108CB00000BF00BF43988009439940EA8160C90A18
:108CC000439A41EA42514840510E41EAC21148409C
:108CD0004699421845994498484043990840459917
:108CE00048401118654A201D52F820000A1803A8B0
:108CF000211D50F8210010440190479881089DF8EB
:108D00001C0141EA807047994A0BBDF81C1142EAE8
:108D1000C141484047998A0D42EA812180EA010217
:108D2000489947980840489B47991943499B1940DF
:108D300008431044029001994A9801444A91DDE9A0
:108D400001010144469100BF00BF4A9881099DF886
:108D5000280141EA80604A99CA0ABDF8281142EA0E
:108D6000415148404A994A0E42EAC111484045994A
:108D700042184399449848404A99084044994840C9
:108D800011183E4A601D52F820000A1803A8611D00
:108D900050F8210010440190469881089DF8180170
:108DA00041EA807046994A0BBDF8181142EAC14168
:108DB000484046998A0D42EA812180EA010247999A
:108DC00046980840479B46991943489B19400843D9
:108DD000104402900199499801444991DDE901014B
:108DE0000144459100BF00BF499881099DF82401C5
:108DF00041EA80614998C20ABDF8240142EA405024
:108E0000484049994A0E42EAC111484044994218E3
:108E100043994A9848404999084043994840111855
:108E2000164AA01D52F820000A1803A8A11D50F8E8
:108E3000210010440190459881089DF8140141EAF1
:108E4000807045994A0BBDF8141142EAC14148406F
:108E500045998A0D42EA812180EA010246994598A6
:108E60000840469B45991943479B194008431044C5
:108E70000290019948980144489101E05CD70008AC
:108E8000DDE901010144449100BF00BF4898810918
:108E90009DF8200141EA80604899CA0ABDF8201176
:108EA00042EA4151484048994A0E42EAC1114840BD
:108EB000439942184A9949984840489908404A9924
:108EC00048401118FE4AE01D52F820000A1803A875
:108ED000E11D50F8210010440190449881089DF84C
:108EE000100141EA807044994A0BBDF8101142EA22
:108EF000C141484044998A0D42EA812180EA010239
:108F0000459944980840459B44991943469B19400C
:108F10000843104402900199479801444791DDE9C4
:108F200001010844439000BF0834102CFFF48BADBE
:108F30001024FDE300BFA01E03A951F82000420C3D
:108F4000A11E03A850F8210042EAC03003AA52F83B
:108F50002110CB0CA11E52F8211043EA41314840A8
:108F6000A11E52F8211080EA9122E11F03A850F8B7
:108F700021001044083903AA52F82110CB09A4F1AA
:108F80000F0112F8211043EA4161A4F10F0203AB73
:108F900053F82220970CA4F10F0253F8222047EA3D
:108FA00082325140A4F10F0253F8222081EAD2010B
:108FB0004218A4F1100103A850F82100024403A8AC
:108FC00040F82420479881099DF81C0141EA8060FF
:108FD0004799CB0ABDF81C1143EA415148404799D3
:108FE0004B0E43EAC11148404A99431849994898A1
:108FF000484047990840499948401844B04951F8B9
:10900000241008441044019043988008439940EA92
:109010008170490B439A41EAC2414840910D41EAAF
:10902000822180EA0102449943980840449B439975
:109030001943459B194008431044029001994698F2
:1090400001444691DDE9010101444A9100BF00BF9E
:10905000601E03A951F82000420C601E51F8200048
:1090600042EAC031601E03AA52F82000C30C601E01
:1090700052F8200043EA40304140601E52F8200080
:1090800081EA9022A01F03A951F820001118A4F131
:109090000E0003AA52F82000C309A4F10E0012F832
:1090A000200043EA4062A4F10E0003AB53F8200015
:1090B000870CA4F10E0053F8200047EA80304240AC
:1090C000A4F10E0053F8200082EAD0000A18A4F19F
:1090D0000F0003A951F82000024403A8611C40F8C6
:1090E0002120469881099DF8180141EA806046993F
:1090F000CB0ABDF8181143EA4151484046994B0E3E
:1091000043EAC11148404999431848994798484053
:1091100046990840489948401918694B601C53F813
:1091200020000844104401904A9881089DF82801C5
:1091300041EA80704A994A0BBDF8281142EAC141C0
:1091400048404A998A0D42EA812180EA0102439906
:109150004A980840439B4A991943449B1940084345
:10916000104402900199459801444591DDE90101BF
:109170000144499100BF00BF03A951F82400420CEB
:1091800003A850F8240042EAC03103AA52F8240090
:10919000C30C52F8240043EA4030414052F8240006
:1091A00081EA9022601F03A951F820001118A4F150
:1091B0000D0003AA52F82000C309A4F10D0012F813
:1091C000200043EA4062A4F10D0003AB53F82000F5
:1091D000870CA4F10D0053F8200047EA803042408C
:1091E000A4F10D0053F8200082EAD0000A18A4F17F
:1091F0000E0003A951F82000024403A8A11C40F866
:109200002120459881099DF8140141EA8060459923
:10921000CB0ABDF8141143EA4151484045994B0E21
:1092200043EAC11148404899431847994698484035
:1092300045990840479948401918214BA01C53F8FC
:109240002000084410440190499881089DF82401A9
:1092500041EA807049994A0BBDF8241142EAC141A4
:10926000484049998A0D42EA812180EA01024A99DF
:10927000499808404A9B49991943439B1940084320
:10928000104402900199449801444491DDE90101A0
:109290000144489100BF00BF601C03A951F82000A1
:1092A000420C601C51F8200042EAC031601C03AA45
:1092B00052F82000C30C601C52F8200002E00000AD
:1092C0005CD7000843EA40304140601C52F820005F
:1092D00081EA9022201F03A951F820001118A4F15F
:1092E0000C0003AA52F82000C309A4F10C0012F8E4
:1092F000200043EA4062A4F10C0003AB53F82000C5
:10930000870CA4F10C0053F8200047EA803042405B
:10931000A4F10C0053F8200082EAD0000A18A4F14E
:109320000D0003A951F82000024403A8E11C40F8F5
:109330002120449881099DF8100141EA80604499F8
:10934000CB0ABDF8101143EA4151484044994B0EF5
:1093500043EAC11148404799431845994698484007
:1093600044990840469948401918FE4BE01C53F8B0
:109370002000084410440190489881089DF820017D
:1093800041EA807048994A0BBDF8201142EAC14178
:10939000484048998A0D42EA812180EA01024999B0
:1093A00048980840499B489919434A9B19400843EB
:1093B000104402900199439808444390DDE901016B
:1093C0000144479100BF00BFA01C03A951F8200031
:1093D000420CA01C51F8200042EAC031A01C03AA94
:1093E00052F82000C30CA01C52F8200043EA403081
:1093F0004140A01C52F8200081EA9022E11E03A8FF
:1094000050F821001118A4F10B0003AA52F8200013
:10941000C309A4F10B0012F8200043EA4062A4F152
:109420000B0003AB53F82000870CA4F10B0053F89A
:10943000200047EA80304240A4F10B0053F820009E
:1094400082EAD0000A18A4F10C0003A951F8200008
:10945000024403A8211D40F8212043988009439924
:1094600040EA8160C90A439B41EA43514840590E92
:1094700041EAC311484046994318459944984840E9
:1094800043990840459948401918B64B201D53F898
:109490002000084410440190479881089DF81C0161
:1094A00041EA807047994A0BBDF81C1142EAC1415C
:1094B000484047998A0D42EA812180EA0102489991
:1094C00047980840489B47991943499B19400843CE
:1094D0001044029001994A9801444A91DDE9010142
:1094E0000144469100BF00BFE01C03A951F82000D1
:1094F000420CE11C03A850F8210042EAC031E01CF4
:1095000003AA52F82000C30CE01C52F8200043EAE2
:1095100040304140E01C52F8200081EA9022A01E19
:1095200003A951F820001118A4F10A0003AA52F867
:109530002000C309A4F10A0012F8200043EA4062A7
:10954000A4F10A0003AB53F82000870CA4F10A0031
:1095500053F8200047EA80304240A4F10A0053F853
:10956000200082EAD0000A18A4F10B0003A951F8E8
:109570002000024403A8611D40F821204A98810977
:109580009DF8280141EA80604A99CB0ABDF828116C
:1095900043EA415148404A994B0E43EAC1114840C1
:1095A000459943184399449848404A99084044993A
:1095B000484019186B4B601D53F8200008441044B4
:1095C0000190469881089DF8180141EA80704699FB
:1095D0004A0BBDF8181142EAC141484046998A0D2C
:1095E00042EA812180EA0102479946980840479B58
:1095F00046991943489B1940084310440290019929
:10960000499801444991DDE901010144459100BFB8
:1096100000BF201D03A951F82000420C201D51F865
:10962000200042EAC031201D03AA52F82000C30CDA
:10963000201D52F8200043EA40304140201D52F8DE
:10964000200081EA9022601E03A951F82000111821
:10965000A4F1090003AA52F82000C309A4F10900EB
:1096600012F8200043EA4062A4F1090003AB53F86A
:109670002000870CA4F1090053F8200047EA80304D
:109680004240A4F1090053F8200082EAD0000A18F1
:10969000A4F10A0003A951F82000024403A8A11D67
:1096A00040F82120499881099DF8240141EA806110
:1096B0004998C30ABDF8240143EA405048404999FB
:1096C0004B0E43EAC11148404499431843994A98C4
:1096D000484049990840439948401918214BA01D1A
:1096E00053F82000084410440190459881089DF8E3
:1096F000140141EA807045994A0BBDF8141142EA01
:10970000C141484045998A0D42EA812180EA01021F
:10971000469945980840469B45991943479B1940EF
:10972000084310440290019948980144489100E090
:109730009BE0DDE901010144449100BF00BF601DD1
:1097400003A951F82000420C601D51F8200042EAA4
:10975000C031601D03AA52F82000C30C601D52F8EE
:10976000200001E05CD7000843EA40304140601D22
:1097700052F8200081EA902203A951F82400111820
:10978000A4F1080003AA52F82000C309A4F10800BC
:1097900012F8200043EA4062A4F1080003AB53F83A
:1097A0002000870CA4F1080053F8200047EA80301D
:1097B0004240A4F1080053F8200082EAD0000A18C1
:1097C000A4F1090003A951F82000024403A8E11DF7
:1097D00040F82120489881099DF8200141EA8060E5
:1097E0004899CB0ABDF8201143EA415148404899B5
:1097F0004B0E43EAC11148404399431849994A988E
:109800004840489908404A9948401918254BE01D9E
:1098100053F82000084410440190449881089DF8B2
:10982000100141EA807044994A0BBDF8101142EAD8
:10983000C141484044998A0D42EA812180EA0102EF
:10984000459944980840459B44991943469B1940C3
:109850000843104402900199479801444791DDE97B
:1098600001010844439000BF0834402CFFF462AB70
:1098700000240CE006F1080050F8241043A850F82A
:109880002400014406F1080040F82410641C082C50
:10989000F0D34FF4947101A800F006F800204BB00B
:1098A000F0BD00005CD7000870B505460C4600BF4F
:1098B00000BF2CB1224600212846024B1B68984766
:1098C00070BD0000AC01002070B504460D4629466D
:1098D000204600F001F870BD2DE9F04704460D4622
:1098E0006FF06D0900BF00BF00BF00BF207800F01F
:1098F0003F0680223046761C04F11C010A54382EA3
:1099000007D8C6F1380104F11C029019F6F729FCBA
:1099100016E0C6F1400104F11C029019F6F721FC93
:1099200004F11C012046FDF771FB5FEA000902D03B
:109930004846BDE8F087382104F11C00F6F711FC19
:109940002068400F616840EAC10720684FEAC008FC
:10995000380E84F85400390C84F85510390A84F80C
:10996000561084F857704FEA186084F858004FEA90
:10997000184184F859104FEA182184F85A1084F8D5
:109980005B8004F11C012046FDF740FB5FEA000903
:1099900001D04846CDE7A068000E2870A068000CF2
:1099A00068702089000AA870207AE870E068000ECC
:1099B0002871E068000C6871A089000AA871207BFA
:1099C000E8712069000E28722069000C6872208AF4
:1099D000000AA872207CE8726069000E2873606932
:1099E000000C6873A08A000AA873207DE873A06940
:1099F000000E2874A069000C6874208B000AA874FB
:109A0000207EE874002094E710B5044600BF00BF34
:109A10005C212046F6F7A5FB10BD00B503461846AD
:109A200000F002F800BD0000014600BF00BF0020AA
:109A30000860486006488860064ACA60C2430A61F6
:109A4000044AD2434A61044A8A61002070470000F8
:109A50000123456789ABCDEFF0E1D2C370B5044671
:109A60000D46164632462946204600F001F870BDE4
:109A70002DE9F0470446884615466FF06D0900BF92
:109A800000BF00BF00BF15B90020BDE8F0872078F7
:109A900000F03F07C7F14006206828442060206896
:109AA00020602068A84202D26068401C6060AFB1AC
:109AB000B54213D304F11C01C81932464146F6F7EA
:109AC00037FB04F11C012046FDF7A0FA5FEA00090C
:109AD00001D04846D9E7B044AD1B00270BE0414612
:109AE0002046FDF793FA5FEA000901D04846CCE72B
:109AF00008F14008403D402DF1D235B104F11C0180
:109B0000C8192A464146F6F713FB0020BDE770B599
:109B100004460D462946204600F001F870BD2DE9A7
:109B2000F04704460D466FF06D0900BF00BF00BF4F
:109B300000BF207800F03F0680223046761C04F1FA
:109B400028010A54382E07D8C6F1380104F128023A
:109B50009019F6F706FB16E0C6F1400104F1280261
:109B60009019F6F7FEFA04F128012046FEF73CFFB3
:109B70005FEA000902D04846BDE8F087382104F1C9
:109B80002800F6F7EEFA2068400F616840EAC10746
:109B900020684FEAC008380E84F86000390C84F859
:109BA0006110390A84F8621084F863704FEA186013
:109BB00084F864004FEA184184F865104FEA1821D0
:109BC00084F8661084F8678004F128012046FEF7C7
:109BD0000BFF5FEA000901D04846CDE7A068000E00
:109BE0002870A068000C68702089000AA870207A8C
:109BF000E870E068000E2871E068000C6871A089C8
:109C0000000AA871207BE8712069000E2872206983
:109C1000000C6872208A000AA872207CE8726069D1
:109C2000000E28736069000C6873A08A000AA8738C
:109C3000207DE873A069000E2874A069000C687488
:109C4000208B000AA874207EE874E069000E287555
:109C5000E069000C6875A08B000AA875207FE87584
:109C6000206A000E2876206A000C6876208C000A94
:109C7000A8762020005DE876A06E58B9606A000ED4
:109C80002877606A000C6877A08C000AA8772420E7
:109C9000005DE87700206FE710B5044600BF00BF05
:109CA0006C212046F6F75DFA10BD30B504460D462E
:109CB0002946204600F002F830BD0000024600BFF1
:109CC00000BF00BF00BF00201060506081B9124883
:109CD0009060124BD360124B1361124B5361124BC5
:109CE0009361124BD361124B1362124B53620FE01C
:109CF00011489060114BD360114B1361114B5361AC
:109D0000114B9361114BD361114B1362114B536291
:109D1000916600207047000067E6096A85AE67BB60
:109D200072F36E3C3AF54FA57F520E518C68059B3D
:109D3000ABD9831F19CDE05BD89E05C107D57C3612
:109D400017DD703039590EF7310BC0FF1115586807
:109D5000A78FF964A44FFABE70B504460D461646A7
:109D600032462946204600F001F870BD2DE9F04743
:109D70000446884615466FF06D0900BF00BF00BF5E
:109D800000BF15B90020BDE8F087207800F03F073C
:109D9000C7F14006206828442060206820602068C1
:109DA000A84202D26068401C6060AFB1B54213D3D4
:109DB00004F12801C81932464146F6F7B9F904F111
:109DC00028012046FEF710FE5FEA000901D0484650
:109DD000D9E7B044AD1B00270BE041462046FEF713
:109DE00003FE5FEA000901D04846CCE708F14008CD
:109DF000403D402DF1D235B104F12801C8192A4661
:109E00004146F6F795F90020BDE700002DE9F04F37
:109E10008BB081460C469246282222A101A8F6F773
:109E200087F90026BAF10A0F09D1B9F1000F06DA55
:109E3000C9F100072D223046761C225400E04F461F
:109E400000BFB7FBFAF00AFB107001A90A5C3046AC
:109E5000761C2254B7FBFAF7002FF2D10020A05550
:109E600020782D2802D14FF0010801E04FF00008C2
:109E700045460CE014F805B0701E4044401B205CC1
:109E80006055701E4044401B04F800B06D1C701EED
:109E900000EBD071B5EB610FECDD20460BB0BDE8F7
:109EA000F08F0000303132333435363738394142A3
:109EB000434445464748494A4B4C4D4E4F505152FA
:109EC000535455565758595A000000000A48006824
:109ED000401C0949086009480068401C074908609F
:109EE00007484068401C0649486006480068401C16
:109EF0000449086070470000A0000020D400002042
:109F0000E40000201C00002010B5042000F0B4FE86
:109F1000022010BD2DE9F0478AB006460027002533
:109F2000202102A8F6F71DF964213348F6F719F944
:109F3000314CA41C082221463048F9F7A3FF2046E3
:109F4000F6F738F92EA109780155F6F7D5FF2D4817
:109F5000D0F8881002A888470746022F03D1384658
:109F60000AB0BDE8F0872046F6F724F900EB0408B4
:109F70001F2202A94046F6F7DBF8234800884FF479
:109F80007A7190FBF1F201FB12081F48008890FBE8
:109F9000F1F92046F6F70EF900EB040A4B461BA236
:109FA0000A215046CDF80080F8F786FE21461AA017
:109FB000F7F7F8FC1049891C1CA0F7F7F3FC0A23FB
:109FC00004221F491F48F7F7AFFF0A221C49204609
:109FD000F7F77DFA0546280A074908704D702046B4
:109FE000F6F7E8F880462A46414617A0F7F7DAFC6C
:109FF000A81C30700120B3E7241F0020840100203A
:10A0000026000000E40000208C0100202625642E9C
:10A010002530336400000000646576696365206460
:10A020006174613A25730D0A00000000726567696A
:10A03000737420646174613A25730D0A0000000096
:10A04000881F00208F0100207374726C656E64613C
:10A0500074613A25642C646174616C656E3D25649D
:10A060000D0A00002DE9F04180460C46002500272E
:10A07000E068B0F57A7F02D30020BDE8F081E068A7
:10A08000401CE060A1682068405C5B2800D05FE075
:10A09000A068401CA0602046F9F7F6FB4CB1D4E95B
:10A0A0000110884205D2A1682068405C5D2800D17B
:10A0B0003FE01CB1D4E90110884203D3A068401EE0
:10A0C000A06045E0A068401EA06000BF04F1100041
:10A0D000F9F749FF064606B93AE015B9354637465D
:10A0E00002E03E6077603746A068401CA0602046D2
:10A0F000F9F7CAFB2146384600F060FA00B927E0BC
:10A100002046F9F7C1FB44B1D4E90110884204D2DA
:10A11000A1682068405C2C28D8D044B1D4E9011053
:10A12000884204D2A1682068405C5D2800D00FE01E
:10A1300000BFE068401EE06005B16F602020C8F8F5
:10A140000C00C8F80850A068401CA060012094E7EB
:10A1500015B12846F9F7BEFE00208EE7024600231F
:10A16000002100BF23E0505C302806DB505C39281A
:10A1700003DC505C3038034415E0505C412806DBBA
:10A18000505C462803DC505C373803440BE0505CDD
:10A19000612806DB505C662803DC505C57380344BA
:10A1A00001E000207047032900D21B01491C04294B
:10A1B000D9D31846F6E700002DE9F04391B0804668
:10A1C0000C4600BF00201090FBF7D0FD8146002513
:10A1D0000CB1206818B9002011B0BDE8F08300254B
:10A1E0003CE0A16820680844405D342820D00ADCA7
:10A1F000A0F12B0009282ED2DFE800F0202D212A23
:10A200002D1617181900382816D006DC352810D05E
:10A2100036280FD037281ED10DE039280DD045281B
:10A220000FD0652817D10BE000BF00BF00BF00BFF3
:10A2300000BF00BF00BF00BF00BF00BF00BF00BF26
:10A2400000BFA16820680844405D0DF8050003E0E8
:10A250000DF8059000E00AE000BF6D1C3F2D05D20F
:10A2600024B1A068284461688842BAD300BF0020A6
:10A270000DF8050010A9684600F0BAFD06460F4625
:10A2800068461099884201D10020A5E7C8E9066711
:10A29000144A154B30463946F6F70EFB04D86FF0DA
:10A2A0000040C8F8140011E00022104B3046394637
:10A2B000F6F7EAFA04D84FF00040C8F8140005E0B9
:10A2C00030463946F6F7C1FAC8F814000820C8F835
:10A2D0000C00A0686A461099891A0844A060012001
:10A2E0007AE700000000C0FFFFFFDF410000E0C18F
:10A2F0002DE9F04180460C4600260025E068B0F5C7
:10A300007A7F02D30020BDE8F081E068401CE06065
:10A3100044B1D4E90110884204D2A1682068405CAD
:10A320007B2800D07DE0A068401CA0602046F9F7A3
:10A33000ABFA4CB1D4E90110884205D2A16820687B
:10A34000405C7D2800D15DE01CB1D4E90110884259
:10A3500003D3A068401EA06063E0A068401EA06018
:10A3600000BF04F11000F9F7FEFD074607B958E0F9
:10A3700016B93E463D4602E02F607D603D46A0682E
:10A38000401CA0602046F9F77FFA2146284600F0DD
:10A390004EF800B945E02046F9F776FA28692862B8
:10A3A0000020286144B1D4E90110884204D2A16898
:10A3B0002068405C3A2800D033E0A068401CA060D0
:10A3C0002046F9F761FA2146284600F0F7F800B96F
:10A3D00027E02046F9F758FA44B1D4E90110884241
:10A3E00004D2A1682068405C2C28BAD044B1D4E9DA
:10A3F0000110884204D2A1682068405C7D2800D00A
:10A400000FE000BFE068401EE06006B175604020CC
:10A41000C8F80C00C8F80860A068401CA0600120C3
:10A4200071E716B13046F9F755FD00206BE72DE9CD
:10A43000F84F80460C46A16820680844461CA16875
:10A4400020680844451C002000900027A16820686F
:10A45000405C222800D0A6E04FF0000AD1460DE073
:10A4600028785C2809D1681C2168401A61688842F4
:10A4700000D398E009F101096D1C6D1C2068281AB1
:10A480006168884202D228782228E9D12068281AF7
:10A490006168884202D22878222800D083E0A1682F
:10A4A00020680844281AA0EB090A0AF10100216972
:10A4B0008847074607B976E0009761E030785C2866
:10A4C00007D016F8010B009908700098401C009006
:10A4D00056E04FF00209A81B012800DA63E070780B
:10A4E000662819D008DC222832D02F2832D05C28E8
:10A4F0002FD0622840D108E06E2814D0722819D0DD
:10A5000074281ED0752837D12BE0082000990870D8
:10A510000098401C009030E00C20009908700098D2
:10A52000401C009029E00A20009908700098401C07
:10A53000009022E00D20009908700098401C0090C7
:10A540001BE00920009908700098401C009014E05E
:10A5500000BF00BF7078009908700098401C009000
:10A560000BE06A462946304600F056FC8146B9F1B8
:10A57000000F00D117E000E015E000BF4E4400BF1F
:10A58000AE429BD30020009908701020C8F80C0040
:10A59000C8F810702068281AA060A068401CA0604D
:10A5A0000120BDE8F88F17B138466169884716B1B8
:10A5B0002068301AA0600020F3E7000070B505465F
:10A5C0000C460CB1206808B9002070BD9CB1A06891
:10A5D000001D616888420ED8A2682168881804228C
:10A5E0003FA1F5F705FE30B90420E860A068001D22
:10A5F000A0600120E9E79CB1A068401D6168884225
:10A600000ED8A26821688818052237A1F5F7F0FD59
:10A6100030B90120E860A068401DA0600120D4E7A7
:10A62000ACB1A068001D6168884210D8A26821689A
:10A63000881804222EA1F5F7DBFD40B90220E8605E
:10A6400001206861A068001DA0600120BDE76CB119
:10A65000D4E90110884209D2A1682068405C222810
:10A6600004D121462846FFF7E2FEAEE7BCB1D4E9AB
:10A670000110884213D2A1682068405C2D2809D0BF
:10A68000A1682068405C302809DBA1682068405C34
:10A69000392804DC21462846FFF78EFD95E76CB18A
:10A6A000D4E90110884209D2A1682068405C5B2887
:10A6B00004D121462846FFF7D5FC86E76CB1D4E9E2
:10A6C0000110884209D2A1682068405C7B2804D12F
:10A6D00021462846FFF70CFE77E7002075E70000CB
:10A6E0006E756C6C0000000066616C7365000000A4
:10A6F000747275650000000010B5094890F86E008E
:10A7000000B910BD07480078012800D1F9E7F7F734
:10A7100039FAF7F721FEF6F70FFC00BFF1E700006A
:10A72000B4160020DC0000202DE9F04704008A4622
:10A7300016D054F8047CD4F800903E1F564500D93A
:10A7400056462046F8F7F6FA054688463246214630
:10A750005046FBF7C3FB40B1C0F80090BDE8F0875E
:10A76000BDE8F0470846F8F713BB44E9017955B155
:10A7700029686A18211F8A4202D9611B091F2960B2
:10A78000C5F80480EAE7024AC2F80080E6E7000064
:10A79000B40100202DE9F041ADF5027D05460E46DD
:10A7A00031462846F6F79DFC04464FF4807142A8D6
:10A7B000F5F7D7FC42AA31462846F6F777FC214642
:10A7C00039A0F7F7EFF844B932213C48F5F7C9FC56
:10A7D00000200DF5027DBDE8F0819DF808017B2881
:10A7E0004DD1601E42A9085C7D2848D142A8F9F7E6
:10A7F000C7FB804642AA214631A0F7F7D3F81421BF
:10A800003448F5F7AEFC32212C48F5F7AAFC32A10A
:10A810004046F9F79CFB48B12FA14046F9F78EFB63
:10A82000076939462B48F5F7DAFC00BF2CA14046F2
:10A83000F9F78DFB40B12AA14046F9F77FFB808AEA
:10A8400087B22A48076000BF29A14046F9F77FFB7D
:10A8500048B127A14046F9F771FB07693946174807
:10A86000F5F7BDFC00BF2148144A1A49036822A02D
:10A87000F7F798F84046F9F72DFB0120A9E74FF4C8
:10A88000807102A8F5F76DFC02A8234642AA1F4971
:10A8900000901F4800F056FB87B202AA39461DA05F
:10A8A000F7F780F8022094E77061796C6F6164B308
:10A8B000A4B6C83A2025640D0A000000190900203A
:10A8C000706C61696E74657874282564293A202556
:10A8D000730D0A000509002072616E646F6D00003F
:10A8E0007365714F66667365740000008400002014
:10A8F000746F6B656E0000000D0A2825732C2025EF
:10A90000732C202564290D0A000000008A00002015
:10A910004B0B00200D0A706C61696E7465787428A9
:10A920002564293A2025730D0A00000070B588B00F
:10A93000002006900490039000244B49086980474A
:10A940004948016A012088470446022C02D10020B0
:10A9500008B070BD4448816A012088470446022C33
:10A9600001D10020F4E74048016B022088470446EB
:10A97000022C01D10020EBE7002511E04FF4C87054
:10A98000F9F70EFC384803AB05AA07A9866B3748D0
:10A99000B04704469DF81C00012800D114256D1C09
:10A9A000142DEBDB022C01D10020D1E79DF81C0017
:10A9B00030B99DF81C102EA0F6F7F4FF0020C7E771
:10A9C00004A80121CDE900102748856C2B48038895
:10A9D0002B482CA102682C480078A8470446022C7A
:10A9E00005D1214629A0F6F7DDFF0020B0E7022CB3
:10A9F00001D10020ACE706A8FFF78CFA04469DF8C9
:10AA0000181026A0F6F7CEFF022C01D100209FE7F8
:10AA100015489DF818202649036E1B480078984772
:10AA20000446022C01D1002092E7F8F74BFE0446C1
:10AA3000022C01D100208BE70B48016D12480078F1
:10AA400088470446022C01D1002081E70648816A2C
:10AA5000002088470446022C01D1002078E70249F3
:10AA600008698047012073E7E40000208E01002080
:10AA700020737461743D25640D0A0000A801002054
:10AA8000A401002054435000A001002020726573EF
:10AA9000756C743D25640D0A0000000064617461EA
:10AAA000206C656E6774683D25640D0A0000000027
:10AAB000241F002038B50020174981F86E000024BB
:10AAC000084690F86E1015A0F6F76CFF6F22124939
:10AAD0001848F7F79FF90A20F9F762FB0E4890F83B
:10AAE0006E0001280DD10C4850300090503890F87D
:10AAF0006E1000F1320302460F48F6F753FF0120B3
:10AB000038BDFFF713FF04460CB90020F8E700F04A
:10AB1000DDF80120F4E70000B4160020B6C1C8A19A
:10AB2000C7B0726561645F666C61673A25640D0A3F
:10AB30000000000000E0070890D9000870B5054645
:10AB40000C462846F6F72EFF284600F01BF850B1B9
:10AB5000204600F02DF8012000F08EF8002000F0D3
:10AB600091F8002070BD02A0F6F71CFF0220F9E763
:10AB70004154D6B8C1EEB7A2CBCDCAA7B0DC0D0AFE
:10AB80000000000070B5044600250448007818B99C
:10AB90002046F6F7FFF90125284670BDC0010020C8
:10ABA00070B504460D4629462046F6F7E5F970BD16
:10ABB0000149488070470000E40000202DE9FF4370
:10ABC0000646884614461F464FF0000900200390B1
:10ABD0000290019000903D8826480088301A1FFAA4
:10ABE00080F92448068003AA01A94846F9F772FAB9
:10ABF00002AA69464046F9F78DFA9DF804109DF8BF
:10AC0000000061F31F10C2B22846691C8DB22254A5
:10AC10009DF804000D2806DBBDF80C00C2B22846E2
:10AC2000691C8DB222549DF804000E2807D1BDF88E
:10AC30000C00002002122846691C8DB222549DF897
:10AC400000000D2806DBBDF80800C2B22846691CCA
:10AC50008DB222549DF800000E2807D1BDF80800DF
:10AC6000002002122846691C8DB222543D80BDE8A6
:10AC7000FF830000E00000200149087070470000D9
:10AC8000E40000200149486070470000E400002013
:10AC900010B504461CB1206808B1A06808B10020B6
:10ACA00010BD7CB1A068001D616888420AD2A2680C
:10ACB00021688818032204A1F5F79AFA10B9A06850
:10ACC000C01CA0602046EBE7EFBBBF0010B50748F3
:10ACD0000078012802D100F01DF806E004A0F6F784
:10ACE00061FE00200A4981F86E0010BD800100203D
:10ACF000CAFDBEDDBDE2CEF6CAA7B0DCA3ACC3BBC5
:10AD0000D3D0B4E6B4A2666C6173680D0A0000008B
:10AD1000B416002008B501201A4981F86E000846D3
:10AD200090F86E0001F1500301F13202009016A07C
:10AD3000F6F738FE6F2123A0F6F734FE0A20F9F764
:10AD40002FFA6F220F492448F7F778F800200D49B1
:10AD500081F86E000A20F9F723FA20A0F6F722FE08
:10AD60006F2208491C48F7F755F806485030009004
:10AD7000503890F86E1000F1320302461B48F6F787
:10AD800011FE08BDB41600206465766963655365DD
:10AD9000637265743A25732C70726F647563744BBB
:10ADA00065793A25732C6465766963654E616D65D6
:10ADB0003A25732C726561645F666C61673A25643D
:10ADC0000D0A0000BDE1B9B9CCE5B4F3D0A13A2039
:10ADD00025640D0A0000000000E00708D0B4C8EBAD
:10ADE000CAFDBEDDCDEAB3C90D0A00004CD900088A
:10ADF00000B583B00A460021CDE90011014668463E
:10AE0000F5F781FEDDE9000103B000BD10B50220B9
:10AE1000FFF732FF012010BD2DE9FF5F8046894614
:10AE2000154600240026C246002003908346029067
:10AE30000190A9EB0A00062800DA81E00AF102007D
:10AE4000FFF78CF90646B6F55C4F03D3B6F5604FB5
:10AE500000D275E0B6F5584F29D3B6F55C4F26D22F
:10AE60000AF10607002000900C200290A9EB0700D1
:10AE7000062800DA64E038785C2802D178787528F2
:10AE800000D05DE0B81CFFF769F900900098B0F5BC
:10AE90005C4F03D30098B0F5604F00D350E0C6F389
:10AEA0000901009861F39F2000F5803402E006203C
:10AEB00002903446802C02D20120039018E0B4F5B1
:10AEC000006F04D202200390C020019010E0B4F57E
:10AED000803F04D203200390E020019008E0B4F505
:10AEE000881F04D204200390F020019000E027E0A6
:10AEF0000398401E00F0FF0B0BE004F0BF0040F091
:10AF00008000296801F80B00A409ABF1010000F0F2
:10AF1000FF0BBBF1000FF0DC0398012804DD019862
:10AF200020432968087003E004F07F002968087056
:10AF30002968039808442860029804B0BDE8F09F8F
:10AF40000020FAE72DE9F041CCB0054688461646C8
:10AF50001C46529F0020489049904A904B90E11720
:10AF600004EB11710911A4EB011129B1B4F5807F33
:10AF700002DD4CB0BDE8F0811022414648A8F5F74B
:10AF8000D7F802A8FBF738FA8022294602A8FBF777
:10AF90003DFA48AB2246002102A8CDE90067FBF745
:10AFA00099F93846F9F7D6F802A8FBF71AFA3846A5
:10AFB000F5F700F9DDE72DE9F043ADF50D7D054628
:10AFC0000F4614461E46002089908A908B908C90E4
:10AFD0004FF4807149A8F5F7C4F82046F5F7EAF870
:10AFE0001030B0F5807F04D900200DF50D7DBDE84F
:10AFF000F0831022394689A8F5F79AF82046F5F72C
:10B00000D9F881464A46214649A8F5F791F849A85A
:10B01000FAF730FE804603A8FBF7EEF980222946B6
:10B0200003A8FBF767FA49A889AB42460121CDE99D
:10B03000000603A8FBF74EF903A8FBF7D2F9404638
:10B04000D3E72DE9F043ADF50D7D05460F461646D5
:10B050001C46DDF85082002089908A908B908C905D
:10B060004FF4807149A8F5F77CF804F11000B0F5B1
:10B07000807F05DD4FF0FF300DF50D7DBDE8F083DD
:10B080001022394689A8F5F753F82246314649A8D7
:10B09000F5F74EF8214649A8FAF711FE814603A8B4
:10B0A000FBF7AAF98022294603A8FBF723FA49A84F
:10B0B00089AB4A460121CDE9000803A8FBF70AF94C
:10B0C00003A8FBF78EF94846D6E72DE9F043BDB05B
:10B0D0000546884616461F46DDF810910DB106B1AB
:10B0E00017B93DB0BDE8F083B9F1400F00DDF8E7D6
:10B0F000402116A8F5F735F8402106A8F5F731F8F4
:10B100004A46394616A8F5F713F84A46394606A8BE
:10B11000F5F70EF800240CE016A8005D80F036006C
:10B1200016A9085506A8005D80F05C0006A9085520
:10B13000641C402CF0DB26A8FEF766FC26A8FEF770
:10B140006CFC402216A926A8FEF788FC4246294638
:10B1500026A8FEF783FC01A926A8FEF7B5FB26A8C2
:10B16000FEF752FC26A8FEF758FC402206A926A8A6
:10B17000FEF774FC142201A926A8FEF76FFC01A9B2
:10B1800026A8FEF7A1FB1422314601A8F8F77AFEA3
:10B1900000BFA6E770B59CB004460D46164601A850
:10B1A000FEF77AFD002101A8FEF77FFD2A46214621
:10B1B00001A8FEF7D1FD314601A8FEF7A8FC1CB09E
:10B1C00070BD000010B50446FAF7BEFD18B1FAF7DD
:10B1D000BBFDA04201D1012010BD02A0F6F7E2FBA9
:10B1E0000020F9E76163746976654944202072653F
:10B1F0007065746974696F6E210D0A0010B50C4892
:10B20000007830B900200B49086001200849087017
:10B210000CE00848006808490968884206D90748D0
:10B220000078FAF707FE00200149087010BD000001
:10B230009E000020A0000020A40000202500002087
:10B240002DE9F04105460E461746002407E036F882
:10B2500014102846F6F7A2F9AD1C601C84B2BC425B
:10B26000F5DBBDE8F081014601F0800020B11B2034
:10B2700080EA4100C0B270474806000EFBE710B5F7
:10B2800004462046FFF7EFFF604010BD70B504464E
:10B290002046FFF7E8FF0546FFF7E5FF70BD70B5F4
:10B2A00004462046FFF7DFFF0646FFF7DCFF0546B2
:10B2B000FFF7D9FF70BD10B504462046FFF7EFFF3A
:10B2C000604010BD70B504462046FFF7E8FF054614
:10B2D0002046FFF7C8FF454085EA040070BD70B501
:10B2E00004462046FFF7DBFF05462046FFF7CEFF6A
:10B2F000454085EA040070BD70B504462046FFF75E
:10B30000CEFF05462046FFF7C1FF45402046FFF728
:10B31000AAFF684070BD00000100000000000000AE
:10B3200000000000010000000000637C777BF26BEE
:10B330006FC53001672BFED7AB76CA82C97DFA593B
:10B3400047F0ADD4A2AF9CA472C0B7FD9326363FA0
:10B35000F7CC34A5E5F171D8311504C723C318968D
:10B36000059A071280E2EB27B27509832C1A1B6E2F
:10B370005AA0523BD6B329E32F8453D100ED20FCD1
:10B38000B15B6ACBBE394A4C58CFD0EFAAFB434DD4
:10B39000338545F9027F503C9FA851A3408F929D71
:10B3A00038F5BCB6DA2110FFF3D2CD0C13EC5F9761
:10B3B0004417C4A77E3D645D197360814FDC222A67
:10B3C000908846EEB814DE5E0BDBE0323A0A49069E
:10B3D000245CC2D3AC629195E479E7C8376D8DD512
:10B3E0004EA96C56F4EA657AAE08BA78252E1CA6EA
:10B3F000B4C6E8DD741F4BBD8B8A703EB56648034A
:10B40000F60E613557B986C11D9EE1F8981169D9CC
:10B410008E949B1E87E9CE5528DF8CA1890DBFE64F
:10B42000426841992D0FB054BB1652096AD5303687
:10B43000A538BF40A39E81F3D7FB7CE339829B2FC5
:10B44000FF87348E4344C4DEE9CB547B9432A6C2DA
:10B45000233DEE4C950B42FAC34E082EA16628D927
:10B4600024B2765BA2496D8BD12572F8F6648668AA
:10B470009816D4A45CCC5D65B6926C704850FDED16
:10B48000B9DA5E154657A78D9D8490D8AB008CBC69
:10B49000D30AF7E45805B8B34506D02C1E8FCA3F2F
:10B4A0000F02C1AFBD0301138A6B3A9111414F677F
:10B4B000DCEA97F2CFCEF0B4E67396AC7422E7AD37
:10B4C0003585E2F937E81C75DF6E47F11A711D29E1
:10B4D000C5896FB7620EAA18BE1BFC563E4BC6D27A
:10B4E00079209ADBC0FE78CD5AF41FDDA833880797
:10B4F000C731B11210592780EC5F60517FA919B58F
:10B500004A0D2DE57A9F93C99CEFA0E03B4DAE2AF2
:10B51000F5B0C8EBBB3C83539961172B047EBA7717
:10B52000D626E169146355210C7D01020408102020
:10B5300040801B36637C777BF26B6FC53001672BD5
:10B54000FED7AB76CA82C97DFA5947F0ADD4A2AF17
:10B550009CA472C0B7FD9326363FF7CC34A5E5F125
:10B5600071D8311504C723C31896059A071280E2D3
:10B57000EB27B27509832C1A1B6E5AA0523BD6B327
:10B5800029E32F8453D100ED20FCB15B6ACBBE3997
:10B590004A4C58CFD0EFAAFB434D338545F9027F83
:10B5A000503C9FA851A3408F929D38F5BCB6DA213C
:10B5B00010FFF3D2CD0C13EC5F974417C4A77E3D68
:10B5C000645D197360814FDC222A908846EEB814BE
:10B5D000DE5E0BDBE0323A0A4906245CC2D3AC6281
:10B5E0009195E479E7C8376D8DD54EA96C56F4EA8C
:10B5F000657AAE08BA78252E1CA6B4C6E8DD741F9D
:10B600004BBD8B8A703EB5664803F60E613557B95F
:10B6100086C11D9EE1F8981169D98E949B1E87E919
:10B62000CE5528DF8CA1890DBFE6426841992D0FC8
:10B63000B054BB16C66363A5F87C7C84EE7777991B
:10B64000F67B7B8DFFF2F20DD66B6BBDDE6F6FB1BB
:10B6500091C5C5546030305002010103CE6767A91F
:10B66000562B2B7DE7FEFE19B5D7D7624DABABE667
:10B67000EC76769A8FCACA451F82829D89C9C940D5
:10B68000FA7D7D87EFFAFA15B25959EB8E4747C913
:10B69000FBF0F00B41ADADECB3D4D4675FA2A2FDDB
:10B6A00045AFAFEA239C9CBF53A4A4F7E472729603
:10B6B0009BC0C05B75B7B7C2E1FDFD1C3D9393AE67
:10B6C0004C26266A6C36365A7E3F3F41F5F7F70224
:10B6D00083CCCC4F6834345C51A5A5F4D1E5E53476
:10B6E000F9F1F108E2717193ABD8D873623131533B
:10B6F0002A15153F0804040C95C7C7524623236535
:10B700009DC3C35E30181828379696A10A05050F09
:10B710002F9A9AB50E070709241212361B80809BB8
:10B72000DFE2E23DCDEBEB264E2727697FB2B2CDBB
:10B73000EA75759F1209091B1D83839E582C2C7472
:10B74000341A1A2E361B1B2DDC6E6EB2B45A5AEE0A
:10B750005BA0A0FBA45252F6763B3B4DB7D6D66118
:10B760007DB3B3CE5229297BDDE3E33E5E2F2F71FB
:10B7700013848497A65353F5B9D1D1680000000013
:10B78000C1EDED2C40202060E3FCFC1F79B1B1C875
:10B79000B65B5BEDD46A6ABE8DCBCB4667BEBED9C5
:10B7A0007239394B944A4ADE984C4CD4B05858E818
:10B7B00085CFCF4ABBD0D06BC5EFEF2A4FAAAAE501
:10B7C000EDFBFB16864343C59A4D4DD76633335583
:10B7D000118585948A4545CFE9F9F91004020206DE
:10B7E000FE7F7F81A05050F0783C3C44259F9FBA5B
:10B7F0004BA8A8E3A25151F35DA3A3FE804040C033
:10B80000058F8F8A3F9292AD219D9DBC703838483C
:10B81000F1F5F50463BCBCDF77B6B6C1AFDADA7513
:10B820004221216320101030E5FFFF1AFDF3F30ED3
:10B83000BFD2D26D81CDCD4C180C0C14261313350C
:10B84000C3ECEC2FBE5F5FE1359797A2884444CCF0
:10B850002E17173993C4C45755A7A7F2FC7E7E82D2
:10B860007A3D3D47C86464ACBA5D5DE73219192B77
:10B87000E6737395C06060A0198181989E4F4FD187
:10B88000A3DCDC7F44222266542A2A7E3B9090ABC4
:10B890000B8888838C4646CAC7EEEE296BB8B8D3AE
:10B8A0002814143CA7DEDE79BC5E5EE2160B0B1D8D
:10B8B000ADDBDB76DBE0E03B64323256743A3A4E85
:10B8C000140A0A1E924949DB0C06060A4824246C15
:10B8D000B85C5CE49FC2C25DBDD3D36E43ACACEF39
:10B8E000C46262A6399191A8319595A4D3E4E43756
:10B8F000F279798BD5E7E7328BC8C8436E37375971
:10B90000DA6D6DB7018D8D8CB1D5D5649C4E4ED25C
:10B9100049A9A9E0D86C6CB4AC5656FAF3F4F40714
:10B92000CFEAEA25CA6565AFF47A7A8E47AEAEE90A
:10B93000100808186FBABAD5F07878884A25256FAC
:10B940005C2E2E72381C1C2457A6A6F173B4B4C703
:10B9500097C6C651CBE8E823A1DDDD7CE874749C72
:10B960003E1F1F21964B4BDD61BDBDDC0D8B8B86D1
:10B970000F8A8A85E07070907C3E3E4271B5B5C4F6
:10B98000CC6666AA904848D806030305F7F6F60188
:10B990001C0E0E12C26161A36A35355FAE5757F9AE
:10B9A00069B9B9D01786869199C1C1583A1D1D272A
:10B9B000279E9EB9D9E1E138EBF8F8132B9898B39C
:10B9C00022111133D26969BBA9D9D970078E8E892A
:10B9D000339494A72D9B9BB63C1E1E2215878792FD
:10B9E000C9E9E92087CECE49AA5555FF50282878C5
:10B9F000A5DFDF7A038C8C8F59A1A1F80989898092
:10BA00001A0D0D1765BFBFDAD7E6E631844242C68C
:10BA1000D06868B8824141C3299999B05A2D2D77D1
:10BA20001E0F0F117BB0B0CBA85454FC6DBBBBD61E
:10BA30002C16163AA5C6636384F87C7C99EE77775A
:10BA40008DF67B7B0DFFF2F2BDD66B6BB1DE6F6FB7
:10BA50005491C5C55060303003020101A9CE67671B
:10BA60007D562B2B19E7FEFE62B5D7D7E64DABAB63
:10BA70009AEC7676458FCACA9D1F82824089C9C9D1
:10BA800087FA7D7D15EFFAFAEBB25959C98E47470F
:10BA90000BFBF0F0EC41ADAD67B3D4D4FD5FA2A2D7
:10BAA000EA45AFAFBF239C9CF753A4A496E47272FF
:10BAB0005B9BC0C0C275B7B71CE1FDFDAE3D939363
:10BAC0006A4C26265A6C3636417E3F3F02F5F7F720
:10BAD0004F83CCCC5C683434F451A5A534D1E5E572
:10BAE00008F9F1F193E2717173ABD8D85362313137
:10BAF0003F2A15150C0804045295C7C76546232331
:10BB00005E9DC3C328301818A13796960F0A050505
:10BB1000B52F9A9A090E0707362412129B1B8080B4
:10BB20003DDFE2E226CDEBEB694E2727CD7FB2B2B7
:10BB30009FEA75751B1209099E1D838374582C2C6E
:10BB40002E341A1A2D361B1BB2DC6E6EEEB45A5A06
:10BB5000FB5BA0A0F6A452524D763B3B61B7D6D614
:10BB6000CE7DB3B37B5229293EDDE3E3715E2F2FF7
:10BB700097138484F5A6535368B9D1D1000000000F
:10BB80002CC1EDED604020201FE3FCFCC879B1B171
:10BB9000EDB65B5BBED46A6A468DCBCBD967BEBEC1
:10BBA0004B723939DE944A4AD4984C4CE8B0585814
:10BBB0004A85CFCF6BBBD0D02AC5EFEFE54FAAAAFD
:10BBC00016EDFBFBC5864343D79A4D4D556633337F
:10BBD00094118585CF8A454510E9F9F906040202DA
:10BBE00081FE7F7FF0A0505044783C3CBA259F9F57
:10BBF000E34BA8A8F3A25151FE5DA3A3C08040402F
:10BC00008A058F8FAD3F9292BC219D9D4870383838
:10BC100004F1F5F5DF63BCBCC177B6B675AFDADA0F
:10BC200063422121302010101AE5FFFF0EFDF3F3CF
:10BC30006DBFD2D24C81CDCD14180C0C3526131308
:10BC40002FC3ECECE1BE5F5FA2359797CC884444EC
:10BC5000392E17175793C4C4F255A7A782FC7E7ECE
:10BC6000477A3D3DACC86464E7BA5D5D2B32191973
:10BC700095E67373A0C0606098198181D19E4F4F83
:10BC80007FA3DCDC664422227E542A2AAB3B9090C0
:10BC9000830B8888CA8C464629C7EEEED36BB8B8AA
:10BCA0003C28141479A7DEDEE2BC5E5E1D160B0B89
:10BCB00076ADDBDB3BDBE0E0566432324E743A3A81
:10BCC0001E140A0ADB9249490A0C06066C48242411
:10BCD000E4B85C5C5D9FC2C26EBDD3D3EF43ACAC35
:10BCE000A6C46262A8399191A431959537D3E4E452
:10BCF0008BF2797932D5E7E7438BC8C8596E37376D
:10BD0000B7DA6D6D8C018D8D64B1D5D5D29C4E4E58
:10BD1000E049A9A9B4D86C6CFAAC565607F3F4F410
:10BD200025CFEAEAAFCA65658EF47A7AE947AEAE06
:10BD300018100808D56FBABA88F078786F4A2525A8
:10BD4000725C2E2E24381C1CF157A6A6C773B4B4FF
:10BD50005197C6C623CBE8E87CA1DDDD9CE874746E
:10BD6000213E1F1FDD964B4BDC61BDBD860D8B8BCD
:10BD7000850F8A8A90E07070427C3E3EC471B5B5F2
:10BD8000AACC6666D89048480506030301F7F6F684
:10BD9000121C0E0EA3C261615F6A3535F9AE5757AA
:10BDA000D069B9B9911786865899C1C1273A1D1D26
:10BDB000B9279E9E38D9E1E113EBF8F8B32B989898
:10BDC00033221111BBD2696970A9D9D989078E8E26
:10BDD000A7339494B62D9B9B223C1E1E92158787F9
:10BDE00020C9E9E94987CECEFFAA555578502828C1
:10BDF0007AA5DFDF8F038C8CF859A1A1800989898E
:10BE0000171A0D0DDA65BFBF31D7E6E6C684424288
:10BE1000B8D06868C3824141B0299999775A2D2DCD
:10BE2000111E0F0FCB7BB0B0FCA85454D66DBBBB1A
:10BE30003A2C161663A5C6637C84F87C7799EE7756
:10BE40007B8DF67BF20DFFF26BBDD66B6FB1DE6FB3
:10BE5000C55491C5305060300103020167A9CE6717
:10BE60002B7D562BFE19E7FED762B5D7ABE64DAB5F
:10BE7000769AEC76CA458FCA829D1F82C94089C9CD
:10BE80007D87FA7DFA15EFFA59EBB25947C98E470B
:10BE9000F00BFBF0ADEC41ADD467B3D4A2FD5FA2D3
:10BEA000AFEA45AF9CBF239CA4F753A47296E472FB
:10BEB000C05B9BC0B7C275B7FD1CE1FD93AE3D935F
:10BEC000266A4C26365A6C363F417E3FF702F5F71C
:10BED000CC4F83CC345C6834A5F451A5E534D1E56E
:10BEE000F108F9F17193E271D873ABD83153623133
:10BEF000153F2A15040C0804C75295C7236546232D
:10BF0000C35E9DC31828301896A13796050F0A0501
:10BF10009AB52F9A07090E0712362412809B1B80B0
:10BF2000E23DDFE2EB26CDEB27694E27B2CD7FB2B3
:10BF3000759FEA75091B1209839E1D832C74582C6A
:10BF40001A2E341A1B2D361B6EB2DC6E5AEEB45A02
:10BF5000A0FB5BA052F6A4523B4D763BD661B7D610
:10BF6000B3CE7DB3297B5229E33EDDE32F715E2FF3
:10BF70008497138453F5A653D168B9D1000000000B
:10BF8000ED2CC1ED20604020FC1FE3FCB1C879B16D
:10BF90005BEDB65B6ABED46ACB468DCBBED967BEBD
:10BFA000394B72394ADE944A4CD4984C58E8B05810
:10BFB000CF4A85CFD06BBBD0EF2AC5EFAAE54FAAF9
:10BFC000FB16EDFB43C586434DD79A4D335566337B
:10BFD0008594118545CF8A45F910E9F902060402D6
:10BFE0007F81FE7F50F0A0503C44783C9FBA259F53
:10BFF000A8E34BA851F3A251A3FE5DA340C080402B
:10C000008F8A058F92AD3F929DBC219D3848703834
:10C01000F504F1F5BCDF63BCB6C177B6DA75AFDA0B
:10C020002163422110302010FF1AE5FFF30EFDF3CB
:10C03000D26DBFD2CD4C81CD0C14180C1335261304
:10C04000EC2FC3EC5FE1BE5F97A2359744CC8844E8
:10C0500017392E17C45793C4A7F255A77E82FC7ECA
:10C060003D477A3D64ACC8645DE7BA5D192B32196F
:10C070007395E67360A0C060819819814FD19E4F7F
:10C08000DC7FA3DC226644222A7E542A90AB3B90BC
:10C0900088830B8846CA8C46EE29C7EEB8D36BB8A6
:10C0A000143C2814DE79A7DE5EE2BC5E0B1D160B85
:10C0B000DB76ADDBE03BDBE0325664323A4E743A7D
:10C0C0000A1E140A49DB9249060A0C06246C48240D
:10C0D0005CE4B85CC25D9FC2D36EBDD3ACEF43AC31
:10C0E00062A6C46291A8399195A43195E437D3E44E
:10C0F000798BF279E732D5E7C8438BC837596E3769
:10C100006DB7DA6D8D8C018DD564B1D54ED29C4E54
:10C11000A9E049A96CB4D86C56FAAC56F407F3F40C
:10C12000EA25CFEA65AFCA657A8EF47AAEE947AE02
:10C1300008181008BAD56FBA7888F078256F4A25A4
:10C140002E725C2E1C24381CA6F157A6B4C773B4FB
:10C15000C65197C6E823CBE8DD7CA1DD749CE8746A
:10C160001F213E1F4BDD964BBDDC61BD8B860D8BC9
:10C170008A850F8A7090E0703E427C3EB5C471B5EE
:10C1800066AACC6648D8904803050603F601F7F680
:10C190000E121C0E61A3C261355F6A3557F9AE57A6
:10C1A000B9D069B986911786C15899C11D273A1D22
:10C1B0009EB9279EE138D9E1F813EBF898B32B9894
:10C1C0001133221169BBD269D970A9D98E89078E22
:10C1D00094A733949BB62D9B1E223C1E87921587F5
:10C1E000E920C9E9CE4987CE55FFAA5528785028BD
:10C1F000DF7AA5DF8C8F038CA1F859A1898009898A
:10C200000D171A0DBFDA65BFE631D7E642C6844284
:10C2100068B8D06841C3824199B029992D775A2DC9
:10C220000F111E0FB0CB7BB054FCA854BBD66DBB16
:10C23000163A2C166363A5C67C7C84F8777799EE52
:10C240007B7B8DF6F2F20DFF6B6BBDD66F6FB1DEAF
:10C25000C5C5549130305060010103026767A9CE13
:10C260002B2B7D56FEFE19E7D7D762B5ABABE64D5B
:10C2700076769AECCACA458F82829D1FC9C94089C9
:10C280007D7D87FAFAFA15EF5959EBB24747C98E07
:10C29000F0F00BFBADADEC41D4D467B3A2A2FD5FCF
:10C2A000AFAFEA459C9CBF23A4A4F753727296E4F7
:10C2B000C0C05B9BB7B7C275FDFD1CE19393AE3D5B
:10C2C00026266A4C36365A6C3F3F417EF7F702F518
:10C2D000CCCC4F8334345C68A5A5F451E5E534D16A
:10C2E000F1F108F9717193E2D8D873AB313153622F
:10C2F00015153F2A04040C08C7C752952323654629
:10C30000C3C35E9D181828309696A13705050F0AFD
:10C310009A9AB52F0707090E1212362480809B1BAC
:10C32000E2E23DDFEBEB26CD2727694EB2B2CD7FAF
:10C3300075759FEA09091B1283839E1D2C2C745866
:10C340001A1A2E341B1B2D366E6EB2DC5A5AEEB4FE
:10C35000A0A0FB5B5252F6A43B3B4D76D6D661B70C
:10C36000B3B3CE7D29297B52E3E33EDD2F2F715EEF
:10C37000848497135353F5A6D1D168B90000000007
:10C38000EDED2CC120206040FCFC1FE3B1B1C87969
:10C390005B5BEDB66A6ABED4CBCB468DBEBED967B9
:10C3A00039394B724A4ADE944C4CD4985858E8B00C
:10C3B000CFCF4A85D0D06BBBEFEF2AC5AAAAE54FF5
:10C3C000FBFB16ED4343C5864D4DD79A3333556677
:10C3D000858594114545CF8AF9F910E902020604D2
:10C3E0007F7F81FE5050F0A03C3C44789F9FBA254F
:10C3F000A8A8E34B5151F3A2A3A3FE5D4040C08027
:10C400008F8F8A059292AD3F9D9DBC213838487030
:10C41000F5F504F1BCBCDF63B6B6C177DADA75AF07
:10C420002121634210103020FFFF1AE5F3F30EFDC7
:10C43000D2D26DBFCDCD4C810C0C14181313352600
:10C44000ECEC2FC35F5FE1BE9797A2354444CC88E4
:10C450001717392EC4C45793A7A7F2557E7E82FCC6
:10C460003D3D477A6464ACC85D5DE7BA19192B326B
:10C47000737395E66060A0C0818198194F4FD19E7B
:10C48000DCDC7FA3222266442A2A7E549090AB3BB8
:10C490008888830B4646CA8CEEEE29C7B8B8D36BA2
:10C4A00014143C28DEDE79A75E5EE2BC0B0B1D1681
:10C4B000DBDB76ADE0E03BDB323256643A3A4E7479
:10C4C0000A0A1E144949DB9206060A0C24246C4809
:10C4D0005C5CE4B8C2C25D9FD3D36EBDACACEF432D
:10C4E0006262A6C49191A8399595A431E4E437D34A
:10C4F00079798BF2E7E732D5C8C8438B3737596E65
:10C500006D6DB7DA8D8D8C01D5D564B14E4ED29C50
:10C51000A9A9E0496C6CB4D85656FAACF4F407F308
:10C52000EAEA25CF6565AFCA7A7A8EF4AEAEE947FE
:10C5300008081810BABAD56F787888F025256F4AA0
:10C540002E2E725C1C1C2438A6A6F157B4B4C773F7
:10C55000C6C65197E8E823CBDDDD7CA174749CE866
:10C560001F1F213E4B4BDD96BDBDDC618B8B860DC5
:10C570008A8A850F707090E03E3E427CB5B5C471EA
:10C580006666AACC4848D89003030506F6F601F77C
:10C590000E0E121C6161A3C235355F6A5757F9AEA2
:10C5A000B9B9D06986869117C1C158991D1D273A1E
:10C5B0009E9EB927E1E138D9F8F813EB9898B32B90
:10C5C000111133226969BBD2D9D970A98E8E89071E
:10C5D0009494A7339B9BB62D1E1E223C87879215F1
:10C5E000E9E920C9CECE49875555FFAA28287850B9
:10C5F000DFDF7AA58C8C8F03A1A1F8598989800986
:10C600000D0D171ABFBFDA65E6E631D74242C68480
:10C610006868B8D04141C3829999B0292D2D775AC5
:10C620000F0F111EB0B0CB7B5454FCA8BBBBD66D12
:10C6300016163A2C52096AD53036A538BF40A39E4B
:10C6400081F3D7FB7CE339829B2FFF87348E4344F1
:10C65000C4DEE9CB547B9432A6C2233DEE4C950B4D
:10C6600042FAC34E082EA16628D924B2765BA249AD
:10C670006D8BD12572F8F66486689816D4A45CCCCC
:10C680005D65B6926C704850FDEDB9DA5E1546579F
:10C69000A78D9D8490D8AB008CBCD30AF7E45805D5
:10C6A000B8B34506D02C1E8FCA3F0F02C1AFBD03E1
:10C6B00001138A6B3A9111414F67DCEA97F2CFCEB2
:10C6C000F0B4E67396AC7422E7AD3585E2F937E84D
:10C6D0001C75DF6E47F11A711D29C5896FB7620E8F
:10C6E000AA18BE1BFC563E4BC6D279209ADBC0FE70
:10C6F00078CD5AF41FDDA8338807C731B11210591D
:10C700002780EC5F60517FA919B54A0D2DE57A9F0E
:10C7100093C99CEFA0E03B4DAE2AF5B0C8EBBB3C03
:10C7200083539961172B047EBA77D626E169146387
:10C7300055210C7D51F4A7507E4165531A17A4C3AF
:10C740003A275E963BAB6BCB1F9D45F1ACFA58ABDD
:10C750004BE303932030FA55AD766DF688CC769195
:10C76000F5024C254FE5D7FCC52ACBD726354480AA
:10C77000B562A38FDEB15A4925BA1B6745EA0E9808
:10C780005DFEC0E1C32F7502814CF0128D4697A368
:10C790006BD3F9C6038F5FE715929C95BF6D7AEB5B
:10C7A000955259DAD4BE832D587421D349E06929B2
:10C7B0008EC9C84475C2896AF48E797899583E6BDF
:10C7C00027B971DDBEE14FB6F088AD17C920AC6660
:10C7D0007DCE3AB463DF4A18E51A3182975133604F
:10C7E00062537F45B16477E0BB6BAE84FE81A01CD1
:10C7F000F9082B94704868588F45FD1994DE6C87B2
:10C80000527BF8B7AB73D323724B02E2E31F8F570F
:10C810006655AB2AB2EB28072FB5C20386C57B9AB3
:10C82000D33708A5302887F223BFA5B202036ABA1E
:10C83000ED16825C8ACF1C2BA779B492F307F2F035
:10C840004E69E2A165DAF4CD0605BED5D134621F8A
:10C85000C4A6FE8A342E539DA2F355A0058AE13268
:10C86000A4F6EB750B83EC394060EFAA5E719F066E
:10C87000BD6E10513E218AF996DD063DDD3E05AEC6
:10C880004DE6BD4691548DB571C45D050406D46F67
:10C89000605015FF1998FB24D6BDE997894043CC19
:10C8A00067D99E77B0E842BD07898B88E7195B3866
:10C8B00079C8EEDBA17C0A477C420FE9F8841EC9E7
:10C8C0000000000009808683322BED481E1170ACF9
:10C8D0006C5A724EFD0EFFFB0F8538563DAED51ECD
:10C8E000362D39270A0FD964685CA6219B5B54D189
:10C8F00024362E3A0C0A67B19357E70FB4EE96D25E
:10C900001B9B919E80C0C54F61DC20A25A774B696A
:10C910001C121A16E293BA0AC0A02AE53C22E04390
:10C92000121B171D0E090D0BF28BC7AD2DB6A8B942
:10C93000141EA9C857F11985AF75074CEE99DDBBD8
:10C94000A37F60FDF701269F5C72F5BC44663BC582
:10C950005BFB7E348B432976CB23C6DCB6EDFC68CB
:10C96000B8E4F163D731DCCA4263851013972240E3
:10C9700084C61120854A247DD2BB3DF8AEF9321120
:10C98000C729A16D1D9E2F4BDCB230F30D8652ECF2
:10C9900077C1E3D02BB3166CA970B999119448FAFA
:10C9A00047E96422A8FC8CC4A0F03F1A567D2CD81D
:10C9B000223390EF87494EC7D938D1C18CCAA2FE25
:10C9C00098D40B36A6F581CFA57ADE28DAB78E2665
:10C9D0003FADBFA42C3A9DE45078920D6A5FCC9B8A
:10C9E000547E4662F68D13C290D8B8E82E39F75EB1
:10C9F00082C3AFF59F5D80BE69D0937C6FD52DA9B2
:10CA0000CF2512B3C8AC993B10187DA7E89C636E84
:10CA1000DB3BBB7BCD2678096E5918F4EC9AB70145
:10CA2000834F9AA8E6956E65AAFFE67E21BCCF08E3
:10CA3000EF15E8E6BAE79BD94A6F36CEEA9F09D4EC
:10CA400029B07CD631A4B2AF2A3F2331C6A5943099
:10CA500035A266C0744EBC37FC82CAA6E090D0B046
:10CA600033A7D815F104984A41ECDAF77FCD500E80
:10CA70001791F62F764DD68D43EFB04DCCAA4D547D
:10CA8000E49604DF9ED1B5E34C6A881BC12C1FB825
:10CA90004665517F9D5EEA04018C355DFA877473AB
:10CAA000FB0B412EB3671D5A92DBD252E91056336D
:10CAB0006DD647139AD7618C37A10C7A59F8148E2A
:10CAC000EB133C89CEA927EEB761C935E11CE5ED32
:10CAD0007A47B13C9CD2DF5955F2733F1814CE7996
:10CAE00073C737BF53F7CDEA5FFDAA5BDF3D6F1415
:10CAF0007844DB86CAAFF381B968C43E3824342C4D
:10CB0000C2A3405F161DC372BCE2250C283C498BB2
:10CB1000FF0D954139A80171080CB3DED8B4E49C2F
:10CB20006456C1907BCB8461D532B670486C5C741E
:10CB3000D0B857425051F4A7537E4165C31A17A489
:10CB4000963A275ECB3BAB6BF11F9D45ABACFA58D9
:10CB5000934BE303552030FAF6AD766D9188CC7691
:10CB600025F5024CFC4FE5D7D7C52ACB80263544A6
:10CB70008FB562A349DEB15A6725BA1B9845EA0E04
:10CB8000E15DFEC002C32F7512814CF0A38D469764
:10CB9000C66BD3F9E7038F5F9515929CEBBF6D7A57
:10CBA000DA9552592DD4BE83D35874212949E069AE
:10CBB000448EC9C86A75C28978F48E796B99583EDB
:10CBC000DD27B971B6BEE14F17F088AD66C920AC5C
:10CBD000B47DCE3A1863DF4A82E51A31609751334B
:10CBE0004562537FE0B1647784BB6BAE1CFE81A0CD
:10CBF00094F9082B58704868198F45FD8794DE6CAE
:10CC0000B7527BF823AB73D3E2724B0257E31F8F0B
:10CC10002A6655AB07B2EB28032FB5C29A86C57BAF
:10CC2000A5D33708F2302887B223BFA5BA02036A1A
:10CC30005CED16822B8ACF1C92A779B4F0F307F231
:10CC4000A14E69E2CD65DAF4D50605BE1FD1346286
:10CC50008AC4A6FE9D342E53A0A2F35532058AE164
:10CC600075A4F6EB390B83ECAA4060EF065E719F6A
:10CC700051BD6E10F93E218A3D96DD06AEDD3E05C2
:10CC8000464DE6BDB591548D0571C45D6F0406D463
:10CC9000FF605015241998FB97D6BDE9CC89404315
:10CCA0007767D99EBDB0E8428807898B38E7195B62
:10CCB000DB79C8EE47A17C0AE97C420FC9F8841EE3
:10CCC000000000008309808648322BEDAC1E1170F5
:10CCD0004E6C5A72FBFD0EFF560F85381E3DAED5C9
:10CCE00027362D39640A0FD921685CA6D19B5B5485
:10CCF0003A24362EB10C0A670F9357E7D2B4EE965A
:10CD00009E1B9B914F80C0C5A261DC20695A774B66
:10CD1000161C121A0AE293BAE5C0A02A433C22E08C
:10CD20001D121B170B0E090DADF28BC7B92DB6A83E
:10CD3000C8141EA98557F1194CAF7507BBEE99DDD4
:10CD4000FDA37F609FF70126BC5C72F5C544663B7E
:10CD5000345BFB7E768B4329DCCB23C668B6EDFCC7
:10CD600063B8E4F1CAD731DC1042638540139722DF
:10CD70002084C6117D854A24F8D2BB3D11AEF9321C
:10CD80006DC729A14B1D9E2FF3DCB230EC0D8652EE
:10CD9000D077C1E36C2BB31699A970B9FA119448F6
:10CDA0002247E964C4A8FC8C1AA0F03FD8567D2C19
:10CDB000EF223390C787494EC1D938D1FE8CCAA221
:10CDC0003698D40BCFA6F58128A57ADE26DAB78E61
:10CDD000A43FADBFE42C3A9D0D5078929B6A5FCC86
:10CDE00062547E46C2F68D13E890D8B85E2E39F7AD
:10CDF000F582C3AFBE9F5D807C69D093A96FD52DAE
:10CE0000B3CF25123BC8AC99A710187D6EE89C6380
:10CE10007BDB3BBB09CD2678F46E591801EC9AB741
:10CE2000A8834F9A65E6956E7EAAFFE60821BCCFDF
:10CE3000E6EF15E8D9BAE79BCE4A6F36D4EA9F09E8
:10CE4000D629B07CAF31A4B2312A3F2330C6A59495
:10CE5000C035A26637744EBCA6FC82CAB0E090D042
:10CE60001533A7D84AF10498F741ECDA0E7FCD507C
:10CE70002F1791F68D764DD64D43EFB054CCAA4D79
:10CE8000DFE49604E39ED1B51B4C6A88B8C12C1F21
:10CE90007F466551049D5EEA5D018C3573FA8774A7
:10CEA0002EFB0B415AB3671D5292DBD233E9105669
:10CEB000136DD6478C9AD7617A37A10C8E59F81426
:10CEC00089EB133CEECEA92735B761C9EDE11CE52E
:10CED0003C7A47B1599CD2DF3F55F273791814CE92
:10CEE000BF73C737EA53F7CD5B5FFDAA14DF3D6F11
:10CEF000867844DB81CAAFF33EB968C42C38243449
:10CF00005FC2A34072161DC30CBCE2258B283C49AE
:10CF100041FF0D957139A801DE080CB39CD8B4E42B
:10CF2000906456C1617BCB8470D532B674486C5C1A
:10CF300042D0B857A75051F465537E41A4C31A1785
:10CF40005E963A276BCB3BAB45F11F9D58ABACFAD5
:10CF500003934BE3FA5520306DF6AD76769188CC8D
:10CF60004C25F502D7FC4FE5CBD7C52A44802635A2
:10CF7000A38FB5625A49DEB11B6725BA0E9845EA00
:10CF8000C0E15DFE7502C32FF012814C97A38D4660
:10CF9000F9C66BD35FE7038F9C9515927AEBBF6D53
:10CFA00059DA9552832DD4BE21D35874692949E0AA
:10CFB000C8448EC9896A75C27978F48E3E6B9958D7
:10CFC00071DD27B94FB6BEE1AD17F088AC66C92058
:10CFD0003AB47DCE4A1863DF3182E51A3360975147
:10CFE0007F45625377E0B164AE84BB6BA01CFE81C9
:10CFF0002B94F90868587048FD198F456C8794DEAA
:10D00000F8B7527BD323AB7302E2724B8F57E31F07
:10D01000AB2A66552807B2EBC2032FB57B9A86C5AB
:10D0200008A5D33787F23028A5B223BF6ABA020316
:10D03000825CED161C2B8ACFB492A779F2F0F3072D
:10D04000E2A14E69F4CD65DABED50605621FD13482
:10D05000FE8AC4A6539D342E55A0A2F3E132058A60
:10D06000EB75A4F6EC390B83EFAA40609F065E7166
:10D070001051BD6E8AF93E21063D96DD05AEDD3EBE
:10D08000BD464DE68DB591545D0571C4D46F04065F
:10D0900015FF6050FB241998E997D6BD43CC894011
:10D0A0009E7767D942BDB0E88B8807895B38E7195E
:10D0B000EEDB79C80A47A17C0FE97C421EC9F884DF
:10D0C0000000000086830980ED48322B70AC1E11F1
:10D0D000724E6C5AFFFBFD0E38560F85D51E3DAEC5
:10D0E0003927362DD9640A0FA621685C54D19B5B81
:10D0F0002E3A243667B10C0AE70F935796D2B4EE56
:10D10000919E1B9BC54F80C020A261DC4B695A7762
:10D110001A161C12BA0AE2932AE5C0A0E0433C2288
:10D12000171D121B0D0B0E09C7ADF28BA8B92DB63A
:10D13000A9C8141E198557F1074CAF75DDBBEE99D0
:10D1400060FDA37F269FF701F5BC5C723BC544667A
:10D150007E345BFB29768B43C6DCCB23FC68B6EDC3
:10D16000F163B8E4DCCAD7318510426322401397DB
:10D17000112084C6247D854A3DF8D2BB3211AEF918
:10D18000A16DC7292F4B1D9E30F3DCB252EC0D86EA
:10D19000E3D077C1166C2BB3B999A97048FA1194F2
:10D1A000642247E98CC4A8FC3F1AA0F02CD8567D15
:10D1B00090EF22334EC78749D1C1D938A2FE8CCA1D
:10D1C0000B3698D481CFA6F5DE28A57A8E26DAB75D
:10D1D000BFA43FAD9DE42C3A920D5078CC9B6A5F82
:10D1E0004662547E13C2F68DB8E890D8F75E2E39A9
:10D1F000AFF582C380BE9F5D937C69D02DA96FD5AA
:10D2000012B3CF25993BC8AC7DA71018636EE89C7C
:10D21000BB7BDB3B7809CD2618F46E59B701EC9A3D
:10D220009AA8834F6E65E695E67EAAFFCF0821BCDB
:10D23000E8E6EF159BD9BAE736CE4A6F09D4EA9FE4
:10D240007CD629B0B2AF31A423312A3F9430C6A591
:10D2500066C035A2BC37744ECAA6FC82D0B0E0903E
:10D26000D81533A7984AF104DAF741EC500E7FCD78
:10D27000F62F1791D68D764DB04D43EF4D54CCAA75
:10D2800004DFE496B5E39ED1881B4C6A1FB8C12C1D
:10D29000517F4665EA049D5E355D018C7473FA87A3
:10D2A000412EFB0B1D5AB367D25292DB5633E91065
:10D2B00047136DD6618C9AD70C7A37A1148E59F822
:10D2C0003C89EB1327EECEA9C935B761E5EDE11C2A
:10D2D000B13C7A47DF599CD2733F55F2CE7918148E
:10D2E00037BF73C7CDEA53F7AA5B5FFD6F14DF3D0D
:10D2F000DB867844F381CAAFC43EB968342C382445
:10D30000405FC2A3C372161D250CBCE2498B283CAA
:10D310009541FF0D017139A8B3DE080CE49CD8B427
:10D32000C190645684617BCBB670D5325C74486C16
:10D330005742D0B8F4A750514165537E17A4C31A81
:10D34000275E963AAB6BCB3B9D45F11FFA58ABACD1
:10D35000E303934B30FA5520766DF6ADCC76918889
:10D36000024C25F5E5D7FC4F2ACBD7C5354480269E
:10D3700062A38FB5B15A49DEBA1B6725EA0E9845FC
:10D38000FEC0E15D2F7502C34CF012814697A38D5C
:10D39000D3F9C66B8F5FE703929C95156D7AEBBF4F
:10D3A0005259DA95BE832DD47421D358E0692949A6
:10D3B000C9C8448EC2896A758E7978F4583E6B99D3
:10D3C000B971DD27E14FB6BE88AD17F020AC66C954
:10D3D000CE3AB47DDF4A18631A3182E55133609743
:10D3E000537F45626477E0B16BAE84BB81A01CFEC5
:10D3F000082B94F94868587045FD198FDE6C8794A6
:10D400007BF8B75273D323AB4B02E2721F8F57E303
:10D4100055AB2A66EB2807B2B5C2032FC57B9A86A7
:10D420003708A5D32887F230BFA5B223036ABA0212
:10D4300016825CEDCF1C2B8A79B492A707F2F0F329
:10D4400069E2A14EDAF4CD6505BED50634621FD17E
:10D45000A6FE8AC42E539D34F355A0A28AE132055C
:10D46000F6EB75A483EC390B60EFAA40719F065E62
:10D470006E1051BD218AF93EDD063D963E05AEDDBA
:10D48000E6BD464D548DB591C45D057106D46F045B
:10D490005015FF6098FB2419BDE997D64043CC890D
:10D4A000D99E7767E842BDB0898B8807195B38E75A
:10D4B000C8EEDB797C0A47A1420FE97C841EC9F8DB
:10D4C00000000000808683092BED48321170AC1EED
:10D4D0005A724E6C0EFFFBFD8538560FAED51E3DC1
:10D4E0002D3927360FD9640A5CA621685B54D19B7D
:10D4F000362E3A240A67B10C57E70F93EE96D2B452
:10D500009B919E1BC0C54F80DC20A261774B695A5E
:10D51000121A161C93BA0AE2A02AE5C022E0433C84
:10D520001B171D12090D0B0E8BC7ADF2B6A8B92D36
:10D530001EA9C814F119855775074CAF99DDBBEECC
:10D540007F60FDA301269FF772F5BC5C663BC54476
:10D55000FB7E345B4329768B23C6DCCBEDFC68B6BF
:10D56000E4F163B831DCCAD76385104297224013D7
:10D57000C61120844A247D85BB3DF8D2F93211AE14
:10D5800029A16DC79E2F4B1DB230F3DC8652EC0DE6
:10D59000C1E3D077B3166C2B70B999A99448FA11EE
:10D5A000E9642247FC8CC4A8F03F1AA07D2CD85611
:10D5B0003390EF22494EC78738D1C1D9CAA2FE8C19
:10D5C000D40B3698F581CFA67ADE28A5B78E26DA59
:10D5D000ADBFA43F3A9DE42C78920D505FCC9B6A7E
:10D5E0007E4662548D13C2F6D8B8E89039F75E2EA5
:10D5F000C3AFF5825D80BE9FD0937C69D52DA96FA6
:10D600002512B3CFAC993BC8187DA7109C636EE878
:10D610003BBB7BDB267809CD5918F46E9AB701EC39
:10D620004F9AA883956E65E6FFE67EAABCCF0821D7
:10D6300015E8E6EFE79BD9BA6F36CE4A9F09D4EAE0
:10D64000B07CD629A4B2AF313F23312AA59430C68D
:10D65000A266C0354EBC377482CAA6FC90D0B0E03A
:10D66000A7D8153304984AF1ECDAF741CD500E7F74
:10D6700091F62F174DD68D76EFB04D43AA4D54CC71
:10D680009604DFE4D1B5E39E6A881B4C2C1FB8C119
:10D6900065517F465EEA049D8C355D01877473FA9F
:10D6A0000B412EFB671D5AB3DBD25292105633E961
:10D6B000D647136DD7618C9AA10C7A37F8148E591E
:10D6C000133C89EBA927EECE61C935B71CE5EDE126
:10D6D00047B13C7AD2DF599CF2733F5514CE79188A
:10D6E000C737BF73F7CDEA53FDAA5B5F3D6F14DF09
:10D6F00044DB8678AFF381CA68C43EB924342C3841
:10D70000A3405FC21DC37216E2250CBC3C498B28A6
:10D710000D9541FFA80171390CB3DE08B4E49CD823
:10D7200056C19064CB84617B32B670D56C5C744812
:10D73000B85742D0010000000200000004000000C1
:10D740000800000010000000200000004000000061
:10D75000800000001B00000036000000982F8A4265
:10D7600091443771CFFBC0B5A5DBB5E95BC2563933
:10D77000F111F159A4823F92D55E1CAB98AA07D84B
:10D78000015B8312BE853124C37D0C55745DBE726E
:10D79000FEB1DE80A706DC9B74F19BC1C1699BE4EE
:10D7A0008647BEEFC69DC10FCCA10C246F2CE92D7E
:10D7B000AA84744ADCA9B05CDA88F97652513E98A2
:10D7C0006DC631A8C82703B0C77F59BFF30BE0C6A9
:10D7D0004791A7D55163CA0667292914850AB72737
:10D7E00038211B2EFC6D2C4D130D385354730A65D4
:10D7F000BB0A6A762EC9C281852C7292A1E8BFA2AB
:10D800004B661AA8708B4BC2A3516CC719E892D112
:10D81000240699D685350EF470A06A1016C1A41995
:10D82000086C371E4C774827B5BCB034B30C1C3994
:10D830004AAAD84E4FCA9C5BF36F2E68EE828F7453
:10D840006F63A5781478C8840802C78CFAFFBE906D
:10D85000EB6C50A4F7A3F9BEF27871C600404040CB
:10D8600040404040404041414141414040404040B3
:10D87000404040404040404040404040400502025F
:10D88000020202020202020202020202022020201E
:10D89000202020202020200202020202020290907A
:10D8A0009090909010101010101010101010101078
:10D8B00010101010101010100202020202028888CC
:10D8C00088888888080808080808080808080808D8
:10D8D00008080808080808080202020240000000C0
:10D8E0005DD800087B22636C69656E744964223AD6
:10D8F000222573222C227369676E6D6574686F64CC
:10D90000223A22686D616373686131222C22736947
:10D91000676E223A222573222C2270726F6475631F
:10D92000744B6579223A222573222C22646576692C
:10D9300063654E616D65223A222573222C22736540
:10D9400071223A222573227D00000000B6C1C8A1D1
:10D95000CDEAB3C9726561645F666C61673A25643C
:10D960002C6465766963655365637265743A2573E3
:10D970002C70726F647563744B65793A25732C64EF
:10D9800065766963654E616D653A25730D0A000021
:10D99000B6C1C8A1666C617368B3C9B9A672656186
:10D9A000645F666C61673A25642C0A646576696316
:10D9B000655365637265743A25732C0A2070726F23
:10D9C000647563744B65793A25732C0A64657669CE
:10D9D00063654E616D653A25730D0A003833333740
:10D9E0003233397966342E796963702E66756E002C
:10D9F00010DA000800000020C0010000A20E00089C
:10DA000038DB0008C0010020B82E0000F02D00080F
:10DA1000412D01020304043809060708090204061F
:10DA20000814D1900D0561317433716C554E446307
:10DA30005050104C544563617431636573686930AC
:10DA400030318021343932396137383836306636F2
:10DA5000363365633732653263333133613465653C
:10DA60006537616384363636633216A01135343338
:10DA700079686A79393761653766796667021F0A9E
:10DA800013912D1B0835041329A739BC41FBB004A1
:10DA9000C511133D54140859431B08490413C54DBF
:10DAA00014084D4F1408095B1408415C14085556BE
:10DAB0001408FD5714082558140885591408B94945
:10DAC0001408CD4B1B0875241361511B08693413CE
:10DAD0007D451408E9411B08210C1AAD241BE15AAD
:10DAE0005019541A213C1AE1241361531B080510E4
:10DAF0001ABD2813B9461B088D141AE1081A814C67
:10DB000013054C1B089D740114100B37383934353C
:10DB10003637380804101174756F72656E7A68694B
:10DB20006E656E67687561320213DCD924088B5606
:08DB30000B106701400000002A
:04000005080000ED02
:00000001FF
